 Brackets

 Timestamp is 5c3fd699 (Thu Jan 17 04:12:57 2019)

 Preferred load address is 0000000180000000

 Start         Length     Name                   Class
 0001:00000000 00000008H .CRT$XCA                CODE
 0001:00000008 00000008H .CRT$XCZ                CODE
 0001:00000010 00000008H .CRT$XIA                CODE
 0001:00000018 00000018H .CRT$XIC                CODE
 0001:00000030 00000008H .CRT$XIZ                CODE
 0001:00000038 00000008H .CRT$XPA                CODE
 0001:00000040 00000010H .CRT$XPX                CODE
 0001:00000050 00000008H .CRT$XPXA               CODE
 0001:00000058 00000008H .CRT$XPZ                CODE
 0001:00000060 00000008H .CRT$XTA                CODE
 0001:00000068 00000008H .CRT$XTZ                CODE
 0001:00000070 00000000H .gfids$y                CODE
 0001:00000070 00007430H .rdata                  CODE
 0001:000074a0 000001f4H .rdata$r                CODE
 0001:00007694 000002b4H .rdata$zzzdbg           CODE
 0001:00007948 00000008H .rtc$IAA                CODE
 0001:00007950 00000008H .rtc$IZZ                CODE
 0001:00007958 00000008H .rtc$TAA                CODE
 0001:00007960 00000010H .rtc$TZZ                CODE
 0001:00007970 0000d180H .text$mn                CODE
 0001:00014af0 00000020H .text$mn$00             CODE
 0001:00014b10 00000250H .text$x                 CODE
 0001:00014d60 00000b98H .xdata                  CODE
 0001:000158f8 000000f8H .xdata$x                CODE
 0001:000159f0 000000a6H .edata                  CODE
 0002:00000000 00000950H .data                   DATA
 0002:00000950 000000a0H .data$r                 DATA
 0002:000009f0 00001390H .bss                    DATA
 0003:00000000 00000ec4H .pdata                  DATA
 0004:00000000 00000248H .idata$5                DATA
 0004:00000248 00000010H .00cfg                  DATA
 0004:00000258 00000028H .idata$2                DATA
 0004:00000280 00000018H .idata$3                DATA
 0004:00000298 00000248H .idata$4                DATA
 0004:000004e0 00000534H .idata$6                DATA
 0005:00000000 00000060H .rsrc$01                DATA
 0005:00000060 00000380H .rsrc$02                DATA

  Address         Publics by Value              Rva+Base               Lib:Object

 0000:00000000       __guard_iat_count          0000000000000000     <absolute>
 0000:00000000       __dynamic_value_reloc_table 0000000000000000     <absolute>
 0000:00000000       __hybrid_code_map          0000000000000000     <absolute>
 0000:00000000       __hybrid_code_map_count    0000000000000000     <absolute>
 0000:00000000       __guard_iat_table          0000000000000000     <absolute>
 0000:00000000       __hybrid_auxiliary_iat     0000000000000000     <absolute>
 0000:00000000       __guard_longjmp_table      0000000000000000     <absolute>
 0000:00000000       __guard_longjmp_count      0000000000000000     <absolute>
 0000:00000000       __guard_fids_count         0000000000000000     <absolute>
 0000:00000000       __enclave_config           0000000000000000     <absolute>
 0000:00000000       ___safe_se_handler_table   0000000000000000     <absolute>
 0000:00000000       ___safe_se_handler_count   0000000000000000     <absolute>
 0000:00000000       __guard_fids_table         0000000000000000     <absolute>
 0000:00000100       __guard_flags              0000000000000100     <absolute>
 0000:00000000       __ImageBase                0000000180000000     <linker-defined>
 0001:00000000       __xc_a                     0000000180001000     LIBCMT:initializers.obj
 0001:00000008       __xc_z                     0000000180001008     LIBCMT:initializers.obj
 0001:00000010       __xi_a                     0000000180001010     LIBCMT:initializers.obj
 0001:00000018       __acrt_multibyte_initializer 0000000180001018     libucrt:multibyte_initializer.obj
 0001:00000020       __acrt_stdio_initializer   0000000180001020     libucrt:stdio_initializer.obj
 0001:00000028       __acrt_tran_fma3_initializer 0000000180001028     libucrt:fma3_initializer.obj
 0001:00000030       __xi_z                     0000000180001030     LIBCMT:initializers.obj
 0001:00000038       __xp_a                     0000000180001038     LIBCMT:initializers.obj
 0001:00000040       __acrt_locale_terminator   0000000180001040     libucrt:locale_initializer.obj
 0001:00000048       __dcrt_console_output_terminator 0000000180001048     libucrt:console_output_initializer.obj
 0001:00000050       __acrt_stdio_terminator    0000000180001050     libucrt:stdio_initializer.obj
 0001:00000058       __xp_z                     0000000180001058     LIBCMT:initializers.obj
 0001:00000060       __xt_a                     0000000180001060     LIBCMT:initializers.obj
 0001:00000068       __xt_z                     0000000180001068     LIBCMT:initializers.obj
 0001:00000070       MainGuid                   0000000180001070     Brackets.obj
 0001:00000080       MenuGuid                   0000000180001080     Brackets.obj
 0001:00000090       DialogGuid                 0000000180001090     Brackets.obj
 0001:000000a0       ??_7?$DialogItemBinding@UFarDialogItem@@@@6B@ 00000001800010a0     Brackets.obj
 0001:000000b0       ??_7PluginCheckBoxBinding@@6B@ 00000001800010b0     Brackets.obj
 0001:000000c0       ??_7PluginRadioButtonBinding@@6B@ 00000001800010c0     Brackets.obj
 0001:000000d0       ??_7PluginEditFieldBinding@@6B@ 00000001800010d0     Brackets.obj
 0001:000000e0       ??_7PluginIntEditFieldBinding@@6B@ 00000001800010e0     Brackets.obj
 0001:000000f0       ??_C@_15EFLNJKHH@?$AA?$CF?$AAu?$AA?$AA@ 00000001800010f0     Brackets.obj
 0001:000000f8       ??_7PluginUIntEditFieldBinding@@6B@ 00000001800010f8     Brackets.obj
 0001:00000108       ??_7?$DialogBuilderBase@UFarDialogItem@@@@6B@ 0000000180001108     Brackets.obj
 0001:00000150       ??_7PluginDialogBuilder@@6B@ 0000000180001150     Brackets.obj
 0001:00000198       ??_C@_11LOCGONAA@?$AA?$AA@ 0000000180001198     Brackets.obj
 0001:000001a0       ??_C@_1BC@GJFAHMHB@?$AAB?$AAr?$AAa?$AAc?$AAk?$AAe?$AAt?$AAs?$AA?$AA@ 00000001800011a0     Brackets.obj
 0001:000001c0       ??_C@_1EE@CJLEEDHO@?$AAB?$AAr?$AAa?$AAc?$AAk?$AAe?$AAt?$AAs?$AA?5?$AAm?$AAa?$AAt?$AAc?$AAh?$AAi?$AAn?$AAg?$AA?5?$AAf?$AAo?$AAr?$AA?5?$AAF?$AAa?$AAr?$AA?5?$AAM?$AAa?$AAn?$AAa?$AAg?$AAe@ 00000001800011c0     Brackets.obj
 0001:00000208       ??_C@_1DE@BGKMIKPD@?$AAE?$AAu?$AAg?$AAe?$AAn?$AAe?$AA?5?$AAR?$AAo?$AAs?$AAh?$AAa?$AAl?$AA?5?$AA?$CG?$AA?5?$AAF?$AAa?$AAr?$AA?5?$AAG?$AAr?$AAo?$AAu?$AAp?$AA?$AA@ 0000000180001208     Brackets.obj
 0001:00000240       ??_C@_1BK@LFBLPBJM@?$AAI?$AAg?$AAn?$AAo?$AAr?$AAe?$AAQ?$AAu?$AAo?$AAt?$AAe?$AAs?$AA?$AA@ 0000000180001240     Brackets.obj
 0001:00000260       ??_C@_1BI@LPBIFPPH@?$AAI?$AAg?$AAn?$AAo?$AAr?$AAe?$AAA?$AAf?$AAt?$AAe?$AAr?$AA?$AA@ 0000000180001260     Brackets.obj
 0001:00000278       ??_C@_1BK@LJLNAEDP@?$AAB?$AAr?$AAa?$AAc?$AAk?$AAe?$AAt?$AAP?$AAr?$AAi?$AAo?$AAr?$AA?$AA@ 0000000180001278     Brackets.obj
 0001:00000298       ??_C@_1BG@KDMBKMK@?$AAJ?$AAu?$AAm?$AAp?$AAT?$AAo?$AAP?$AAa?$AAi?$AAr?$AA?$AA@ 0000000180001298     Brackets.obj
 0001:000002b0       ??_C@_19CNDHNALO@?$AAB?$AAe?$AAe?$AAp?$AA?$AA@ 00000001800012b0     Brackets.obj
 0001:000002c0       ??_C@_1BG@KHOAFHB@?$AA?8?$AA?8?$AA?$CC?$AA?$CC?$AA?$GA?$AA?8?$AA?$GA?$AA?$GA?5?$BO?5?$BN?$AA?$AA@ 00000001800012c0     Brackets.obj
 0001:000002d8       ??_C@_1BG@ICHMEPOB@?$AAQ?$AAu?$AAo?$AAt?$AAe?$AAs?$AAT?$AAy?$AAp?$AAe?$AA?$AA@ 00000001800012d8     Brackets.obj
 0001:000002f0       ??_C@_1CC@FLEKOJBB@?$AA?$DM?$AA?$DO?$AA?$HL?$AA?$HN?$AA?$FL?$AA?$FN?$AA?$CI?$AA?$CJ?$AA?$CC?$AA?$CC?$AA?8?$AA?8?$AA?$CF?$AA?$CF?$AA?$KL?$AA?$LL?$AA?$AA@ 00000001800012f0     Brackets.obj
 0001:00000318       ??_C@_1BE@CHAAIDDE@?$AAB?$AAr?$AAa?$AAc?$AAk?$AAe?$AAt?$AAs?$AA1?$AA?$AA@ 0000000180001318     Brackets.obj
 0001:00000330       ??_C@_1BK@EKFLELHE@?$AA?1?$AA?$CK?$AA?$CK?$AA?1?$AA?$DM?$AA?$DP?$AA?$DP?$AA?$DO?$AA?$DM?$AA?$CF?$AA?$CF?$AA?$DO?$AA?$AA@ 0000000180001330     Brackets.obj
 0001:00000350       ??_C@_1BE@DFLFCMNK@?$AAB?$AAr?$AAa?$AAc?$AAk?$AAe?$AAt?$AAs?$AA2?$AA?$AA@ 0000000180001350     Brackets.obj
 0001:00000368       ??_C@_19MGMPFFIA@?$AAF?$AAi?$AAn?$AAd?$AA?$AA@ 0000000180001368     Brackets.obj
 0001:00000378       ??_C@_1O@MDCABJAO@?$AAD?$AAi?$AAr?$AAe?$AAc?$AAt?$AA?$AA@ 0000000180001378     Brackets.obj
 0001:00000388       ??_C@_1BE@LCCGEFEM@?$AAS?$AAE?$AAA?$AAR?$AAC?$AAH?$AAF?$AAW?$AAD?$AA?$AA@ 0000000180001388     Brackets.obj
 0001:000003a0       ??_C@_1BG@LIFFHAGC@?$AAS?$AAE?$AAA?$AAR?$AAC?$AAH?$AAB?$AAA?$AAC?$AAK?$AA?$AA@ 00000001800013a0     Brackets.obj
 0001:000003b8       ??_C@_1BE@IFIBPANP@?$AAS?$AAE?$AAL?$AAE?$AAC?$AAT?$AAF?$AAW?$AAD?$AA?$AA@ 00000001800013b8     Brackets.obj
 0001:000003d0       ??_C@_1BG@FJDCNJBP@?$AAS?$AAE?$AAL?$AAE?$AAC?$AAT?$AAB?$AAA?$AAC?$AAK?$AA?$AA@ 00000001800013d0     Brackets.obj
 0001:000003e8       ??_C@_1O@BAHOLLMK@?$AAC?$AAO?$AAN?$AAF?$AAI?$AAG?$AA?$AA@ 00000001800013e8     Brackets.obj
 0001:00000400       __xmm@ffffffffffffffff0000000000000002 0000000180001400     Brackets.obj
 0001:00000410       __xmm@ffffffffffffffffffffffffffffffff 0000000180001410     Brackets.obj
 0001:00000420       _pRawDllMain               0000000180001420     LIBCMT:dll_dllmain.obj
 0001:00000420       _pDefaultRawDllMain        0000000180001420     LIBCMT:dll_dllmain.obj
 0001:00000430       ??_7exception@std@@6B@     0000000180001430     LIBCMT:throw_bad_alloc.obj
 0001:00000440       ??_C@_0BC@EOODALEL@Unknown?5exception?$AA@ 0000000180001440     LIBCMT:throw_bad_alloc.obj
 0001:00000460       ??_7bad_alloc@std@@6B@     0000000180001460     LIBCMT:throw_bad_alloc.obj
 0001:00000470       ??_C@_0P@GHFPNOJB@bad?5allocation?$AA@ 0000000180001470     LIBCMT:throw_bad_alloc.obj
 0001:00000488       ??_7bad_array_new_length@std@@6B@ 0000000180001488     LIBCMT:throw_bad_alloc.obj
 0001:00000498       ??_C@_0BF@KINCDENJ@bad?5array?5new?5length?$AA@ 0000000180001498     LIBCMT:throw_bad_alloc.obj
 0001:000004b8       ??_7type_info@@6B@         00000001800014b8     LIBCMT:std_type_info_static.obj
 0001:00000830       ??_C@_08EHJDFFNH@__based?$CI?$AA@ 0000000180001830     libvcruntime:undname.obj
 0001:00000840       ??_C@_07KOLFKCDI@__cdecl?$AA@ 0000000180001840     libvcruntime:undname.obj
 0001:00000848       ??_C@_08GHMPAG@__pascal?$AA@ 0000000180001848     libvcruntime:undname.obj
 0001:00000858       ??_C@_09IFJBGAPI@__stdcall?$AA@ 0000000180001858     libvcruntime:undname.obj
 0001:00000868       ??_C@_0L@NPHFGOKO@__thiscall?$AA@ 0000000180001868     libvcruntime:undname.obj
 0001:00000878       ??_C@_0L@JMKHOMEK@__fastcall?$AA@ 0000000180001878     libvcruntime:undname.obj
 0001:00000888       ??_C@_0N@BCKKPABJ@__vectorcall?$AA@ 0000000180001888     libvcruntime:undname.obj
 0001:00000898       ??_C@_09HIJEGCPM@__clrcall?$AA@ 0000000180001898     libvcruntime:undname.obj
 0001:000008a4       ??_C@_06GHPCKEAG@__eabi?$AA@ 00000001800018a4     libvcruntime:undname.obj
 0001:000008b0       ??_C@_07EECFKIPL@__swift?$AA@ 00000001800018b0     libvcruntime:undname.obj
 0001:000008b8       ??_C@_07JOMMBBKO@__ptr64?$AA@ 00000001800018b8     libvcruntime:undname.obj
 0001:000008c0       ??_C@_0L@PILCLIHE@__restrict?$AA@ 00000001800018c0     libvcruntime:undname.obj
 0001:000008d0       ??_C@_0M@GFIIJFMG@__unaligned?$AA@ 00000001800018d0     libvcruntime:undname.obj
 0001:000008e0       ??_C@_09DHDLOLLB@restrict?$CI?$AA@ 00000001800018e0     libvcruntime:undname.obj
 0001:000008ea       ??_C@_00CNPNBAHC@?$AA@     00000001800018ea     libvcruntime:undname.obj
 0001:000008ec       ??_C@_04NIHEBCM@?5new?$AA@ 00000001800018ec     libvcruntime:undname.obj
 0001:000008f8       ??_C@_07FPCDHGMM@?5delete?$AA@ 00000001800018f8     libvcruntime:undname.obj
 0001:00000900       ??_C@_01NEMOKFLO@?$DN?$AA@ 0000000180001900     libvcruntime:undname.obj
 0001:00000904       ??_C@_02GPIOPFAK@?$DO?$DO?$AA@ 0000000180001904     libvcruntime:undname.obj
 0001:00000908       ??_C@_02FODMEDOG@?$DM?$DM?$AA@ 0000000180001908     libvcruntime:undname.obj
 0001:0000090c       ??_C@_01DCLJPIOD@?$CB?$AA@ 000000018000190c     libvcruntime:undname.obj
 0001:00000910       ??_C@_02EGOFBIJA@?$DN?$DN?$AA@ 0000000180001910     libvcruntime:undname.obj
 0001:00000914       ??_C@_02FDNJECIE@?$CB?$DN?$AA@ 0000000180001914     libvcruntime:undname.obj
 0001:00000918       ??_C@_02GPECMEKF@?$FL?$FN?$AA@ 0000000180001918     libvcruntime:undname.obj
 0001:00000920       ??_C@_08LHJFAFGD@operator?$AA@ 0000000180001920     libvcruntime:undname.obj
 0001:0000092c       ??_C@_02HBOOOICD@?9?$DO?$AA@ 000000018000192c     libvcruntime:undname.obj
 0001:00000930       ??_C@_01NBENCBCI@?$CK?$AA@ 0000000180001930     libvcruntime:undname.obj
 0001:00000934       ??_C@_02ECNGHCIF@?$CL?$CL?$AA@ 0000000180001934     libvcruntime:undname.obj
 0001:00000938       ??_C@_02BAABKJLB@?9?9?$AA@ 0000000180001938     libvcruntime:undname.obj
 0001:0000093c       ??_C@_01JOAMLHOP@?9?$AA@   000000018000193c     libvcruntime:undname.obj
 0001:00000940       ??_C@_01MIFGBAGJ@?$CL?$AA@ 0000000180001940     libvcruntime:undname.obj
 0001:00000944       ??_C@_01HNPIGOCE@?$CG?$AA@ 0000000180001944     libvcruntime:undname.obj
 0001:00000948       ??_C@_03MNHNFDLC@?9?$DO?$CK?$AA@ 0000000180001948     libvcruntime:undname.obj
 0001:0000094c       ??_C@_01KMDKNFGN@?1?$AA@   000000018000194c     libvcruntime:undname.obj
 0001:00000950       ??_C@_01FGNFDNOH@?$CF?$AA@ 0000000180001950     libvcruntime:undname.obj
 0001:00000954       ??_C@_01MNNFJEPP@?$DM?$AA@ 0000000180001954     libvcruntime:undname.obj
 0001:00000958       ??_C@_02EHCHHCKH@?$DM?$DN?$AA@ 0000000180001958     libvcruntime:undname.obj
 0001:0000095c       ??_C@_01PPODPGHN@?$DO?$AA@ 000000018000195c     libvcruntime:undname.obj
 0001:00000960       ??_C@_02EEKDKGMJ@?$DO?$DN?$AA@ 0000000180001960     libvcruntime:undname.obj
 0001:00000964       ??_C@_01IHBHIGKO@?0?$AA@   0000000180001964     libvcruntime:undname.obj
 0001:00000968       ??_C@_02HCKGKOFO@?$CI?$CJ?$AA@ 0000000180001968     libvcruntime:undname.obj
 0001:0000096c       ??_C@_01PJKLJHI@?$HO?$AA@  000000018000196c     libvcruntime:undname.obj
 0001:00000970       ??_C@_01JKBOJNNK@?$FO?$AA@ 0000000180001970     libvcruntime:undname.obj
 0001:00000974       ??_C@_01DNKMNLPK@?$HM?$AA@ 0000000180001974     libvcruntime:undname.obj
 0001:00000978       ??_C@_02PPKAJPJL@?$CG?$CG?$AA@ 0000000180001978     libvcruntime:undname.obj
 0001:0000097c       ??_C@_02NONPIBCD@?$HM?$HM?$AA@ 000000018000197c     libvcruntime:undname.obj
 0001:00000980       ??_C@_02FPIMKNGF@?$CK?$DN?$AA@ 0000000180001980     libvcruntime:undname.obj
 0001:00000984       ??_C@_02FOEOMHFC@?$CL?$DN?$AA@ 0000000180001984     libvcruntime:undname.obj
 0001:00000988       ??_C@_02FKMDLLOA@?9?$DN?$AA@ 0000000180001988     libvcruntime:undname.obj
 0001:0000098c       ??_C@_02FJEHGPIO@?1?$DN?$AA@ 000000018000198c     libvcruntime:undname.obj
 0001:00000990       ??_C@_02FENAOKFI@?$CF?$DN?$AA@ 0000000180001990     libvcruntime:undname.obj
 0001:00000994       ??_C@_03IKFCCPFF@?$DO?$DO?$DN?$AA@ 0000000180001994     libvcruntime:undname.obj
 0001:00000998       ??_C@_03CDNPDDLA@?$DM?$DM?$DN?$AA@ 0000000180001998     libvcruntime:undname.obj
 0001:0000099c       ??_C@_02FGJGFEAB@?$CG?$DN?$AA@ 000000018000199c     libvcruntime:undname.obj
 0001:000009a0       ??_C@_02DHLNPPGH@?$HM?$DN?$AA@ 00000001800019a0     libvcruntime:undname.obj
 0001:000009a4       ??_C@_02MHEGNOJ@?$FO?$DN?$AA@ 00000001800019a4     libvcruntime:undname.obj
 0001:000009a8       ??_C@_09IFPLHPGF@?$GAvftable?8?$AA@ 00000001800019a8     libvcruntime:undname.obj
 0001:000009b8       ??_C@_09BLBHBJP@?$GAvbtable?8?$AA@ 00000001800019b8     libvcruntime:undname.obj
 0001:000009c8       ??_C@_07FEEIOKP@?$GAvcall?8?$AA@ 00000001800019c8     libvcruntime:undname.obj
 0001:000009d0       ??_C@_08LLFFHHDJ@?$GAtypeof?8?$AA@ 00000001800019d0     libvcruntime:undname.obj
 0001:000009e0       ??_C@_0BF@KDPPACIK@?$GAlocal?5static?5guard?8?$AA@ 00000001800019e0     libvcruntime:undname.obj
 0001:000009f8       ??_C@_08OBABFOLI@?$GAstring?8?$AA@ 00000001800019f8     libvcruntime:undname.obj
 0001:00000a08       ??_C@_0BD@JDLKDPAB@?$GAvbase?5destructor?8?$AA@ 0000000180001a08     libvcruntime:undname.obj
 0001:00000a20       ??_C@_0BN@DEGPLNFK@?$GAvector?5deleting?5destructor?8?$AA@ 0000000180001a20     libvcruntime:undname.obj
 0001:00000a40       ??_C@_0BO@OBMKPJIG@?$GAdefault?5constructor?5closure?8?$AA@ 0000000180001a40     libvcruntime:undname.obj
 0001:00000a60       ??_C@_0BN@IMDCHIKM@?$GAscalar?5deleting?5destructor?8?$AA@ 0000000180001a60     libvcruntime:undname.obj
 0001:00000a80       ??_C@_0BO@PFGOCPJJ@?$GAvector?5constructor?5iterator?8?$AA@ 0000000180001a80     libvcruntime:undname.obj
 0001:00000aa0       ??_C@_0BN@LFPFMEDL@?$GAvector?5destructor?5iterator?8?$AA@ 0000000180001aa0     libvcruntime:undname.obj
 0001:00000ac0       ??_C@_0CE@IKBNEHA@?$GAvector?5vbase?5constructor?5iterat@ 0000000180001ac0     libvcruntime:undname.obj
 0001:00000ae8       ??_C@_0BL@NILFHHPC@?$GAvirtual?5displacement?5map?8?$AA@ 0000000180001ae8     libvcruntime:undname.obj
 0001:00000b08       ??_C@_0CB@JONCMFFK@?$GAeh?5vector?5constructor?5iterator?8@ 0000000180001b08     libvcruntime:undname.obj
 0001:00000b30       ??_C@_0CA@GCEOPDGL@?$GAeh?5vector?5destructor?5iterator?8?$AA@ 0000000180001b30     libvcruntime:undname.obj
 0001:00000b50       ??_C@_0CH@OOJPLCPH@?$GAeh?5vector?5vbase?5constructor?5ite@ 0000000180001b50     libvcruntime:undname.obj
 0001:00000b78       ??_C@_0BL@LLKPOHJI@?$GAcopy?5constructor?5closure?8?$AA@ 0000000180001b78     libvcruntime:undname.obj
 0001:00000b98       ??_C@_0BA@KBCDOMBN@?$GAudt?5returning?8?$AA@ 0000000180001b98     libvcruntime:undname.obj
 0001:00000ba8       ??_C@_03KLGMFNMG@?$GAEH?$AA@ 0000000180001ba8     libvcruntime:undname.obj
 0001:00000bac       ??_C@_05KHLCHHI@?$GARTTI?$AA@ 0000000180001bac     libvcruntime:undname.obj
 0001:00000bb8       ??_C@_0BA@KKLDJDLB@?$GAlocal?5vftable?8?$AA@ 0000000180001bb8     libvcruntime:undname.obj
 0001:00000bc8       ??_C@_0CE@IIHCMGGL@?$GAlocal?5vftable?5constructor?5closu@ 0000000180001bc8     libvcruntime:undname.obj
 0001:00000bec       ??_C@_06FHBGPFGH@?5new?$FL?$FN?$AA@ 0000000180001bec     libvcruntime:undname.obj
 0001:00000bf8       ??_C@_09LBNFPBCA@?5delete?$FL?$FN?$AA@ 0000000180001bf8     libvcruntime:undname.obj
 0001:00000c08       ??_C@_0P@HJKNJFNN@?$GAomni?5callsig?8?$AA@ 0000000180001c08     libvcruntime:undname.obj
 0001:00000c18       ??_C@_0BL@CNOONJFP@?$GAplacement?5delete?5closure?8?$AA@ 0000000180001c18     libvcruntime:undname.obj
 0001:00000c38       ??_C@_0BN@CKNJLHMB@?$GAplacement?5delete?$FL?$FN?5closure?8?$AA@ 0000000180001c38     libvcruntime:undname.obj
 0001:00000c58       ??_C@_0CG@CFDHKGGD@?$GAmanaged?5vector?5constructor?5iter@ 0000000180001c58     libvcruntime:undname.obj
 0001:00000c80       ??_C@_0CF@IMGKMJNO@?$GAmanaged?5vector?5destructor?5itera@ 0000000180001c80     libvcruntime:undname.obj
 0001:00000ca8       ??_C@_0CG@HLDDJMAG@?$GAeh?5vector?5copy?5constructor?5iter@ 0000000180001ca8     libvcruntime:undname.obj
 0001:00000cd0       ??_C@_0CM@FCBBDIGB@?$GAeh?5vector?5vbase?5copy?5constructo@ 0000000180001cd0     libvcruntime:undname.obj
 0001:00000d00       ??_C@_0BL@CLIPGLGB@?$GAdynamic?5initializer?5for?5?8?$AA@ 0000000180001d00     libvcruntime:undname.obj
 0001:00000d20       ??_C@_0CB@PDBIFEP@?$GAdynamic?5atexit?5destructor?5for?5?8@ 0000000180001d20     libvcruntime:undname.obj
 0001:00000d48       ??_C@_0CD@CGAJBKEJ@?$GAvector?5copy?5constructor?5iterato@ 0000000180001d48     libvcruntime:undname.obj
 0001:00000d70       ??_C@_0CJ@GJELGAMM@?$GAvector?5vbase?5copy?5constructor?5i@ 0000000180001d70     libvcruntime:undname.obj
 0001:00000da0       ??_C@_0CL@FGIJHLCE@?$GAmanaged?5vector?5copy?5constructor@ 0000000180001da0     libvcruntime:undname.obj
 0001:00000dd0       ??_C@_0BM@PMGGMLDN@?$GAlocal?5static?5thread?5guard?8?$AA@ 0000000180001dd0     libvcruntime:undname.obj
 0001:00000df0       ??_C@_0N@BDNMDMOL@operator?5?$CC?$CC?5?$AA@ 0000000180001df0     libvcruntime:undname.obj
 0001:00000e00       ??_C@_0BC@GGEBGALA@operator?5co_await?$AA@ 0000000180001e00     libvcruntime:undname.obj
 0001:00000e18       ??_C@_0BC@DAFEJGAK@?5Type?5Descriptor?8?$AA@ 0000000180001e18     libvcruntime:undname.obj
 0001:00000e30       ??_C@_0BM@LDKODKLH@?5Base?5Class?5Descriptor?5at?5?$CI?$AA@ 0000000180001e30     libvcruntime:undname.obj
 0001:00000e50       ??_C@_0BD@LGICGFMM@?5Base?5Class?5Array?8?$AA@ 0000000180001e50     libvcruntime:undname.obj
 0001:00000e68       ??_C@_0BN@MECKDCOJ@?5Class?5Hierarchy?5Descriptor?8?$AA@ 0000000180001e68     libvcruntime:undname.obj
 0001:00000e88       ??_C@_0BK@CFCOFLF@?5Complete?5Object?5Locator?8?$AA@ 0000000180001e88     libvcruntime:undname.obj
 0001:00000ec0       ??_C@_1DM@KHCHBNEB@?$AAa?$AAp?$AAi?$AA?9?$AAm?$AAs?$AA?9?$AAw?$AAi?$AAn?$AA?9?$AAc?$AAo?$AAr?$AAe?$AA?9?$AAf?$AAi?$AAb?$AAe?$AAr?$AAs?$AA?9?$AAl?$AA1?$AA?9?$AA1?$AA?9?$AA1?$AA?$AA@ 0000000180001ec0     libvcruntime:winapi_downlevel.obj
 0001:00000f00       ??_C@_1DK@LPPGFMPP@?$AAa?$AAp?$AAi?$AA?9?$AAm?$AAs?$AA?9?$AAw?$AAi?$AAn?$AA?9?$AAc?$AAo?$AAr?$AAe?$AA?9?$AAs?$AAy?$AAn?$AAc?$AAh?$AA?9?$AAl?$AA1?$AA?9?$AA2?$AA?9?$AA0?$AA?$AA@ 0000000180001f00     libvcruntime:winapi_downlevel.obj
 0001:00000f40       ??_C@_1BC@GDMECMAK@?$AAk?$AAe?$AAr?$AAn?$AAe?$AAl?$AA3?$AA2?$AA?$AA@ 0000000180001f40     libvcruntime:winapi_downlevel.obj
 0001:00000f58       ??_C@_1BA@PFFKHIOG@?$AAa?$AAp?$AAi?$AA?9?$AAm?$AAs?$AA?9?$AA?$AA@ 0000000180001f58     libvcruntime:winapi_downlevel.obj
 0001:00000f68       ??_C@_1BA@IAIFMGEF@?$AAe?$AAx?$AAt?$AA?9?$AAm?$AAs?$AA?9?$AA?$AA@ 0000000180001f68     libvcruntime:winapi_downlevel.obj
 0001:00000f80       ??_C@_08KNHFBNJ@FlsAlloc?$AA@ 0000000180001f80     libvcruntime:winapi_downlevel.obj
 0001:00000f98       ??_C@_07PEJMOBNF@FlsFree?$AA@ 0000000180001f98     libvcruntime:winapi_downlevel.obj
 0001:00000fa8       ??_C@_0M@GDNOONDI@FlsGetValue?$AA@ 0000000180001fa8     libvcruntime:winapi_downlevel.obj
 0001:00000fc0       ??_C@_0M@JCPCPOEF@FlsSetValue?$AA@ 0000000180001fc0     libvcruntime:winapi_downlevel.obj
 0001:00000fd8       ??_C@_0BM@HCFOFFN@InitializeCriticalSectionEx?$AA@ 0000000180001fd8     libvcruntime:winapi_downlevel.obj
 0001:00000ff8       _pDestructExceptionObject  0000000180001ff8     libvcruntime:ehhelpers.obj
 0001:00001000       __acrt_exception_action_table 0000000180002000     libucrt:exception_filter.obj
 0001:000010c0       __acrt_signal_action_table_count 00000001800020c0     libucrt:exception_filter.obj
 0001:000010c8       __acrt_signal_action_first_fpe_index 00000001800020c8     libucrt:exception_filter.obj
 0001:000010d0       __acrt_signal_action_fpe_count 00000001800020d0     libucrt:exception_filter.obj
 0001:000010d8       ??_C@_1BI@BGOHAHKC@?$AAm?$AAs?$AAc?$AAo?$AAr?$AAe?$AAe?$AA?4?$AAd?$AAl?$AAl?$AA?$AA@ 00000001800020d8     libucrt:exit.obj
 0001:000010f0       ??_C@_0P@MIGLKIOC@CorExitProcess?$AA@ 00000001800020f0     libucrt:exit.obj
 0001:00001380       ??_C@_1M@HPNHIDJI@?$AAj?$AAa?$AA?9?$AAJ?$AAP?$AA?$AA@ 0000000180002380     libucrt:mbctype.obj
 0001:00001390       ??_C@_1M@BIBDDEMK@?$AAz?$AAh?$AA?9?$AAC?$AAN?$AA?$AA@ 0000000180002390     libucrt:mbctype.obj
 0001:000013a0       ??_C@_1M@JLOOOEGK@?$AAk?$AAo?$AA?9?$AAK?$AAR?$AA?$AA@ 00000001800023a0     libucrt:mbctype.obj
 0001:000013b0       ??_C@_1M@CLNBBOPM@?$AAz?$AAh?$AA?9?$AAT?$AAW?$AA?$AA@ 00000001800023b0     libucrt:mbctype.obj
 0001:00001460       ??_C@_1EA@JGEFHKEI@?$AAa?$AAp?$AAi?$AA?9?$AAm?$AAs?$AA?9?$AAw?$AAi?$AAn?$AA?9?$AAc?$AAo?$AAr?$AAe?$AA?9?$AAd?$AAa?$AAt?$AAe?$AAt?$AAi?$AAm?$AAe?$AA?9?$AAl?$AA1?$AA?9?$AA1?$AA?9?$AA1?$AA?$AA@ 0000000180002460     libucrt:winapi_thunks.obj
 0001:000014a0       ??_C@_1DI@IJCEHOCB@?$AAa?$AAp?$AAi?$AA?9?$AAm?$AAs?$AA?9?$AAw?$AAi?$AAn?$AA?9?$AAc?$AAo?$AAr?$AAe?$AA?9?$AAf?$AAi?$AAl?$AAe?$AA?9?$AAl?$AA1?$AA?9?$AA2?$AA?9?$AA2?$AA?$AA@ 00000001800024a0     libucrt:winapi_thunks.obj
 0001:000014e0       ??_C@_1EI@MPIAOHOC@?$AAa?$AAp?$AAi?$AA?9?$AAm?$AAs?$AA?9?$AAw?$AAi?$AAn?$AA?9?$AAc?$AAo?$AAr?$AAe?$AA?9?$AAl?$AAo?$AAc?$AAa?$AAl?$AAi?$AAz?$AAa?$AAt?$AAi?$AAo?$AAn?$AA?9?$AAl?$AA1?$AA?9@ 00000001800024e0     libucrt:winapi_thunks.obj
 0001:00001530       ??_C@_1FK@FPHCKFIE@?$AAa?$AAp?$AAi?$AA?9?$AAm?$AAs?$AA?9?$AAw?$AAi?$AAn?$AA?9?$AAc?$AAo?$AAr?$AAe?$AA?9?$AAl?$AAo?$AAc?$AAa?$AAl?$AAi?$AAz?$AAa?$AAt?$AAi?$AAo?$AAn?$AA?9?$AAo?$AAb?$AAs@ 0000000180002530     libucrt:winapi_thunks.obj
 0001:00001590       ??_C@_1EM@DILCGIIO@?$AAa?$AAp?$AAi?$AA?9?$AAm?$AAs?$AA?9?$AAw?$AAi?$AAn?$AA?9?$AAc?$AAo?$AAr?$AAe?$AA?9?$AAp?$AAr?$AAo?$AAc?$AAe?$AAs?$AAs?$AAt?$AAh?$AAr?$AAe?$AAa?$AAd?$AAs?$AA?9?$AAl@ 0000000180002590     libucrt:winapi_thunks.obj
 0001:000015e0       ??_C@_1DM@LNCGDDPN@?$AAa?$AAp?$AAi?$AA?9?$AAm?$AAs?$AA?9?$AAw?$AAi?$AAn?$AA?9?$AAc?$AAo?$AAr?$AAe?$AA?9?$AAs?$AAt?$AAr?$AAi?$AAn?$AAg?$AA?9?$AAl?$AA1?$AA?9?$AA1?$AA?9?$AA0?$AA?$AA@ 00000001800025e0     libucrt:winapi_thunks.obj
 0001:00001620       ??_C@_1DO@FPAPJEMD@?$AAa?$AAp?$AAi?$AA?9?$AAm?$AAs?$AA?9?$AAw?$AAi?$AAn?$AA?9?$AAc?$AAo?$AAr?$AAe?$AA?9?$AAs?$AAy?$AAs?$AAi?$AAn?$AAf?$AAo?$AA?9?$AAl?$AA1?$AA?9?$AA2?$AA?9?$AA1?$AA?$AA@ 0000000180002620     libucrt:winapi_thunks.obj
 0001:00001660       ??_C@_1DK@NDHNAHIO@?$AAa?$AAp?$AAi?$AA?9?$AAm?$AAs?$AA?9?$AAw?$AAi?$AAn?$AA?9?$AAc?$AAo?$AAr?$AAe?$AA?9?$AAw?$AAi?$AAn?$AAr?$AAt?$AA?9?$AAl?$AA1?$AA?9?$AA1?$AA?9?$AA0?$AA?$AA@ 0000000180002660     libucrt:winapi_thunks.obj
 0001:000016a0       ??_C@_1DM@KGHDGBCM@?$AAa?$AAp?$AAi?$AA?9?$AAm?$AAs?$AA?9?$AAw?$AAi?$AAn?$AA?9?$AAc?$AAo?$AAr?$AAe?$AA?9?$AAx?$AAs?$AAt?$AAa?$AAt?$AAe?$AA?9?$AAl?$AA2?$AA?9?$AA1?$AA?9?$AA0?$AA?$AA@ 00000001800026a0     libucrt:winapi_thunks.obj
 0001:000016e0       ??_C@_1EO@IJIOEFOH@?$AAa?$AAp?$AAi?$AA?9?$AAm?$AAs?$AA?9?$AAw?$AAi?$AAn?$AA?9?$AAr?$AAt?$AAc?$AAo?$AAr?$AAe?$AA?9?$AAn?$AAt?$AAu?$AAs?$AAe?$AAr?$AA?9?$AAw?$AAi?$AAn?$AAd?$AAo?$AAw?$AA?9@ 00000001800026e0     libucrt:winapi_thunks.obj
 0001:00001730       ??_C@_1FG@HHGEKANL@?$AAa?$AAp?$AAi?$AA?9?$AAm?$AAs?$AA?9?$AAw?$AAi?$AAn?$AA?9?$AAs?$AAe?$AAc?$AAu?$AAr?$AAi?$AAt?$AAy?$AA?9?$AAs?$AAy?$AAs?$AAt?$AAe?$AAm?$AAf?$AAu?$AAn?$AAc?$AAt?$AAi@ 0000000180002730     libucrt:winapi_thunks.obj
 0001:00001790       ??_C@_1EG@DBIOJECG@?$AAe?$AAx?$AAt?$AA?9?$AAm?$AAs?$AA?9?$AAw?$AAi?$AAn?$AA?9?$AAn?$AAt?$AAu?$AAs?$AAe?$AAr?$AA?9?$AAd?$AAi?$AAa?$AAl?$AAo?$AAg?$AAb?$AAo?$AAx?$AA?9?$AAl?$AA1?$AA?9?$AA1@ 0000000180002790     libucrt:winapi_thunks.obj
 0001:000017e0       ??_C@_1EO@FIHMJCLF@?$AAe?$AAx?$AAt?$AA?9?$AAm?$AAs?$AA?9?$AAw?$AAi?$AAn?$AA?9?$AAn?$AAt?$AAu?$AAs?$AAe?$AAr?$AA?9?$AAw?$AAi?$AAn?$AAd?$AAo?$AAw?$AAs?$AAt?$AAa?$AAt?$AAi?$AAo?$AAn?$AA?9@ 00000001800027e0     libucrt:winapi_thunks.obj
 0001:00001830       ??_C@_1BC@DNHGCMLG@?$AAa?$AAd?$AAv?$AAa?$AAp?$AAi?$AA3?$AA2?$AA?$AA@ 0000000180002830     libucrt:winapi_thunks.obj
 0001:00001848       ??_C@_1M@OAIMIKLP@?$AAn?$AAt?$AAd?$AAl?$AAl?$AA?$AA@ 0000000180002848     libucrt:winapi_thunks.obj
 0001:00001860       ??_C@_1EG@DPGNFKGC@?$AAa?$AAp?$AAi?$AA?9?$AAm?$AAs?$AA?9?$AAw?$AAi?$AAn?$AA?9?$AAa?$AAp?$AAp?$AAm?$AAo?$AAd?$AAe?$AAl?$AA?9?$AAr?$AAu?$AAn?$AAt?$AAi?$AAm?$AAe?$AA?9?$AAl?$AA1?$AA?9?$AA1@ 0000000180002860     libucrt:winapi_thunks.obj
 0001:000018a8       ??_C@_1O@BCCLBEOE@?$AAu?$AAs?$AAe?$AAr?$AA3?$AA2?$AA?$AA@ 00000001800028a8     libucrt:winapi_thunks.obj
 0001:000018e8       ??_C@_0O@KKBNKAPF@LCMapStringEx?$AA@ 00000001800028e8     libucrt:winapi_thunks.obj
 0001:00001900       ??_C@_0BB@HBDEELFH@LocaleNameToLCID?$AA@ 0000000180002900     libucrt:winapi_thunks.obj
 0001:00001918       ??_C@_0CF@OJOFEIGO@AppPolicyGetProcessTerminationMe@ 0000000180002918     libucrt:winapi_thunks.obj
 0001:00001940       __lc_time_c                0000000180002940     libucrt:nlsdata.obj
 0001:00001c00       ??_C@_03KOEHGMDN@Sun?$AA@  0000000180002c00     libucrt:nlsdata.obj
 0001:00001c04       ??_C@_03PDAGKDH@Mon?$AA@   0000000180002c04     libucrt:nlsdata.obj
 0001:00001c08       ??_C@_03NAGEINEP@Tue?$AA@  0000000180002c08     libucrt:nlsdata.obj
 0001:00001c0c       ??_C@_03MHOMLAJA@Wed?$AA@  0000000180002c0c     libucrt:nlsdata.obj
 0001:00001c10       ??_C@_03IOFIKPDN@Thu?$AA@  0000000180002c10     libucrt:nlsdata.obj
 0001:00001c14       ??_C@_03IDIOELNC@Fri?$AA@  0000000180002c14     libucrt:nlsdata.obj
 0001:00001c18       ??_C@_03FEFJNEK@Sat?$AA@   0000000180002c18     libucrt:nlsdata.obj
 0001:00001c1c       ??_C@_06OOPIFAJ@Sunday?$AA@ 0000000180002c1c     libucrt:nlsdata.obj
 0001:00001c24       ??_C@_06JLEDEDGH@Monday?$AA@ 0000000180002c24     libucrt:nlsdata.obj
 0001:00001c30       ??_C@_07BAAGCFCM@Tuesday?$AA@ 0000000180002c30     libucrt:nlsdata.obj
 0001:00001c38       ??_C@_09DLIGFAKA@Wednesday?$AA@ 0000000180002c38     libucrt:nlsdata.obj
 0001:00001c48       ??_C@_08HACCIKIA@Thursday?$AA@ 0000000180002c48     libucrt:nlsdata.obj
 0001:00001c54       ??_C@_06JECMNKMI@Friday?$AA@ 0000000180002c54     libucrt:nlsdata.obj
 0001:00001c60       ??_C@_08INBOOONO@Saturday?$AA@ 0000000180002c60     libucrt:nlsdata.obj
 0001:00001c6c       ??_C@_03JIHJHPIE@Jan?$AA@  0000000180002c6c     libucrt:nlsdata.obj
 0001:00001c70       ??_C@_03HJBDCHOM@Feb?$AA@  0000000180002c70     libucrt:nlsdata.obj
 0001:00001c74       ??_C@_03ODNJBKGA@Mar?$AA@  0000000180002c74     libucrt:nlsdata.obj
 0001:00001c78       ??_C@_03LEOLGMJP@Apr?$AA@  0000000180002c78     libucrt:nlsdata.obj
 0001:00001c7c       ??_C@_03CNMDKL@May?$AA@    0000000180002c7c     libucrt:nlsdata.obj
 0001:00001c80       ??_C@_03IDFGHECI@Jun?$AA@  0000000180002c80     libucrt:nlsdata.obj
 0001:00001c84       ??_C@_03LBGABGKK@Jul?$AA@  0000000180002c84     libucrt:nlsdata.obj
 0001:00001c88       ??_C@_03IFJFEIGA@Aug?$AA@  0000000180002c88     libucrt:nlsdata.obj
 0001:00001c8c       ??_C@_03GGCAPAJC@Sep?$AA@  0000000180002c8c     libucrt:nlsdata.obj
 0001:00001c90       ??_C@_03BMAOKBAD@Oct?$AA@  0000000180002c90     libucrt:nlsdata.obj
 0001:00001c94       ??_C@_03JPJOFNIA@Nov?$AA@  0000000180002c94     libucrt:nlsdata.obj
 0001:00001c98       ??_C@_03MKABNOCG@Dec?$AA@  0000000180002c98     libucrt:nlsdata.obj
 0001:00001ca0       ??_C@_07CGJPFGJA@January?$AA@ 0000000180002ca0     libucrt:nlsdata.obj
 0001:00001ca8       ??_C@_08GNJGEPFN@February?$AA@ 0000000180002ca8     libucrt:nlsdata.obj
 0001:00001cb4       ??_C@_05HPCKOFNC@March?$AA@ 0000000180002cb4     libucrt:nlsdata.obj
 0001:00001cbc       ??_C@_05DMJDNLEJ@April?$AA@ 0000000180002cbc     libucrt:nlsdata.obj
 0001:00001cc4       ??_C@_04CNLMGBGM@June?$AA@ 0000000180002cc4     libucrt:nlsdata.obj
 0001:00001ccc       ??_C@_04MIEPOIFP@July?$AA@ 0000000180002ccc     libucrt:nlsdata.obj
 0001:00001cd4       ??_C@_06LBBHFDDG@August?$AA@ 0000000180002cd4     libucrt:nlsdata.obj
 0001:00001ce0       ??_C@_09BHHEALKD@September?$AA@ 0000000180002ce0     libucrt:nlsdata.obj
 0001:00001cf0       ??_C@_07JJNFCEND@October?$AA@ 0000000180002cf0     libucrt:nlsdata.obj
 0001:00001cf8       ??_C@_08HCHEGEOA@November?$AA@ 0000000180002cf8     libucrt:nlsdata.obj
 0001:00001d08       ??_C@_08EDHMEBNP@December?$AA@ 0000000180002d08     libucrt:nlsdata.obj
 0001:00001d14       ??_C@_02DEDBPAFC@AM?$AA@   0000000180002d14     libucrt:nlsdata.obj
 0001:00001d18       ??_C@_02CJNFDJBF@PM?$AA@   0000000180002d18     libucrt:nlsdata.obj
 0001:00001d20       ??_C@_08BPBNCDIB@MM?1dd?1yy?$AA@ 0000000180002d20     libucrt:nlsdata.obj
 0001:00001d30       ??_C@_0BE@CKGJFCPC@dddd?0?5MMMM?5dd?0?5yyyy?$AA@ 0000000180002d30     libucrt:nlsdata.obj
 0001:00001d48       ??_C@_08JCCMCCIL@HH?3mm?3ss?$AA@ 0000000180002d48     libucrt:nlsdata.obj
 0001:00001d58       ??_C@_17MBGCMIPB@?$AAS?$AAu?$AAn?$AA?$AA@ 0000000180002d58     libucrt:nlsdata.obj
 0001:00001d60       ??_C@_17KBOMKBF@?$AAM?$AAo?$AAn?$AA?$AA@ 0000000180002d60     libucrt:nlsdata.obj
 0001:00001d68       ??_C@_17BMKGEGOJ@?$AAT?$AAu?$AAe?$AA?$AA@ 0000000180002d68     libucrt:nlsdata.obj
 0001:00001d70       ??_C@_17CJEDCEPE@?$AAW?$AAe?$AAd?$AA?$AA@ 0000000180002d70     libucrt:nlsdata.obj
 0001:00001d78       ??_C@_17PDPHAADD@?$AAT?$AAh?$AAu?$AA?$AA@ 0000000180002d78     libucrt:nlsdata.obj
 0001:00001d80       ??_C@_17HFOLPPLP@?$AAF?$AAr?$AAi?$AA?$AA@ 0000000180002d80     libucrt:nlsdata.obj
 0001:00001d88       ??_C@_17GGIBDPIH@?$AAS?$AAa?$AAt?$AA?$AA@ 0000000180002d88     libucrt:nlsdata.obj
 0001:00001d90       ??_C@_1O@IHNHDHPB@?$AAS?$AAu?$AAn?$AAd?$AAa?$AAy?$AA?$AA@ 0000000180002d90     libucrt:nlsdata.obj
 0001:00001da0       ??_C@_1O@MMNBFLIA@?$AAM?$AAo?$AAn?$AAd?$AAa?$AAy?$AA?$AA@ 0000000180002da0     libucrt:nlsdata.obj
 0001:00001db0       ??_C@_1BA@ENFBFFEK@?$AAT?$AAu?$AAe?$AAs?$AAd?$AAa?$AAy?$AA?$AA@ 0000000180002db0     libucrt:nlsdata.obj
 0001:00001dc0       ??_C@_1BE@EBOGMDOH@?$AAW?$AAe?$AAd?$AAn?$AAe?$AAs?$AAd?$AAa?$AAy?$AA?$AA@ 0000000180002dc0     libucrt:nlsdata.obj
 0001:00001dd8       ??_C@_1BC@HHMNLIHE@?$AAT?$AAh?$AAu?$AAr?$AAs?$AAd?$AAa?$AAy?$AA?$AA@ 0000000180002dd8     libucrt:nlsdata.obj
 0001:00001df0       ??_C@_1O@PDICJHAG@?$AAF?$AAr?$AAi?$AAd?$AAa?$AAy?$AA?$AA@ 0000000180002df0     libucrt:nlsdata.obj
 0001:00001e00       ??_C@_1BC@ENMNNPAJ@?$AAS?$AAa?$AAt?$AAu?$AAr?$AAd?$AAa?$AAy?$AA?$AA@ 0000000180002e00     libucrt:nlsdata.obj
 0001:00001e18       ??_C@_17DKNBKCHM@?$AAJ?$AAa?$AAn?$AA?$AA@ 0000000180002e18     libucrt:nlsdata.obj
 0001:00001e20       ??_C@_17LMDJEKJN@?$AAF?$AAe?$AAb?$AA?$AA@ 0000000180002e20     libucrt:nlsdata.obj
 0001:00001e28       ??_C@_17CKNLEDEC@?$AAM?$AAa?$AAr?$AA?$AA@ 0000000180002e28     libucrt:nlsdata.obj
 0001:00001e30       ??_C@_17LFPOIHDD@?$AAA?$AAp?$AAr?$AA?$AA@ 0000000180002e30     libucrt:nlsdata.obj
 0001:00001e38       ??_C@_17PNNKMEED@?$AAM?$AAa?$AAy?$AA?$AA@ 0000000180002e38     libucrt:nlsdata.obj
 0001:00001e40       ??_C@_17KCJGOCPB@?$AAJ?$AAu?$AAn?$AA?$AA@ 0000000180002e40     libucrt:nlsdata.obj
 0001:00001e48       ??_C@_17IJPCKHK@?$AAJ?$AAu?$AAl?$AA?$AA@ 0000000180002e48     libucrt:nlsdata.obj
 0001:00001e50       ??_C@_17ICPELBCN@?$AAA?$AAu?$AAg?$AA?$AA@ 0000000180002e50     libucrt:nlsdata.obj
 0001:00001e58       ??_C@_17HCHCOKMG@?$AAS?$AAe?$AAp?$AA?$AA@ 0000000180002e58     libucrt:nlsdata.obj
 0001:00001e60       ??_C@_17FNLKOI@?$AAO?$AAc?$AAt?$AA?$AA@ 0000000180002e60     libucrt:nlsdata.obj
 0001:00001e68       ??_C@_17BBDMLCIG@?$AAN?$AAo?$AAv?$AA?$AA@ 0000000180002e68     libucrt:nlsdata.obj
 0001:00001e70       ??_C@_17EGKACKIF@?$AAD?$AAe?$AAc?$AA?$AA@ 0000000180002e70     libucrt:nlsdata.obj
 0001:00001e78       ??_C@_1BA@EFMEIEBA@?$AAJ?$AAa?$AAn?$AAu?$AAa?$AAr?$AAy?$AA?$AA@ 0000000180002e78     libucrt:nlsdata.obj
 0001:00001e88       ??_C@_1BC@JGDDFFAM@?$AAF?$AAe?$AAb?$AAr?$AAu?$AAa?$AAr?$AAy?$AA?$AA@ 0000000180002e88     libucrt:nlsdata.obj
 0001:00001ea0       ??_C@_1M@IKEENEDF@?$AAM?$AAa?$AAr?$AAc?$AAh?$AA?$AA@ 0000000180002ea0     libucrt:nlsdata.obj
 0001:00001eb0       ??_C@_1M@GJNLMHFD@?$AAA?$AAp?$AAr?$AAi?$AAl?$AA?$AA@ 0000000180002eb0     libucrt:nlsdata.obj
 0001:00001ec0       ??_C@_19EPFLPGAP@?$AAJ?$AAu?$AAn?$AAe?$AA?$AA@ 0000000180002ec0     libucrt:nlsdata.obj
 0001:00001ed0       ??_C@_19BIFMLPCD@?$AAJ?$AAu?$AAl?$AAy?$AA?$AA@ 0000000180002ed0     libucrt:nlsdata.obj
 0001:00001ee0       ??_C@_1O@PAHLKOAC@?$AAA?$AAu?$AAg?$AAu?$AAs?$AAt?$AA?$AA@ 0000000180002ee0     libucrt:nlsdata.obj
 0001:00001ef0       ??_C@_1BE@DKAAMBJL@?$AAS?$AAe?$AAp?$AAt?$AAe?$AAm?$AAb?$AAe?$AAr?$AA?$AA@ 0000000180002ef0     libucrt:nlsdata.obj
 0001:00001f08       ??_C@_1BA@EPANDLNG@?$AAO?$AAc?$AAt?$AAo?$AAb?$AAe?$AAr?$AA?$AA@ 0000000180002f08     libucrt:nlsdata.obj
 0001:00001f18       ??_C@_1BC@BGLIFPF@?$AAN?$AAo?$AAv?$AAe?$AAm?$AAb?$AAe?$AAr?$AA?$AA@ 0000000180002f18     libucrt:nlsdata.obj
 0001:00001f30       ??_C@_1BC@FEMKIFH@?$AAD?$AAe?$AAc?$AAe?$AAm?$AAb?$AAe?$AAr?$AA?$AA@ 0000000180002f30     libucrt:nlsdata.obj
 0001:00001f44       ??_C@_15ODEHAHHF@?$AAA?$AAM?$AA?$AA@ 0000000180002f44     libucrt:nlsdata.obj
 0001:00001f4c       ??_C@_15CLMNNGEL@?$AAP?$AAM?$AA?$AA@ 0000000180002f4c     libucrt:nlsdata.obj
 0001:00001f58       ??_C@_1BC@IEBCMHCM@?$AAM?$AAM?$AA?1?$AAd?$AAd?$AA?1?$AAy?$AAy?$AA?$AA@ 0000000180002f58     libucrt:nlsdata.obj
 0001:00001f70       ??_C@_1CI@KNAKOEBC@?$AAd?$AAd?$AAd?$AAd?$AA?0?$AA?5?$AAM?$AAM?$AAM?$AAM?$AA?5?$AAd?$AAd?$AA?0?$AA?5?$AAy?$AAy?$AAy?$AAy?$AA?$AA@ 0000000180002f70     libucrt:nlsdata.obj
 0001:00001f98       ??_C@_1BC@GDGBMEMK@?$AAH?$AAH?$AA?3?$AAm?$AAm?$AA?3?$AAs?$AAs?$AA?$AA@ 0000000180002f98     libucrt:nlsdata.obj
 0001:00001fb0       ??_C@_1M@BMHNFIME@?$AAe?$AAn?$AA?9?$AAU?$AAS?$AA?$AA@ 0000000180002fb0     libucrt:nlsdata.obj
 0001:00001fc0       __newctype                 0000000180002fc0     libucrt:ctype.obj
 0001:000022c0       __newclmap                 00000001800032c0     libucrt:ctype.obj
 0001:00002440       __newcumap                 0000000180003440     libucrt:ctype.obj
 0001:000025c0       ??_C@_1M@BJNKEDC@?$AAc?$AAa?$AA?9?$AAE?$AAS?$AA?$AA@ 00000001800035c0     libucrt:lcidtoname_downlevel.obj
 0001:000025d0       ??_C@_1M@IJJHFJHA@?$AAc?$AAs?$AA?9?$AAC?$AAZ?$AA?$AA@ 00000001800035d0     libucrt:lcidtoname_downlevel.obj
 0001:000025e0       ??_C@_1M@CLPEOBGI@?$AAd?$AAa?$AA?9?$AAD?$AAK?$AA?$AA@ 00000001800035e0     libucrt:lcidtoname_downlevel.obj
 0001:000025f0       ??_C@_1M@MCMADGCB@?$AAd?$AAe?$AA?9?$AAD?$AAE?$AA?$AA@ 00000001800035f0     libucrt:lcidtoname_downlevel.obj
 0001:00002600       ??_C@_1M@OOCKEMAM@?$AAe?$AAl?$AA?9?$AAG?$AAR?$AA?$AA@ 0000000180003600     libucrt:lcidtoname_downlevel.obj
 0001:00002610       ??_C@_1M@DDNJFGID@?$AAf?$AAi?$AA?9?$AAF?$AAI?$AA?$AA@ 0000000180003610     libucrt:lcidtoname_downlevel.obj
 0001:00002620       ??_C@_1M@GLIPPMAC@?$AAf?$AAr?$AA?9?$AAF?$AAR?$AA?$AA@ 0000000180003620     libucrt:lcidtoname_downlevel.obj
 0001:00002630       ??_C@_1M@GFMCHPE@?$AAh?$AAe?$AA?9?$AAI?$AAL?$AA?$AA@ 0000000180003630     libucrt:lcidtoname_downlevel.obj
 0001:00002640       ??_C@_1M@MHLPGNKM@?$AAh?$AAu?$AA?9?$AAH?$AAU?$AA?$AA@ 0000000180003640     libucrt:lcidtoname_downlevel.obj
 0001:00002650       ??_C@_1M@LPDDNNPN@?$AAi?$AAs?$AA?9?$AAI?$AAS?$AA?$AA@ 0000000180003650     libucrt:lcidtoname_downlevel.obj
 0001:00002660       ??_C@_1M@MADIPODN@?$AAi?$AAt?$AA?9?$AAI?$AAT?$AA?$AA@ 0000000180003660     libucrt:lcidtoname_downlevel.obj
 0001:00002670       ??_C@_1M@IHBJJGG@?$AAn?$AAl?$AA?9?$AAN?$AAL?$AA?$AA@ 0000000180003670     libucrt:lcidtoname_downlevel.obj
 0001:00002680       ??_C@_1M@EANAGDL@?$AAn?$AAb?$AA?9?$AAN?$AAO?$AA?$AA@ 0000000180003680     libucrt:lcidtoname_downlevel.obj
 0001:00002690       ??_C@_1M@NEIEMEGP@?$AAp?$AAl?$AA?9?$AAP?$AAL?$AA?$AA@ 0000000180003690     libucrt:lcidtoname_downlevel.obj
 0001:000026a0       ??_C@_1M@BOCFIGEP@?$AAp?$AAt?$AA?9?$AAB?$AAR?$AA?$AA@ 00000001800036a0     libucrt:lcidtoname_downlevel.obj
 0001:000026b0       ??_C@_1M@IMPFOPBG@?$AAr?$AAo?$AA?9?$AAR?$AAO?$AA?$AA@ 00000001800036b0     libucrt:lcidtoname_downlevel.obj
 0001:000026c0       ??_C@_1M@IDNNEJMM@?$AAr?$AAu?$AA?9?$AAR?$AAU?$AA?$AA@ 00000001800036c0     libucrt:lcidtoname_downlevel.obj
 0001:000026d0       ??_C@_1M@LILEEOGM@?$AAh?$AAr?$AA?9?$AAH?$AAR?$AA?$AA@ 00000001800036d0     libucrt:lcidtoname_downlevel.obj
 0001:000026e0       ??_C@_1M@FKIFEHPB@?$AAs?$AAk?$AA?9?$AAS?$AAK?$AA?$AA@ 00000001800036e0     libucrt:lcidtoname_downlevel.obj
 0001:000026f0       ??_C@_1M@LJMAMNPJ@?$AAs?$AAq?$AA?9?$AAA?$AAL?$AA?$AA@ 00000001800036f0     libucrt:lcidtoname_downlevel.obj
 0001:00002700       ??_C@_1M@GIAKDKJK@?$AAs?$AAv?$AA?9?$AAS?$AAE?$AA?$AA@ 0000000180003700     libucrt:lcidtoname_downlevel.obj
 0001:00002710       ??_C@_1M@MKJKIKCL@?$AAt?$AAh?$AA?9?$AAT?$AAH?$AA?$AA@ 0000000180003710     libucrt:lcidtoname_downlevel.obj
 0001:00002720       ??_C@_1M@MFLCCMPB@?$AAt?$AAr?$AA?9?$AAT?$AAR?$AA?$AA@ 0000000180003720     libucrt:lcidtoname_downlevel.obj
 0001:00002730       ??_C@_1M@OIJHDKJN@?$AAu?$AAr?$AA?9?$AAP?$AAK?$AA?$AA@ 0000000180003730     libucrt:lcidtoname_downlevel.obj
 0001:00002740       ??_C@_1M@LHIPCIEK@?$AAi?$AAd?$AA?9?$AAI?$AAD?$AA?$AA@ 0000000180003740     libucrt:lcidtoname_downlevel.obj
 0001:00002750       ??_C@_1M@MFMOBGI@?$AAu?$AAk?$AA?9?$AAU?$AAA?$AA?$AA@ 0000000180003750     libucrt:lcidtoname_downlevel.obj
 0001:00002760       ??_C@_1M@OBGLJIPL@?$AAb?$AAe?$AA?9?$AAB?$AAY?$AA?$AA@ 0000000180003760     libucrt:lcidtoname_downlevel.obj
 0001:00002770       ??_C@_1M@BCFAJEAD@?$AAs?$AAl?$AA?9?$AAS?$AAI?$AA?$AA@ 0000000180003770     libucrt:lcidtoname_downlevel.obj
 0001:00002780       ??_C@_1M@FKFFEDDN@?$AAe?$AAt?$AA?9?$AAE?$AAE?$AA?$AA@ 0000000180003780     libucrt:lcidtoname_downlevel.obj
 0001:00002790       ??_C@_1M@KGKKAACI@?$AAl?$AAv?$AA?9?$AAL?$AAV?$AA?$AA@ 0000000180003790     libucrt:lcidtoname_downlevel.obj
 0001:000027a0       ??_C@_1M@IFGBIJO@?$AAl?$AAt?$AA?9?$AAL?$AAT?$AA?$AA@ 00000001800037a0     libucrt:lcidtoname_downlevel.obj
 0001:000027b0       ??_C@_1M@FGEAHEDM@?$AAf?$AAa?$AA?9?$AAI?$AAR?$AA?$AA@ 00000001800037b0     libucrt:lcidtoname_downlevel.obj
 0001:000027c0       ??_C@_1M@KBMAIBFN@?$AAv?$AAi?$AA?9?$AAV?$AAN?$AA?$AA@ 00000001800037c0     libucrt:lcidtoname_downlevel.obj
 0001:000027d0       ??_C@_1M@GPCBKDJK@?$AAh?$AAy?$AA?9?$AAA?$AAM?$AA?$AA@ 00000001800037d0     libucrt:lcidtoname_downlevel.obj
 0001:000027e0       ??_C@_1BG@BECMDDJB@?$AAa?$AAz?$AA?9?$AAA?$AAZ?$AA?9?$AAL?$AAa?$AAt?$AAn?$AA?$AA@ 00000001800037e0     libucrt:lcidtoname_downlevel.obj
 0001:000027f8       ??_C@_1M@MAOFCAEA@?$AAe?$AAu?$AA?9?$AAE?$AAS?$AA?$AA@ 00000001800037f8     libucrt:lcidtoname_downlevel.obj
 0001:00002808       ??_C@_1M@IGHABKPI@?$AAm?$AAk?$AA?9?$AAM?$AAK?$AA?$AA@ 0000000180003808     libucrt:lcidtoname_downlevel.obj
 0001:00002818       ??_C@_1M@IAIGNEJG@?$AAt?$AAn?$AA?9?$AAZ?$AAA?$AA?$AA@ 0000000180003818     libucrt:lcidtoname_downlevel.obj
 0001:00002828       ??_C@_1M@IIJCOJFA@?$AAx?$AAh?$AA?9?$AAZ?$AAA?$AA?$AA@ 0000000180003828     libucrt:lcidtoname_downlevel.obj
 0001:00002838       ??_C@_1M@LGPJHNJH@?$AAz?$AAu?$AA?9?$AAZ?$AAA?$AA?$AA@ 0000000180003838     libucrt:lcidtoname_downlevel.obj
 0001:00002848       ??_C@_1M@HOKAOIO@?$AAa?$AAf?$AA?9?$AAZ?$AAA?$AA?$AA@ 0000000180003848     libucrt:lcidtoname_downlevel.obj
 0001:00002858       ??_C@_1M@DPCLHLIE@?$AAk?$AAa?$AA?9?$AAG?$AAE?$AA?$AA@ 0000000180003858     libucrt:lcidtoname_downlevel.obj
 0001:00002868       ??_C@_1M@BLKMHJBI@?$AAf?$AAo?$AA?9?$AAF?$AAO?$AA?$AA@ 0000000180003868     libucrt:lcidtoname_downlevel.obj
 0001:00002878       ??_C@_1M@LGGJAPPB@?$AAh?$AAi?$AA?9?$AAI?$AAN?$AA?$AA@ 0000000180003878     libucrt:lcidtoname_downlevel.obj
 0001:00002888       ??_C@_1M@FIKPIHFE@?$AAm?$AAt?$AA?9?$AAM?$AAT?$AA?$AA@ 0000000180003888     libucrt:lcidtoname_downlevel.obj
 0001:00002898       ??_C@_1M@HEGGPBFA@?$AAs?$AAe?$AA?9?$AAN?$AAO?$AA?$AA@ 0000000180003898     libucrt:lcidtoname_downlevel.obj
 0001:000028a8       ??_C@_1M@EIBJEEPA@?$AAm?$AAs?$AA?9?$AAM?$AAY?$AA?$AA@ 00000001800038a8     libucrt:lcidtoname_downlevel.obj
 0001:000028b8       ??_C@_1M@FHLBGMPP@?$AAk?$AAk?$AA?9?$AAK?$AAZ?$AA?$AA@ 00000001800038b8     libucrt:lcidtoname_downlevel.obj
 0001:000028c8       ??_C@_1M@NGJJLCGI@?$AAk?$AAy?$AA?9?$AAK?$AAG?$AA?$AA@ 00000001800038c8     libucrt:lcidtoname_downlevel.obj
 0001:000028d8       ??_C@_1M@GIENNBFC@?$AAs?$AAw?$AA?9?$AAK?$AAE?$AA?$AA@ 00000001800038d8     libucrt:lcidtoname_downlevel.obj
 0001:000028e8       ??_C@_1BG@NDGMJIMJ@?$AAu?$AAz?$AA?9?$AAU?$AAZ?$AA?9?$AAL?$AAa?$AAt?$AAn?$AA?$AA@ 00000001800038e8     libucrt:lcidtoname_downlevel.obj
 0001:00002900       ??_C@_1M@IDCCIHBC@?$AAt?$AAt?$AA?9?$AAR?$AAU?$AA?$AA@ 0000000180003900     libucrt:lcidtoname_downlevel.obj
 0001:00002910       ??_C@_1M@LOICPMOJ@?$AAb?$AAn?$AA?9?$AAI?$AAN?$AA?$AA@ 0000000180003910     libucrt:lcidtoname_downlevel.obj
 0001:00002920       ??_C@_1M@KPKKNEAH@?$AAp?$AAa?$AA?9?$AAI?$AAN?$AA?$AA@ 0000000180003920     libucrt:lcidtoname_downlevel.obj
 0001:00002930       ??_C@_1M@PJGPPBOG@?$AAg?$AAu?$AA?9?$AAI?$AAN?$AA?$AA@ 0000000180003930     libucrt:lcidtoname_downlevel.obj
 0001:00002940       ??_C@_1M@KMKMOPHI@?$AAt?$AAa?$AA?9?$AAI?$AAN?$AA?$AA@ 0000000180003940     libucrt:lcidtoname_downlevel.obj
 0001:00002950       ??_C@_1M@KFEHEPAC@?$AAt?$AAe?$AA?9?$AAI?$AAN?$AA?$AA@ 0000000180003950     libucrt:lcidtoname_downlevel.obj
 0001:00002960       ??_C@_1M@CDCLMGHI@?$AAk?$AAn?$AA?9?$AAI?$AAN?$AA?$AA@ 0000000180003960     libucrt:lcidtoname_downlevel.obj
 0001:00002970       ??_C@_1M@MIODLDKF@?$AAm?$AAl?$AA?9?$AAI?$AAN?$AA?$AA@ 0000000180003970     libucrt:lcidtoname_downlevel.obj
 0001:00002980       ??_C@_1M@PBIEACPO@?$AAm?$AAr?$AA?9?$AAI?$AAN?$AA?$AA@ 0000000180003980     libucrt:lcidtoname_downlevel.obj
 0001:00002990       ??_C@_1M@NIDEAGPH@?$AAs?$AAa?$AA?9?$AAI?$AAN?$AA?$AA@ 0000000180003990     libucrt:lcidtoname_downlevel.obj
 0001:000029a0       ??_C@_1M@FHIHCBIO@?$AAm?$AAn?$AA?9?$AAM?$AAN?$AA?$AA@ 00000001800039a0     libucrt:lcidtoname_downlevel.obj
 0001:000029b0       ??_C@_1M@JAIJPENP@?$AAc?$AAy?$AA?9?$AAG?$AAB?$AA?$AA@ 00000001800039b0     libucrt:lcidtoname_downlevel.obj
 0001:000029c0       ??_C@_1M@PHGFBEPN@?$AAg?$AAl?$AA?9?$AAE?$AAS?$AA?$AA@ 00000001800039c0     libucrt:lcidtoname_downlevel.obj
 0001:000029d0       ??_C@_1O@KPIPDNCP@?$AAk?$AAo?$AAk?$AA?9?$AAI?$AAN?$AA?$AA@ 00000001800039d0     libucrt:lcidtoname_downlevel.obj
 0001:000029e0       ??_C@_1O@KNHJLDJA@?$AAs?$AAy?$AAr?$AA?9?$AAS?$AAY?$AA?$AA@ 00000001800039e0     libucrt:lcidtoname_downlevel.obj
 0001:000029f0       ??_C@_1O@MKEKBLAH@?$AAd?$AAi?$AAv?$AA?9?$AAM?$AAV?$AA?$AA@ 00000001800039f0     libucrt:lcidtoname_downlevel.obj
 0001:00002a00       ??_C@_1O@OHDCKDDF@?$AAq?$AAu?$AAz?$AA?9?$AAB?$AAO?$AA?$AA@ 0000000180003a00     libucrt:lcidtoname_downlevel.obj
 0001:00002a10       ??_C@_1M@LEPJNLFD@?$AAn?$AAs?$AA?9?$AAZ?$AAA?$AA?$AA@ 0000000180003a10     libucrt:lcidtoname_downlevel.obj
 0001:00002a20       ??_C@_1M@OMLEIIJB@?$AAm?$AAi?$AA?9?$AAN?$AAZ?$AA?$AA@ 0000000180003a20     libucrt:lcidtoname_downlevel.obj
 0001:00002a30       ??_C@_1M@PMPEAILG@?$AAa?$AAr?$AA?9?$AAI?$AAQ?$AA?$AA@ 0000000180003a30     libucrt:lcidtoname_downlevel.obj
 0001:00002a40       ??_C@_1M@CNKPNOEE@?$AAd?$AAe?$AA?9?$AAC?$AAH?$AA?$AA@ 0000000180003a40     libucrt:lcidtoname_downlevel.obj
 0001:00002a50       ??_C@_1M@LKMGMLKO@?$AAe?$AAn?$AA?9?$AAG?$AAB?$AA?$AA@ 0000000180003a50     libucrt:lcidtoname_downlevel.obj
 0001:00002a60       ??_C@_1M@PGKJFFGL@?$AAe?$AAs?$AA?9?$AAM?$AAX?$AA?$AA@ 0000000180003a60     libucrt:lcidtoname_downlevel.obj
 0001:00002a70       ??_C@_1M@DNNANBDC@?$AAf?$AAr?$AA?9?$AAB?$AAE?$AA?$AA@ 0000000180003a70     libucrt:lcidtoname_downlevel.obj
 0001:00002a80       ??_C@_1M@HLGMDFHM@?$AAi?$AAt?$AA?9?$AAC?$AAH?$AA?$AA@ 0000000180003a80     libucrt:lcidtoname_downlevel.obj
 0001:00002a90       ??_C@_1M@CLLBGJH@?$AAn?$AAl?$AA?9?$AAB?$AAE?$AA?$AA@ 0000000180003a90     libucrt:lcidtoname_downlevel.obj
 0001:00002aa0       ??_C@_1M@BODBOGLF@?$AAn?$AAn?$AA?9?$AAN?$AAO?$AA?$AA@ 0000000180003aa0     libucrt:lcidtoname_downlevel.obj
 0001:00002ab0       ??_C@_1M@HFFAHKAD@?$AAp?$AAt?$AA?9?$AAP?$AAT?$AA?$AA@ 0000000180003ab0     libucrt:lcidtoname_downlevel.obj
 0001:00002ac0       ??_C@_1BG@LNOAKHIE@?$AAs?$AAr?$AA?9?$AAS?$AAP?$AA?9?$AAL?$AAa?$AAt?$AAn?$AA?$AA@ 0000000180003ac0     libucrt:lcidtoname_downlevel.obj
 0001:00002ad8       ??_C@_1M@HBMHBGAK@?$AAs?$AAv?$AA?9?$AAF?$AAI?$AA?$AA@ 0000000180003ad8     libucrt:lcidtoname_downlevel.obj
 0001:00002ae8       ??_C@_1BG@DGCJGJBE@?$AAa?$AAz?$AA?9?$AAA?$AAZ?$AA?9?$AAC?$AAy?$AAr?$AAl?$AA?$AA@ 0000000180003ae8     libucrt:lcidtoname_downlevel.obj
 0001:00002b00       ??_C@_1M@KEJDAAHB@?$AAs?$AAe?$AA?9?$AAS?$AAE?$AA?$AA@ 0000000180003b00     libucrt:lcidtoname_downlevel.obj
 0001:00002b10       ??_C@_1M@HEIBJJAD@?$AAm?$AAs?$AA?9?$AAB?$AAN?$AA?$AA@ 0000000180003b10     libucrt:lcidtoname_downlevel.obj
 0001:00002b20       ??_C@_1BG@PBGJMCEM@?$AAu?$AAz?$AA?9?$AAU?$AAZ?$AA?9?$AAC?$AAy?$AAr?$AAl?$AA?$AA@ 0000000180003b20     libucrt:lcidtoname_downlevel.obj
 0001:00002b38       ??_C@_1O@LAOBCMDF@?$AAq?$AAu?$AAz?$AA?9?$AAE?$AAC?$AA?$AA@ 0000000180003b38     libucrt:lcidtoname_downlevel.obj
 0001:00002b48       ??_C@_1M@POEEMAIO@?$AAa?$AAr?$AA?9?$AAE?$AAG?$AA?$AA@ 0000000180003b48     libucrt:lcidtoname_downlevel.obj
 0001:00002b58       ??_C@_1M@EFAKDEDL@?$AAz?$AAh?$AA?9?$AAH?$AAK?$AA?$AA@ 0000000180003b58     libucrt:lcidtoname_downlevel.obj
 0001:00002b68       ??_C@_1M@HKKIJHGI@?$AAd?$AAe?$AA?9?$AAA?$AAT?$AA?$AA@ 0000000180003b68     libucrt:lcidtoname_downlevel.obj
 0001:00002b78       ??_C@_1M@KBFBEHJF@?$AAe?$AAn?$AA?9?$AAA?$AAU?$AA?$AA@ 0000000180003b78     libucrt:lcidtoname_downlevel.obj
 0001:00002b88       ??_C@_1M@MNPLFAAH@?$AAe?$AAs?$AA?9?$AAE?$AAS?$AA?$AA@ 0000000180003b88     libucrt:lcidtoname_downlevel.obj
 0001:00002b98       ??_C@_1M@HJOOJFMA@?$AAf?$AAr?$AA?9?$AAC?$AAA?$AA?$AA@ 0000000180003b98     libucrt:lcidtoname_downlevel.obj
 0001:00002ba8       ??_C@_1BG@JPOFPNAB@?$AAs?$AAr?$AA?9?$AAS?$AAP?$AA?9?$AAC?$AAy?$AAr?$AAl?$AA?$AA@ 0000000180003ba8     libucrt:lcidtoname_downlevel.obj
 0001:00002bc0       ??_C@_1M@LNFOCMOB@?$AAs?$AAe?$AA?9?$AAF?$AAI?$AA?$AA@ 0000000180003bc0     libucrt:lcidtoname_downlevel.obj
 0001:00002bd0       ??_C@_1O@MGJBOAMB@?$AAq?$AAu?$AAz?$AA?9?$AAP?$AAE?$AA?$AA@ 0000000180003bd0     libucrt:lcidtoname_downlevel.obj
 0001:00002be0       ??_C@_1M@GJINLBOK@?$AAa?$AAr?$AA?9?$AAL?$AAY?$AA?$AA@ 0000000180003be0     libucrt:lcidtoname_downlevel.obj
 0001:00002bf0       ??_C@_1M@GGMNHJNL@?$AAz?$AAh?$AA?9?$AAS?$AAG?$AA?$AA@ 0000000180003bf0     libucrt:lcidtoname_downlevel.obj
 0001:00002c00       ??_C@_1M@HOIKODND@?$AAd?$AAe?$AA?9?$AAL?$AAU?$AA?$AA@ 0000000180003c00     libucrt:lcidtoname_downlevel.obj
 0001:00002c10       ??_C@_1M@DDOCCGFG@?$AAe?$AAn?$AA?9?$AAC?$AAA?$AA?$AA@ 0000000180003c10     libucrt:lcidtoname_downlevel.obj
 0001:00002c20       ??_C@_1M@BNOEMJLF@?$AAe?$AAs?$AA?9?$AAG?$AAT?$AA?$AA@ 0000000180003c20     libucrt:lcidtoname_downlevel.obj
 0001:00002c30       ??_C@_1M@EOGNKEK@?$AAf?$AAr?$AA?9?$AAC?$AAH?$AA?$AA@ 0000000180003c30     libucrt:lcidtoname_downlevel.obj
 0001:00002c40       ??_C@_1M@FLIDJFHL@?$AAh?$AAr?$AA?9?$AAB?$AAA?$AA?$AA@ 0000000180003c40     libucrt:lcidtoname_downlevel.obj
 0001:00002c50       ??_C@_1O@FMCELNAJ@?$AAs?$AAm?$AAj?$AA?9?$AAN?$AAO?$AA?$AA@ 0000000180003c50     libucrt:lcidtoname_downlevel.obj
 0001:00002c60       ??_C@_1M@JHGLJMGJ@?$AAa?$AAr?$AA?9?$AAD?$AAZ?$AA?$AA@ 0000000180003c60     libucrt:lcidtoname_downlevel.obj
 0001:00002c70       ??_C@_1M@JKKFDCNP@?$AAz?$AAh?$AA?9?$AAM?$AAO?$AA?$AA@ 0000000180003c70     libucrt:lcidtoname_downlevel.obj
 0001:00002c80       ??_C@_1M@GEEFALPE@?$AAd?$AAe?$AA?9?$AAL?$AAI?$AA?$AA@ 0000000180003c80     libucrt:lcidtoname_downlevel.obj
 0001:00002c90       ??_C@_1M@IGEOFBG@?$AAe?$AAn?$AA?9?$AAN?$AAZ?$AA?$AA@ 0000000180003c90     libucrt:lcidtoname_downlevel.obj
 0001:00002ca0       ??_C@_1M@KDBONEHP@?$AAe?$AAs?$AA?9?$AAC?$AAR?$AA?$AA@ 0000000180003ca0     libucrt:lcidtoname_downlevel.obj
 0001:00002cb0       ??_C@_1M@FHMDOHNN@?$AAf?$AAr?$AA?9?$AAL?$AAU?$AA?$AA@ 0000000180003cb0     libucrt:lcidtoname_downlevel.obj
 0001:00002cc0       ??_C@_1BG@NFKKMAFG@?$AAb?$AAs?$AA?9?$AAB?$AAA?$AA?9?$AAL?$AAa?$AAt?$AAn?$AA?$AA@ 0000000180003cc0     libucrt:lcidtoname_downlevel.obj
 0001:00002cd8       ??_C@_1O@IMNBEMCI@?$AAs?$AAm?$AAj?$AA?9?$AAS?$AAE?$AA?$AA@ 0000000180003cd8     libucrt:lcidtoname_downlevel.obj
 0001:00002ce8       ??_C@_1M@DHHMBNDP@?$AAa?$AAr?$AA?9?$AAM?$AAA?$AA?$AA@ 0000000180003ce8     libucrt:lcidtoname_downlevel.obj
 0001:00002cf8       ??_C@_1M@BNBLJCGH@?$AAe?$AAn?$AA?9?$AAI?$AAE?$AA?$AA@ 0000000180003cf8     libucrt:lcidtoname_downlevel.obj
 0001:00002d08       ??_C@_1M@GEPAFMDL@?$AAe?$AAs?$AA?9?$AAP?$AAA?$AA?$AA@ 0000000180003d08     libucrt:lcidtoname_downlevel.obj
 0001:00002d18       ??_C@_1M@OJONDMDL@?$AAf?$AAr?$AA?9?$AAM?$AAC?$AA?$AA@ 0000000180003d18     libucrt:lcidtoname_downlevel.obj
 0001:00002d28       ??_C@_1BG@OBCNFJB@?$AAs?$AAr?$AA?9?$AAB?$AAA?$AA?9?$AAL?$AAa?$AAt?$AAn?$AA?$AA@ 0000000180003d28     libucrt:lcidtoname_downlevel.obj
 0001:00002d40       ??_C@_1O@KEMEEGPO@?$AAs?$AAm?$AAa?$AA?9?$AAN?$AAO?$AA?$AA@ 0000000180003d40     libucrt:lcidtoname_downlevel.obj
 0001:00002d50       ??_C@_1M@ELMGFODK@?$AAa?$AAr?$AA?9?$AAT?$AAN?$AA?$AA@ 0000000180003d50     libucrt:lcidtoname_downlevel.obj
 0001:00002d60       ??_C@_1M@BHDLHFAF@?$AAe?$AAn?$AA?9?$AAZ?$AAA?$AA?$AA@ 0000000180003d60     libucrt:lcidtoname_downlevel.obj
 0001:00002d70       ??_C@_1M@BMGIGLIF@?$AAe?$AAs?$AA?9?$AAD?$AAO?$AA?$AA@ 0000000180003d70     libucrt:lcidtoname_downlevel.obj
 0001:00002d80       ??_C@_1BG@CMBHIPBE@?$AAs?$AAr?$AA?9?$AAB?$AAA?$AA?9?$AAC?$AAy?$AAr?$AAl?$AA?$AA@ 0000000180003d80     libucrt:lcidtoname_downlevel.obj
 0001:00002d98       ??_C@_1O@HEDBLHNP@?$AAs?$AAm?$AAa?$AA?9?$AAS?$AAE?$AA?$AA@ 0000000180003d98     libucrt:lcidtoname_downlevel.obj
 0001:00002da8       ??_C@_1M@DAGCADIM@?$AAa?$AAr?$AA?9?$AAO?$AAM?$AA?$AA@ 0000000180003da8     libucrt:lcidtoname_downlevel.obj
 0001:00002db8       ??_C@_1M@FODLMICG@?$AAe?$AAn?$AA?9?$AAJ?$AAM?$AA?$AA@ 0000000180003db8     libucrt:lcidtoname_downlevel.obj
 0001:00002dc8       ??_C@_1M@DNMLCIHB@?$AAe?$AAs?$AA?9?$AAV?$AAE?$AA?$AA@ 0000000180003dc8     libucrt:lcidtoname_downlevel.obj
 0001:00002dd8       ??_C@_1O@EOKHMKJK@?$AAs?$AAm?$AAs?$AA?9?$AAF?$AAI?$AA?$AA@ 0000000180003dd8     libucrt:lcidtoname_downlevel.obj
 0001:00002de8       ??_C@_1M@CAFJMKOF@?$AAa?$AAr?$AA?9?$AAY?$AAE?$AA?$AA@ 0000000180003de8     libucrt:lcidtoname_downlevel.obj
 0001:00002df8       ??_C@_1M@CBFHIJLI@?$AAe?$AAn?$AA?9?$AAC?$AAB?$AA?$AA@ 0000000180003df8     libucrt:lcidtoname_downlevel.obj
 0001:00002e08       ??_C@_1M@BGNFLDN@?$AAe?$AAs?$AA?9?$AAC?$AAO?$AA?$AA@ 0000000180003e08     libucrt:lcidtoname_downlevel.obj
 0001:00002e18       ??_C@_1O@JMPHMAMC@?$AAs?$AAm?$AAn?$AA?9?$AAF?$AAI?$AA?$AA@ 0000000180003e18     libucrt:lcidtoname_downlevel.obj
 0001:00002e28       ??_C@_1M@JLANABKE@?$AAa?$AAr?$AA?9?$AAS?$AAY?$AA?$AA@ 0000000180003e28     libucrt:lcidtoname_downlevel.obj
 0001:00002e38       ??_C@_1M@HPKGCFGN@?$AAe?$AAn?$AA?9?$AAB?$AAZ?$AA?$AA@ 0000000180003e38     libucrt:lcidtoname_downlevel.obj
 0001:00002e48       ??_C@_1M@OLJCMLGM@?$AAe?$AAs?$AA?9?$AAP?$AAE?$AA?$AA@ 0000000180003e48     libucrt:lcidtoname_downlevel.obj
 0001:00002e58       ??_C@_1M@MKKGFKLE@?$AAa?$AAr?$AA?9?$AAJ?$AAO?$AA?$AA@ 0000000180003e58     libucrt:lcidtoname_downlevel.obj
 0001:00002e68       ??_C@_1M@EKPGLDNI@?$AAe?$AAn?$AA?9?$AAT?$AAT?$AA?$AA@ 0000000180003e68     libucrt:lcidtoname_downlevel.obj
 0001:00002e78       ??_C@_1M@OONGHFHE@?$AAe?$AAs?$AA?9?$AAA?$AAR?$AA?$AA@ 0000000180003e78     libucrt:lcidtoname_downlevel.obj
 0001:00002e88       ??_C@_1M@OOJFGBHE@?$AAa?$AAr?$AA?9?$AAL?$AAB?$AA?$AA@ 0000000180003e88     libucrt:lcidtoname_downlevel.obj
 0001:00002e98       ??_C@_1M@GCEJHNEG@?$AAe?$AAn?$AA?9?$AAZ?$AAW?$AA?$AA@ 0000000180003e98     libucrt:lcidtoname_downlevel.obj
 0001:00002ea8       ??_C@_1M@JNOCAHJI@?$AAe?$AAs?$AA?9?$AAE?$AAC?$AA?$AA@ 0000000180003ea8     libucrt:lcidtoname_downlevel.obj
 0001:00002eb8       ??_C@_1M@JEFHPGGB@?$AAa?$AAr?$AA?9?$AAK?$AAW?$AA?$AA@ 0000000180003eb8     libucrt:lcidtoname_downlevel.obj
 0001:00002ec8       ??_C@_1M@MLKIBJOJ@?$AAe?$AAn?$AA?9?$AAP?$AAH?$AA?$AA@ 0000000180003ec8     libucrt:lcidtoname_downlevel.obj
 0001:00002ed8       ??_C@_1M@BDNIPEND@?$AAe?$AAs?$AA?9?$AAC?$AAL?$AA?$AA@ 0000000180003ed8     libucrt:lcidtoname_downlevel.obj
 0001:00002ee8       ??_C@_1M@MPNMEKBD@?$AAa?$AAr?$AA?9?$AAA?$AAE?$AA?$AA@ 0000000180003ee8     libucrt:lcidtoname_downlevel.obj
 0001:00002ef8       ??_C@_1M@KBJALCPI@?$AAe?$AAs?$AA?9?$AAU?$AAY?$AA?$AA@ 0000000180003ef8     libucrt:lcidtoname_downlevel.obj
 0001:00002f08       ??_C@_1M@LLCCOAGA@?$AAa?$AAr?$AA?9?$AAB?$AAH?$AA?$AA@ 0000000180003f08     libucrt:lcidtoname_downlevel.obj
 0001:00002f18       ??_C@_1M@PBFNCDEL@?$AAe?$AAs?$AA?9?$AAP?$AAY?$AA?$AA@ 0000000180003f18     libucrt:lcidtoname_downlevel.obj
 0001:00002f28       ??_C@_1M@EDGINPNP@?$AAa?$AAr?$AA?9?$AAQ?$AAA?$AA?$AA@ 0000000180003f28     libucrt:lcidtoname_downlevel.obj
 0001:00002f38       ??_C@_1M@MKDBIIJI@?$AAe?$AAs?$AA?9?$AAB?$AAO?$AA?$AA@ 0000000180003f38     libucrt:lcidtoname_downlevel.obj
 0001:00002f48       ??_C@_1M@CPKKEBLD@?$AAe?$AAs?$AA?9?$AAS?$AAV?$AA?$AA@ 0000000180003f48     libucrt:lcidtoname_downlevel.obj
 0001:00002f58       ??_C@_1M@NDBGMMJL@?$AAe?$AAs?$AA?9?$AAH?$AAN?$AA?$AA@ 0000000180003f58     libucrt:lcidtoname_downlevel.obj
 0001:00002f68       ??_C@_1M@JIJIBHDP@?$AAe?$AAs?$AA?9?$AAN?$AAI?$AA?$AA@ 0000000180003f68     libucrt:lcidtoname_downlevel.obj
 0001:00002f78       ??_C@_1M@CGFMKEEK@?$AAe?$AAs?$AA?9?$AAP?$AAR?$AA?$AA@ 0000000180003f78     libucrt:lcidtoname_downlevel.obj
 0001:00002f88       ??_C@_1O@ICJHKIIK@?$AAz?$AAh?$AA?9?$AAC?$AAH?$AAT?$AA?$AA@ 0000000180003f88     libucrt:lcidtoname_downlevel.obj
 0001:00002f98       ??_C@_15CLNEJCE@?$AAs?$AAr?$AA?$AA@ 0000000180003f98     libucrt:lcidtoname_downlevel.obj
 0001:00003de0       ??_C@_1M@KAHEKEIG@?$AAa?$AAf?$AA?9?$AAz?$AAa?$AA?$AA@ 0000000180004de0     libucrt:lcidtoname_downlevel.obj
 0001:00003df0       ??_C@_1M@GIECOABL@?$AAa?$AAr?$AA?9?$AAa?$AAe?$AA?$AA@ 0000000180004df0     libucrt:lcidtoname_downlevel.obj
 0001:00003e00       ??_C@_1M@BMLMEKGI@?$AAa?$AAr?$AA?9?$AAb?$AAh?$AA?$AA@ 0000000180004e00     libucrt:lcidtoname_downlevel.obj
 0001:00003e10       ??_C@_1M@DAPFDGGB@?$AAa?$AAr?$AA?9?$AAd?$AAz?$AA?$AA@ 0000000180004e10     libucrt:lcidtoname_downlevel.obj
 0001:00003e20       ??_C@_1M@FJNKGKIG@?$AAa?$AAr?$AA?9?$AAe?$AAg?$AA?$AA@ 0000000180004e20     libucrt:lcidtoname_downlevel.obj
 0001:00003e30       ??_C@_1M@FLGKKCLO@?$AAa?$AAr?$AA?9?$AAi?$AAq?$AA?$AA@ 0000000180004e30     libucrt:lcidtoname_downlevel.obj
 0001:00003e40       ??_C@_1M@GNDIPALM@?$AAa?$AAr?$AA?9?$AAj?$AAo?$AA?$AA@ 0000000180004e40     libucrt:lcidtoname_downlevel.obj
 0001:00003e50       ??_C@_1M@DDMJFMGJ@?$AAa?$AAr?$AA?9?$AAk?$AAw?$AA?$AA@ 0000000180004e50     libucrt:lcidtoname_downlevel.obj
 0001:00003e60       ??_C@_1M@EJALMLHM@?$AAa?$AAr?$AA?9?$AAl?$AAb?$AA?$AA@ 0000000180004e60     libucrt:lcidtoname_downlevel.obj
 0001:00003e70       ??_C@_1M@MOBDBLOC@?$AAa?$AAr?$AA?9?$AAl?$AAy?$AA?$AA@ 0000000180004e70     libucrt:lcidtoname_downlevel.obj
 0001:00003e80       ??_C@_1M@JAOCLHDH@?$AAa?$AAr?$AA?9?$AAm?$AAa?$AA?$AA@ 0000000180004e80     libucrt:lcidtoname_downlevel.obj
 0001:00003e90       ??_C@_1M@JHPMKJIE@?$AAa?$AAr?$AA?9?$AAo?$AAm?$AA?$AA@ 0000000180004e90     libucrt:lcidtoname_downlevel.obj
 0001:00003ea0       ??_C@_1M@OEPGHFNH@?$AAa?$AAr?$AA?9?$AAq?$AAa?$AA?$AA@ 0000000180004ea0     libucrt:lcidtoname_downlevel.obj
 0001:00003eb0       ??_C@_1M@KJDONENM@?$AAa?$AAr?$AA?9?$AAs?$AAa?$AA?$AA@ 0000000180004eb0     libucrt:lcidtoname_downlevel.obj
 0001:00003ec0       ??_C@_1M@DMJDKLKM@?$AAa?$AAr?$AA?9?$AAs?$AAy?$AA?$AA@ 0000000180004ec0     libucrt:lcidtoname_downlevel.obj
 0001:00003ed0       ??_C@_1M@OMFIPEDC@?$AAa?$AAr?$AA?9?$AAt?$AAn?$AA?$AA@ 0000000180004ed0     libucrt:lcidtoname_downlevel.obj
 0001:00003ee0       ??_C@_1M@IHMHGAON@?$AAa?$AAr?$AA?9?$AAy?$AAe?$AA?$AA@ 0000000180004ee0     libucrt:lcidtoname_downlevel.obj
 0001:00003ef0       ??_C@_1BG@KDCPGJGB@?$AAa?$AAz?$AA?9?$AAa?$AAz?$AA?9?$AAc?$AAy?$AAr?$AAl?$AA?$AA@ 0000000180004ef0     libucrt:lcidtoname_downlevel.obj
 0001:00003f08       ??_C@_1BG@IBCKDDOE@?$AAa?$AAz?$AA?9?$AAa?$AAz?$AA?9?$AAl?$AAa?$AAt?$AAn?$AA?$AA@ 0000000180004f08     libucrt:lcidtoname_downlevel.obj
 0001:00003f20       ??_C@_1M@EGPFDCPD@?$AAb?$AAe?$AA?9?$AAb?$AAy?$AA?$AA@ 0000000180004f20     libucrt:lcidtoname_downlevel.obj
 0001:00003f30       ??_C@_1M@PCMGMCGC@?$AAb?$AAg?$AA?9?$AAb?$AAg?$AA?$AA@ 0000000180004f30     libucrt:lcidtoname_downlevel.obj
 0001:00003f40       ??_C@_1M@BJBMFGOB@?$AAb?$AAn?$AA?9?$AAi?$AAn?$AA?$AA@ 0000000180004f40     libucrt:lcidtoname_downlevel.obj
 0001:00003f50       ??_C@_1BG@EAKMMACD@?$AAb?$AAs?$AA?9?$AAb?$AAa?$AA?9?$AAl?$AAa?$AAt?$AAn?$AA?$AA@ 0000000180004f50     libucrt:lcidtoname_downlevel.obj
 0001:00003f68       ??_C@_1M@KGADAODK@?$AAc?$AAa?$AA?9?$AAe?$AAs?$AA?$AA@ 0000000180004f68     libucrt:lcidtoname_downlevel.obj
 0001:00003f78       ??_C@_1M@COAJPDHI@?$AAc?$AAs?$AA?9?$AAc?$AAz?$AA?$AA@ 0000000180004f78     libucrt:lcidtoname_downlevel.obj
 0001:00003f88       ??_C@_1M@DHBHFONH@?$AAc?$AAy?$AA?9?$AAg?$AAb?$AA?$AA@ 0000000180004f88     libucrt:lcidtoname_downlevel.obj
 0001:00003f98       ??_C@_1M@IMGKELGA@?$AAd?$AAa?$AA?9?$AAd?$AAk?$AA?$AA@ 0000000180004f98     libucrt:lcidtoname_downlevel.obj
 0001:00003fa8       ??_C@_1M@NNDGDNGA@?$AAd?$AAe?$AA?9?$AAa?$AAt?$AA?$AA@ 0000000180004fa8     libucrt:lcidtoname_downlevel.obj
 0001:00003fb8       ??_C@_1M@IKDBHEEM@?$AAd?$AAe?$AA?9?$AAc?$AAh?$AA?$AA@ 0000000180004fb8     libucrt:lcidtoname_downlevel.obj
 0001:00003fc8       ??_C@_1M@GFFOJMCJ@?$AAd?$AAe?$AA?9?$AAd?$AAe?$AA?$AA@ 0000000180004fc8     libucrt:lcidtoname_downlevel.obj
 0001:00003fd8       ??_C@_1M@MDNLKBPM@?$AAd?$AAe?$AA?9?$AAl?$AAi?$AA?$AA@ 0000000180004fd8     libucrt:lcidtoname_downlevel.obj
 0001:00003fe8       ??_C@_1M@NJBEEJNL@?$AAd?$AAe?$AA?9?$AAl?$AAu?$AA?$AA@ 0000000180004fe8     libucrt:lcidtoname_downlevel.obj
 0001:00003ff8       ??_C@_1O@GNNELBAP@?$AAd?$AAi?$AAv?$AA?9?$AAm?$AAv?$AA?$AA@ 0000000180004ff8     libucrt:lcidtoname_downlevel.obj
 0001:00004008       ??_C@_1M@EJLEOGAE@?$AAe?$AAl?$AA?9?$AAg?$AAr?$AA?$AA@ 0000000180005008     libucrt:lcidtoname_downlevel.obj
 0001:00004018       ??_C@_1M@GMPONJN@?$AAe?$AAn?$AA?9?$AAa?$AAu?$AA?$AA@ 0000000180005018     libucrt:lcidtoname_downlevel.obj
 0001:00004028       ??_C@_1M@NIDIIPGF@?$AAe?$AAn?$AA?9?$AAb?$AAz?$AA?$AA@ 0000000180005028     libucrt:lcidtoname_downlevel.obj
 0001:00004038       ??_C@_1M@JEHMIMFO@?$AAe?$AAn?$AA?9?$AAc?$AAa?$AA?$AA@ 0000000180005038     libucrt:lcidtoname_downlevel.obj
 0001:00004048       ??_C@_1M@IGMJCDLA@?$AAe?$AAn?$AA?9?$AAc?$AAb?$AA?$AA@ 0000000180005048     libucrt:lcidtoname_downlevel.obj
 0001:00004058       ??_C@_1M@BNFIGBKG@?$AAe?$AAn?$AA?9?$AAg?$AAb?$AA?$AA@ 0000000180005058     libucrt:lcidtoname_downlevel.obj
 0001:00004068       ??_C@_1M@LKIFDIGP@?$AAe?$AAn?$AA?9?$AAi?$AAe?$AA?$AA@ 0000000180005068     libucrt:lcidtoname_downlevel.obj
 0001:00004078       ??_C@_1M@PJKFGCCO@?$AAe?$AAn?$AA?9?$AAj?$AAm?$AA?$AA@ 0000000180005078     libucrt:lcidtoname_downlevel.obj
 0001:00004088       ??_C@_1M@KPPKEPBO@?$AAe?$AAn?$AA?9?$AAn?$AAz?$AA?$AA@ 0000000180005088     libucrt:lcidtoname_downlevel.obj
 0001:00004098       ??_C@_1M@GMDGLDOB@?$AAe?$AAn?$AA?9?$AAp?$AAh?$AA?$AA@ 0000000180005098     libucrt:lcidtoname_downlevel.obj
 0001:000040a8       ??_C@_1M@ONGIBJNA@?$AAe?$AAn?$AA?9?$AAt?$AAt?$AA?$AA@ 00000001800050a8     libucrt:lcidtoname_downlevel.obj
 0001:000040b8       ??_C@_1M@LLODPCMM@?$AAe?$AAn?$AA?9?$AAu?$AAs?$AA?$AA@ 00000001800050b8     libucrt:lcidtoname_downlevel.obj
 0001:000040c8       ??_C@_1M@LAKFNPAN@?$AAe?$AAn?$AA?9?$AAz?$AAa?$AA?$AA@ 00000001800050c8     libucrt:lcidtoname_downlevel.obj
 0001:000040d8       ??_C@_1M@MFNHNHEO@?$AAe?$AAn?$AA?9?$AAz?$AAw?$AA?$AA@ 00000001800050d8     libucrt:lcidtoname_downlevel.obj
 0001:000040e8       ??_C@_1M@EJEINPHM@?$AAe?$AAs?$AA?9?$AAa?$AAr?$AA?$AA@ 00000001800050e8     libucrt:lcidtoname_downlevel.obj
 0001:000040f8       ??_C@_1M@GNKPCCJA@?$AAe?$AAs?$AA?9?$AAb?$AAo?$AA?$AA@ 00000001800050f8     libucrt:lcidtoname_downlevel.obj
 0001:00004108       ??_C@_1M@LEEGFONL@?$AAe?$AAs?$AA?9?$AAc?$AAl?$AA?$AA@ 0000000180005108     libucrt:lcidtoname_downlevel.obj
 0001:00004118       ??_C@_1M@KGPDPBDF@?$AAe?$AAs?$AA?9?$AAc?$AAo?$AA?$AA@ 0000000180005118     libucrt:lcidtoname_downlevel.obj
 0001:00004128       ??_C@_1M@EIAHOHH@?$AAe?$AAs?$AA?9?$AAc?$AAr?$AA?$AA@ 0000000180005128     libucrt:lcidtoname_downlevel.obj
 0001:00004138       ??_C@_1M@LLPGMBIN@?$AAe?$AAs?$AA?9?$AAd?$AAo?$AA?$AA@ 0000000180005138     libucrt:lcidtoname_downlevel.obj
 0001:00004148       ??_C@_1M@DKHMKNJA@?$AAe?$AAs?$AA?9?$AAe?$AAc?$AA?$AA@ 0000000180005148     libucrt:lcidtoname_downlevel.obj
 0001:00004158       ??_C@_1M@GKGFPKAP@?$AAe?$AAs?$AA?9?$AAe?$AAs?$AA?$AA@ 0000000180005158     libucrt:lcidtoname_downlevel.obj
 0001:00004168       ??_C@_1M@LKHKGDLN@?$AAe?$AAs?$AA?9?$AAg?$AAt?$AA?$AA@ 0000000180005168     libucrt:lcidtoname_downlevel.obj
 0001:00004178       ??_C@_1M@HEIIGGJD@?$AAe?$AAs?$AA?9?$AAh?$AAn?$AA?$AA@ 0000000180005178     libucrt:lcidtoname_downlevel.obj
 0001:00004188       ??_C@_1M@FBDHPPGD@?$AAe?$AAs?$AA?9?$AAm?$AAx?$AA?$AA@ 0000000180005188     libucrt:lcidtoname_downlevel.obj
 0001:00004198       ??_C@_1M@DPAGLNDH@?$AAe?$AAs?$AA?9?$AAn?$AAi?$AA?$AA@ 0000000180005198     libucrt:lcidtoname_downlevel.obj
 0001:000041a8       ??_C@_1M@MDGOPGDD@?$AAe?$AAs?$AA?9?$AAp?$AAa?$AA?$AA@ 00000001800051a8     libucrt:lcidtoname_downlevel.obj
 0001:000041b8       ??_C@_1M@EMAMGBGE@?$AAe?$AAs?$AA?9?$AAp?$AAe?$AA?$AA@ 00000001800051b8     libucrt:lcidtoname_downlevel.obj
 0001:000041c8       ??_C@_1M@IBMCAOEC@?$AAe?$AAs?$AA?9?$AAp?$AAr?$AA?$AA@ 00000001800051c8     libucrt:lcidtoname_downlevel.obj
 0001:000041d8       ??_C@_1M@FGMDIJED@?$AAe?$AAs?$AA?9?$AAp?$AAy?$AA?$AA@ 00000001800051d8     libucrt:lcidtoname_downlevel.obj
 0001:000041e8       ??_C@_1M@IIDEOLLL@?$AAe?$AAs?$AA?9?$AAs?$AAv?$AA?$AA@ 00000001800051e8     libucrt:lcidtoname_downlevel.obj
 0001:000041f8       ??_C@_1M@GAOBIPA@?$AAe?$AAs?$AA?9?$AAu?$AAy?$AA?$AA@ 00000001800051f8     libucrt:lcidtoname_downlevel.obj
 0001:00004208       ??_C@_1M@JKFFICHJ@?$AAe?$AAs?$AA?9?$AAv?$AAe?$AA?$AA@ 0000000180005208     libucrt:lcidtoname_downlevel.obj
 0001:00004218       ??_C@_1M@PNMLOJDF@?$AAe?$AAt?$AA?9?$AAe?$AAe?$AA?$AA@ 0000000180005218     libucrt:lcidtoname_downlevel.obj
 0001:00004228       ??_C@_1M@GHHLIKEI@?$AAe?$AAu?$AA?9?$AAe?$AAs?$AA?$AA@ 0000000180005228     libucrt:lcidtoname_downlevel.obj
 0001:00004238       ??_C@_1M@PBNONODE@?$AAf?$AAa?$AA?9?$AAi?$AAr?$AA?$AA@ 0000000180005238     libucrt:lcidtoname_downlevel.obj
 0001:00004248       ??_C@_1M@JEEHPMIL@?$AAf?$AAi?$AA?9?$AAf?$AAi?$AA?$AA@ 0000000180005248     libucrt:lcidtoname_downlevel.obj
 0001:00004258       ??_C@_1M@LMDCNDBA@?$AAf?$AAo?$AA?9?$AAf?$AAo?$AA?$AA@ 0000000180005258     libucrt:lcidtoname_downlevel.obj
 0001:00004268       ??_C@_1M@JKEOHLDK@?$AAf?$AAr?$AA?9?$AAb?$AAe?$AA?$AA@ 0000000180005268     libucrt:lcidtoname_downlevel.obj
 0001:00004278       ??_C@_1M@NOHADPMI@?$AAf?$AAr?$AA?9?$AAc?$AAa?$AA?$AA@ 0000000180005278     libucrt:lcidtoname_downlevel.obj
 0001:00004288       ??_C@_1M@KDHIHAEC@?$AAf?$AAr?$AA?9?$AAc?$AAh?$AA?$AA@ 0000000180005288     libucrt:lcidtoname_downlevel.obj
 0001:00004298       ??_C@_1M@MMBBFGAK@?$AAf?$AAr?$AA?9?$AAf?$AAr?$AA?$AA@ 0000000180005298     libucrt:lcidtoname_downlevel.obj
 0001:000042a8       ??_C@_1M@PAFNENNF@?$AAf?$AAr?$AA?9?$AAl?$AAu?$AA?$AA@ 00000001800052a8     libucrt:lcidtoname_downlevel.obj
 0001:000042b8       ??_C@_1M@EOHDJGDD@?$AAf?$AAr?$AA?9?$AAm?$AAc?$AA?$AA@ 00000001800052b8     libucrt:lcidtoname_downlevel.obj
 0001:000042c8       ??_C@_1M@FAPLLOPF@?$AAg?$AAl?$AA?9?$AAe?$AAs?$AA?$AA@ 00000001800052c8     libucrt:lcidtoname_downlevel.obj
 0001:000042d8       ??_C@_1M@FOPBFLOO@?$AAg?$AAu?$AA?9?$AAi?$AAn?$AA?$AA@ 00000001800052d8     libucrt:lcidtoname_downlevel.obj
 0001:000042e8       ??_C@_1M@KBMCINPM@?$AAh?$AAe?$AA?9?$AAi?$AAl?$AA?$AA@ 00000001800052e8     libucrt:lcidtoname_downlevel.obj
 0001:000042f8       ??_C@_1M@BBPHKFPJ@?$AAh?$AAi?$AA?9?$AAi?$AAn?$AA?$AA@ 00000001800052f8     libucrt:lcidtoname_downlevel.obj
 0001:00004308       ??_C@_1M@PMBNDPHD@?$AAh?$AAr?$AA?9?$AAb?$AAa?$AA?$AA@ 0000000180005308     libucrt:lcidtoname_downlevel.obj
 0001:00004318       ??_C@_1M@BPCKOEGE@?$AAh?$AAr?$AA?9?$AAh?$AAr?$AA?$AA@ 0000000180005318     libucrt:lcidtoname_downlevel.obj
 0001:00004328       ??_C@_1M@GACBMHKE@?$AAh?$AAu?$AA?9?$AAh?$AAu?$AA?$AA@ 0000000180005328     libucrt:lcidtoname_downlevel.obj
 0001:00004338       ??_C@_1M@MILPAJJC@?$AAh?$AAy?$AA?9?$AAa?$AAm?$AA?$AA@ 0000000180005338     libucrt:lcidtoname_downlevel.obj
 0001:00004348       ??_C@_1M@BABBICEC@?$AAi?$AAd?$AA?9?$AAi?$AAd?$AA?$AA@ 0000000180005348     libucrt:lcidtoname_downlevel.obj
 0001:00004358       ??_C@_1M@BIKNHHPF@?$AAi?$AAs?$AA?9?$AAi?$AAs?$AA?$AA@ 0000000180005358     libucrt:lcidtoname_downlevel.obj
 0001:00004368       ??_C@_1M@NMPCJPHE@?$AAi?$AAt?$AA?9?$AAc?$AAh?$AA?$AA@ 0000000180005368     libucrt:lcidtoname_downlevel.obj
 0001:00004378       ??_C@_1M@GHKGFEDF@?$AAi?$AAt?$AA?9?$AAi?$AAt?$AA?$AA@ 0000000180005378     libucrt:lcidtoname_downlevel.obj
 0001:00004388       ??_C@_1M@NIEJCJJA@?$AAj?$AAa?$AA?9?$AAj?$AAp?$AA?$AA@ 0000000180005388     libucrt:lcidtoname_downlevel.obj
 0001:00004398       ??_C@_1M@JILFNBIM@?$AAk?$AAa?$AA?9?$AAg?$AAe?$AA?$AA@ 0000000180005398     libucrt:lcidtoname_downlevel.obj
 0001:000043a8       ??_C@_1M@PACPMGPH@?$AAk?$AAk?$AA?9?$AAk?$AAz?$AA?$AA@ 00000001800053a8     libucrt:lcidtoname_downlevel.obj
 0001:000043b8       ??_C@_1M@IELFGMHA@?$AAk?$AAn?$AA?9?$AAi?$AAn?$AA?$AA@ 00000001800053b8     libucrt:lcidtoname_downlevel.obj
 0001:000043c8       ??_C@_1O@IBBJHCH@?$AAk?$AAo?$AAk?$AA?9?$AAi?$AAn?$AA?$AA@ 00000001800053c8     libucrt:lcidtoname_downlevel.obj
 0001:000043d8       ??_C@_1M@DMHAEOGC@?$AAk?$AAo?$AA?9?$AAk?$AAr?$AA?$AA@ 00000001800053d8     libucrt:lcidtoname_downlevel.obj
 0001:000043e8       ??_C@_1M@HBAHBIGA@?$AAk?$AAy?$AA?9?$AAk?$AAg?$AA?$AA@ 00000001800053e8     libucrt:lcidtoname_downlevel.obj
 0001:000043f8       ??_C@_1M@KPMILCJG@?$AAl?$AAt?$AA?9?$AAl?$AAt?$AA?$AA@ 00000001800053f8     libucrt:lcidtoname_downlevel.obj
 0001:00004408       ??_C@_1M@BDEKKCA@?$AAl?$AAv?$AA?9?$AAl?$AAv?$AA?$AA@ 0000000180005408     libucrt:lcidtoname_downlevel.obj
 0001:00004418       ??_C@_1M@ELCKCCJJ@?$AAm?$AAi?$AA?9?$AAn?$AAz?$AA?$AA@ 0000000180005418     libucrt:lcidtoname_downlevel.obj
 0001:00004428       ??_C@_1M@CBOOLAPA@?$AAm?$AAk?$AA?9?$AAm?$AAk?$AA?$AA@ 0000000180005428     libucrt:lcidtoname_downlevel.obj
 0001:00004438       ??_C@_1M@GPHNBJKN@?$AAm?$AAl?$AA?9?$AAi?$AAn?$AA?$AA@ 0000000180005438     libucrt:lcidtoname_downlevel.obj
 0001:00004448       ??_C@_1M@PABJILIG@?$AAm?$AAn?$AA?9?$AAm?$AAn?$AA?$AA@ 0000000180005448     libucrt:lcidtoname_downlevel.obj
 0001:00004458       ??_C@_1M@FGBKKIPG@?$AAm?$AAr?$AA?9?$AAi?$AAn?$AA?$AA@ 0000000180005458     libucrt:lcidtoname_downlevel.obj
 0001:00004468       ??_C@_1M@NDBPDDAL@?$AAm?$AAs?$AA?9?$AAb?$AAn?$AA?$AA@ 0000000180005468     libucrt:lcidtoname_downlevel.obj
 0001:00004478       ??_C@_1M@OPIHOOPI@?$AAm?$AAs?$AA?9?$AAm?$AAy?$AA?$AA@ 0000000180005478     libucrt:lcidtoname_downlevel.obj
 0001:00004488       ??_C@_1M@PPDBCNFM@?$AAm?$AAt?$AA?9?$AAm?$AAt?$AA?$AA@ 0000000180005488     libucrt:lcidtoname_downlevel.obj
 0001:00004498       ??_C@_1M@KDJDKMDD@?$AAn?$AAb?$AA?9?$AAn?$AAo?$AA?$AA@ 0000000180005498     libucrt:lcidtoname_downlevel.obj
 0001:000044a8       ??_C@_1M@KFCFLMJP@?$AAn?$AAl?$AA?9?$AAb?$AAe?$AA?$AA@ 00000001800054a8     libucrt:lcidtoname_downlevel.obj
 0001:000044b8       ??_C@_1M@KPOPDDGO@?$AAn?$AAl?$AA?9?$AAn?$AAl?$AA?$AA@ 00000001800054b8     libucrt:lcidtoname_downlevel.obj
 0001:000044c8       ??_C@_1M@LJKPEMLN@?$AAn?$AAn?$AA?9?$AAn?$AAo?$AA?$AA@ 00000001800054c8     libucrt:lcidtoname_downlevel.obj
 0001:000044d8       ??_C@_1M@BDGHHBFL@?$AAn?$AAs?$AA?9?$AAz?$AAa?$AA?$AA@ 00000001800054d8     libucrt:lcidtoname_downlevel.obj
 0001:000044e8       ??_C@_1M@IDEHOAP@?$AAp?$AAa?$AA?9?$AAi?$AAn?$AA?$AA@ 00000001800054e8     libucrt:lcidtoname_downlevel.obj
 0001:000044f8       ??_C@_1M@HDBKGOGH@?$AAp?$AAl?$AA?9?$AAp?$AAl?$AA?$AA@ 00000001800054f8     libucrt:lcidtoname_downlevel.obj
 0001:00004508       ??_C@_1M@LJLLCMEH@?$AAp?$AAt?$AA?9?$AAb?$AAr?$AA?$AA@ 0000000180005508     libucrt:lcidtoname_downlevel.obj
 0001:00004518       ??_C@_1M@NCMONAAL@?$AAp?$AAt?$AA?9?$AAp?$AAt?$AA?$AA@ 0000000180005518     libucrt:lcidtoname_downlevel.obj
 0001:00004528       ??_C@_1O@EAKMAJDN@?$AAq?$AAu?$AAz?$AA?9?$AAb?$AAo?$AA?$AA@ 0000000180005528     libucrt:lcidtoname_downlevel.obj
 0001:00004538       ??_C@_1O@BHHPIGDN@?$AAq?$AAu?$AAz?$AA?9?$AAe?$AAc?$AA?$AA@ 0000000180005538     libucrt:lcidtoname_downlevel.obj
 0001:00004548       ??_C@_1O@GBAPEKMJ@?$AAq?$AAu?$AAz?$AA?9?$AAp?$AAe?$AA?$AA@ 0000000180005548     libucrt:lcidtoname_downlevel.obj
 0001:00004558       ??_C@_1M@CLGLEFBO@?$AAr?$AAo?$AA?9?$AAr?$AAo?$AA?$AA@ 0000000180005558     libucrt:lcidtoname_downlevel.obj
 0001:00004568       ??_C@_1M@CEEDODME@?$AAr?$AAu?$AA?9?$AAr?$AAu?$AA?$AA@ 0000000180005568     libucrt:lcidtoname_downlevel.obj
 0001:00004578       ??_C@_1M@HPKKKMPP@?$AAs?$AAa?$AA?9?$AAi?$AAn?$AA?$AA@ 0000000180005578     libucrt:lcidtoname_downlevel.obj
 0001:00004588       ??_C@_1M@BKMAIGOJ@?$AAs?$AAe?$AA?9?$AAf?$AAi?$AA?$AA@ 0000000180005588     libucrt:lcidtoname_downlevel.obj
 0001:00004598       ??_C@_1M@NDPIFLFI@?$AAs?$AAe?$AA?9?$AAn?$AAo?$AA?$AA@ 0000000180005598     libucrt:lcidtoname_downlevel.obj
 0001:000045a8       ??_C@_1M@DANKKHJ@?$AAs?$AAe?$AA?9?$AAs?$AAe?$AA?$AA@ 00000001800055a8     libucrt:lcidtoname_downlevel.obj
 0001:000045b8       ??_C@_1M@PNBLONPJ@?$AAs?$AAk?$AA?9?$AAs?$AAk?$AA?$AA@ 00000001800055b8     libucrt:lcidtoname_downlevel.obj
 0001:000045c8       ??_C@_1M@LFMODOAL@?$AAs?$AAl?$AA?9?$AAs?$AAi?$AA?$AA@ 00000001800055c8     libucrt:lcidtoname_downlevel.obj
 0001:000045d8       ??_C@_1O@DFKOMPG@?$AAs?$AAm?$AAa?$AA?9?$AAn?$AAo?$AA?$AA@ 00000001800055d8     libucrt:lcidtoname_downlevel.obj
 0001:000045e8       ??_C@_1O@NDKPBNNH@?$AAs?$AAm?$AAa?$AA?9?$AAs?$AAe?$AA?$AA@ 00000001800055e8     libucrt:lcidtoname_downlevel.obj
 0001:000045f8       ??_C@_1O@PLLKBHAB@?$AAs?$AAm?$AAj?$AA?9?$AAn?$AAo?$AA?$AA@ 00000001800055f8     libucrt:lcidtoname_downlevel.obj
 0001:00004608       ??_C@_1O@CLEPOGCA@?$AAs?$AAm?$AAj?$AA?9?$AAs?$AAe?$AA?$AA@ 0000000180005608     libucrt:lcidtoname_downlevel.obj
 0001:00004618       ??_C@_1O@DLGJGKMK@?$AAs?$AAm?$AAn?$AA?9?$AAf?$AAi?$AA?$AA@ 0000000180005618     libucrt:lcidtoname_downlevel.obj
 0001:00004628       ??_C@_1O@OJDJGAJC@?$AAs?$AAm?$AAs?$AA?9?$AAf?$AAi?$AA?$AA@ 0000000180005628     libucrt:lcidtoname_downlevel.obj
 0001:00004638       ??_C@_1M@BOFOGHPB@?$AAs?$AAq?$AA?9?$AAa?$AAl?$AA?$AA@ 0000000180005638     libucrt:lcidtoname_downlevel.obj
 0001:00004648       ??_C@_1BG@LJBBIPGB@?$AAs?$AAr?$AA?9?$AAb?$AAa?$AA?9?$AAc?$AAy?$AAr?$AAl?$AA?$AA@ 0000000180005648     libucrt:lcidtoname_downlevel.obj
 0001:00004660       ??_C@_1BG@JLBENFOE@?$AAs?$AAr?$AA?9?$AAb?$AAa?$AA?9?$AAl?$AAa?$AAt?$AAn?$AA?$AA@ 0000000180005660     libucrt:lcidtoname_downlevel.obj
 0001:00004678       ??_C@_1BG@KODPNHE@?$AAs?$AAr?$AA?9?$AAs?$AAp?$AA?9?$AAc?$AAy?$AAr?$AAl?$AA?$AA@ 0000000180005678     libucrt:lcidtoname_downlevel.obj
 0001:00004690       ??_C@_1BG@CIOGKHPB@?$AAs?$AAr?$AA?9?$AAs?$AAp?$AA?9?$AAl?$AAa?$AAt?$AAn?$AA?$AA@ 0000000180005690     libucrt:lcidtoname_downlevel.obj
 0001:000046a8       ??_C@_1M@NGFJLMAC@?$AAs?$AAv?$AA?9?$AAf?$AAi?$AA?$AA@ 00000001800056a8     libucrt:lcidtoname_downlevel.obj
 0001:000046b8       ??_C@_1M@MPJEJAJC@?$AAs?$AAv?$AA?9?$AAs?$AAe?$AA?$AA@ 00000001800056b8     libucrt:lcidtoname_downlevel.obj
 0001:000046c8       ??_C@_1M@MPNDHLFK@?$AAs?$AAw?$AA?9?$AAk?$AAe?$AA?$AA@ 00000001800056c8     libucrt:lcidtoname_downlevel.obj
 0001:000046d8       ??_C@_1O@KOHBJJI@?$AAs?$AAy?$AAr?$AA?9?$AAs?$AAy?$AA?$AA@ 00000001800056d8     libucrt:lcidtoname_downlevel.obj
 0001:000046e8       ??_C@_1M@LDCEFHA@?$AAt?$AAa?$AA?9?$AAi?$AAn?$AA?$AA@ 00000001800056e8     libucrt:lcidtoname_downlevel.obj
 0001:000046f8       ??_C@_1M@CNJOFAK@?$AAt?$AAe?$AA?9?$AAi?$AAn?$AA?$AA@ 00000001800056f8     libucrt:lcidtoname_downlevel.obj
 0001:00004708       ??_C@_1M@GNAECACD@?$AAt?$AAh?$AA?9?$AAt?$AAh?$AA?$AA@ 0000000180005708     libucrt:lcidtoname_downlevel.obj
 0001:00004718       ??_C@_1M@CHBIHOJO@?$AAt?$AAn?$AA?9?$AAz?$AAa?$AA?$AA@ 0000000180005718     libucrt:lcidtoname_downlevel.obj
 0001:00004728       ??_C@_1M@GCCMIGPJ@?$AAt?$AAr?$AA?9?$AAt?$AAr?$AA?$AA@ 0000000180005728     libucrt:lcidtoname_downlevel.obj
 0001:00004738       ??_C@_1M@CELMCNBK@?$AAt?$AAt?$AA?9?$AAr?$AAu?$AA?$AA@ 0000000180005738     libucrt:lcidtoname_downlevel.obj
 0001:00004748       ??_C@_1M@KLMCELGA@?$AAu?$AAk?$AA?9?$AAu?$AAa?$AA?$AA@ 0000000180005748     libucrt:lcidtoname_downlevel.obj
 0001:00004758       ??_C@_1M@EPAJJAJF@?$AAu?$AAr?$AA?9?$AAp?$AAk?$AA?$AA@ 0000000180005758     libucrt:lcidtoname_downlevel.obj
 0001:00004768       ??_C@_1BG@GEGPMCDJ@?$AAu?$AAz?$AA?9?$AAu?$AAz?$AA?9?$AAc?$AAy?$AAr?$AAl?$AA?$AA@ 0000000180005768     libucrt:lcidtoname_downlevel.obj
 0001:00004780       ??_C@_1BG@EGGKJILM@?$AAu?$AAz?$AA?9?$AAu?$AAz?$AA?9?$AAl?$AAa?$AAt?$AAn?$AA?$AA@ 0000000180005780     libucrt:lcidtoname_downlevel.obj
 0001:00004798       ??_C@_1M@GFOCLFF@?$AAv?$AAi?$AA?9?$AAv?$AAn?$AA?$AA@ 0000000180005798     libucrt:lcidtoname_downlevel.obj
 0001:000047a8       ??_C@_1M@CPAMEDFI@?$AAx?$AAh?$AA?9?$AAz?$AAa?$AA?$AA@ 00000001800057a8     libucrt:lcidtoname_downlevel.obj
 0001:000047b8       ??_C@_1O@EBKIFIGN@?$AAz?$AAh?$AA?9?$AAc?$AAh?$AAs?$AA?$AA@ 00000001800057b8     libucrt:lcidtoname_downlevel.obj
 0001:000047c8       ??_C@_1O@NMHPGANE@?$AAz?$AAh?$AA?9?$AAc?$AAh?$AAt?$AA?$AA@ 00000001800057c8     libucrt:lcidtoname_downlevel.obj
 0001:000047d8       ??_C@_1M@LPINJOMC@?$AAz?$AAh?$AA?9?$AAc?$AAn?$AA?$AA@ 00000001800057d8     libucrt:lcidtoname_downlevel.obj
 0001:000047e8       ??_C@_1M@OCJEJODD@?$AAz?$AAh?$AA?9?$AAh?$AAk?$AA?$AA@ 00000001800057e8     libucrt:lcidtoname_downlevel.obj
 0001:000047f8       ??_C@_1M@DNDLJINH@?$AAz?$AAh?$AA?9?$AAm?$AAo?$AA?$AA@ 00000001800057f8     libucrt:lcidtoname_downlevel.obj
 0001:00004808       ??_C@_1M@MBFDNDND@?$AAz?$AAh?$AA?9?$AAs?$AAg?$AA?$AA@ 0000000180005808     libucrt:lcidtoname_downlevel.obj
 0001:00004818       ??_C@_1M@IMEPLEPE@?$AAz?$AAh?$AA?9?$AAt?$AAw?$AA?$AA@ 0000000180005818     libucrt:lcidtoname_downlevel.obj
 0001:00004828       ??_C@_1M@BBGHNHJP@?$AAz?$AAu?$AA?9?$AAz?$AAa?$AA?$AA@ 0000000180005828     libucrt:lcidtoname_downlevel.obj
 0001:00005680       ??_C@_15EMKDOKLE@?$AAa?$AAr?$AA?$AA@ 0000000180006680     libucrt:lcidtoname_downlevel.obj
 0001:00005688       ??_C@_15KNPADPLH@?$AAb?$AAg?$AA?$AA@ 0000000180006688     libucrt:lcidtoname_downlevel.obj
 0001:00005690       ??_C@_15EDMHLDMO@?$AAc?$AAa?$AA?$AA@ 0000000180006690     libucrt:lcidtoname_downlevel.obj
 0001:00005698       ??_C@_1O@BPEAJADD@?$AAz?$AAh?$AA?9?$AAC?$AAH?$AAS?$AA?$AA@ 0000000180006698     libucrt:lcidtoname_downlevel.obj
 0001:000056a8       ??_C@_15LJNHCMNK@?$AAc?$AAs?$AA?$AA@ 00000001800066a8     libucrt:lcidtoname_downlevel.obj
 0001:000056b0       ??_C@_15FOMCIDHG@?$AAd?$AAa?$AA?$AA@ 00000001800066b0     libucrt:lcidtoname_downlevel.obj
 0001:000056b8       ??_C@_15NBKABECB@?$AAd?$AAe?$AA?$AA@ 00000001800066b8     libucrt:lcidtoname_downlevel.obj
 0001:000056c0       ??_C@_15GHPEIIAO@?$AAe?$AAl?$AA?$AA@ 00000001800066c0     libucrt:lcidtoname_downlevel.obj
 0001:000056c8       ??_C@_15MNPNEAIF@?$AAe?$AAn?$AA?$AA@ 00000001800066c8     libucrt:lcidtoname_downlevel.obj
 0001:000056d0       ??_C@_15GPIOMPMH@?$AAe?$AAs?$AA?$AA@ 00000001800066d0     libucrt:lcidtoname_downlevel.obj
 0001:000056d8       ??_C@_15NGLOAKJC@?$AAf?$AAi?$AA?$AA@ 00000001800066d8     libucrt:lcidtoname_downlevel.obj
 0001:000056e0       ??_C@_15FBKGNKAM@?$AAf?$AAr?$AA?$AA@ 00000001800066e0     libucrt:lcidtoname_downlevel.obj
 0001:000056e8       ??_C@_15KGGCNEFK@?$AAh?$AAe?$AA?$AA@ 00000001800066e8     libucrt:lcidtoname_downlevel.obj
 0001:000056f0       ??_C@_15PGHLIDMF@?$AAh?$AAu?$AA?$AA@ 00000001800066f0     libucrt:lcidtoname_downlevel.obj
 0001:000056f8       ??_C@_15BIEMAPLM@?$AAi?$AAs?$AA?$AA@ 00000001800066f8     libucrt:lcidtoname_downlevel.obj
 0001:00005700       ??_C@_15IFJLDHAF@?$AAi?$AAt?$AA?$AA@ 0000000180006700     libucrt:lcidtoname_downlevel.obj
 0001:00005708       ??_C@_15GEMIOCAG@?$AAj?$AAa?$AA?$AA@ 0000000180006708     libucrt:lcidtoname_downlevel.obj
 0001:00005710       ??_C@_15EPELEGJA@?$AAk?$AAo?$AA?$AA@ 0000000180006710     libucrt:lcidtoname_downlevel.obj
 0001:00005718       ??_C@_15NDDHIMN@?$AAn?$AAl?$AA?$AA@ 0000000180006718     libucrt:lcidtoname_downlevel.obj
 0001:00005720       ??_C@_15BPIGNHCD@?$AAn?$AAo?$AA?$AA@ 0000000180006720     libucrt:lcidtoname_downlevel.obj
 0001:00005728       ??_C@_15DEOPBLCG@?$AAp?$AAl?$AA?$AA@ 0000000180006728     libucrt:lcidtoname_downlevel.obj
 0001:00005730       ??_C@_15KBECGEFG@?$AAp?$AAt?$AA?$AA@ 0000000180006730     libucrt:lcidtoname_downlevel.obj
 0001:00005738       ??_C@_15GLJCBFMD@?$AAr?$AAo?$AA?$AA@ 0000000180006738     libucrt:lcidtoname_downlevel.obj
 0001:00005740       ??_C@_15FEDGKCDI@?$AAr?$AAu?$AA?$AA@ 0000000180006740     libucrt:lcidtoname_downlevel.obj
 0001:00005748       ??_C@_15GLKMLLHM@?$AAh?$AAr?$AA?$AA@ 0000000180006748     libucrt:lcidtoname_downlevel.obj
 0001:00005750       ??_C@_15CPKMFBDB@?$AAs?$AAk?$AA?$AA@ 0000000180006750     libucrt:lcidtoname_downlevel.obj
 0001:00005758       ??_C@_15BAAIOGMK@?$AAs?$AAq?$AA?$AA@ 0000000180006758     libucrt:lcidtoname_downlevel.obj
 0001:00005760       ??_C@_15INNPNOHD@?$AAs?$AAv?$AA?$AA@ 0000000180006760     libucrt:lcidtoname_downlevel.obj
 0001:00005768       ??_C@_15CABMMOGH@?$AAt?$AAh?$AA?$AA@ 0000000180006768     libucrt:lcidtoname_downlevel.obj
 0001:00005770       ??_C@_15BPLIHJJM@?$AAt?$AAr?$AA?$AA@ 0000000180006770     libucrt:lcidtoname_downlevel.obj
 0001:00005778       ??_C@_15NEOEKKDJ@?$AAu?$AAr?$AA?$AA@ 0000000180006778     libucrt:lcidtoname_downlevel.obj
 0001:00005780       ??_C@_15NFICGAJK@?$AAi?$AAd?$AA?$AA@ 0000000180006780     libucrt:lcidtoname_downlevel.obj
 0001:00005788       ??_C@_15PJPFLCCM@?$AAu?$AAk?$AA?$AA@ 0000000180006788     libucrt:lcidtoname_downlevel.obj
 0001:00005790       ??_C@_15HPJPHDM@?$AAb?$AAe?$AA?$AA@ 0000000180006790     libucrt:lcidtoname_downlevel.obj
 0001:00005798       ??_C@_15LCHLGJII@?$AAs?$AAl?$AA?$AA@ 0000000180006798     libucrt:lcidtoname_downlevel.obj
 0001:000057a0       ??_C@_15PCFJPHHO@?$AAe?$AAt?$AA?$AA@ 00000001800067a0     libucrt:lcidtoname_downlevel.obj
 0001:000057a8       ??_C@_15HPFPGODN@?$AAl?$AAv?$AA?$AA@ 00000001800067a8     libucrt:lcidtoname_downlevel.obj
 0001:000057b0       ??_C@_15NFFGKGLG@?$AAl?$AAt?$AA?$AA@ 00000001800067b0     libucrt:lcidtoname_downlevel.obj
 0001:000057b8       ??_C@_15BDAKCCHN@?$AAf?$AAa?$AA?$AA@ 00000001800067b8     libucrt:lcidtoname_downlevel.obj
 0001:000057c0       ??_C@_15NFGIAIAJ@?$AAv?$AAi?$AA?$AA@ 00000001800067c0     libucrt:lcidtoname_downlevel.obj
 0001:000057c8       ??_C@_15LMKNDMHN@?$AAh?$AAy?$AA?$AA@ 00000001800067c8     libucrt:lcidtoname_downlevel.obj
 0001:000057d0       ??_C@_15IJBHMCFL@?$AAa?$AAz?$AA?$AA@ 00000001800067d0     libucrt:lcidtoname_downlevel.obj
 0001:000057d8       ??_C@_15EKOFJABL@?$AAe?$AAu?$AA?$AA@ 00000001800067d8     libucrt:lcidtoname_downlevel.obj
 0001:000057e0       ??_C@_15BGHADCNK@?$AAm?$AAk?$AA?$AA@ 00000001800067e0     libucrt:lcidtoname_downlevel.obj
 0001:000057e8       ??_C@_15JDNICKHM@?$AAa?$AAf?$AA?$AA@ 00000001800067e8     libucrt:lcidtoname_downlevel.obj
 0001:000057f0       ??_C@_15KPJEDBKD@?$AAk?$AAa?$AA?$AA@ 00000001800067f0     libucrt:lcidtoname_downlevel.obj
 0001:000057f8       ??_C@_15PDNFFFEO@?$AAf?$AAo?$AA?$AA@ 00000001800067f8     libucrt:lcidtoname_downlevel.obj
 0001:00005800       ??_C@_15OMLEGLOC@?$AAh?$AAi?$AA?$AA@ 0000000180006800     libucrt:lcidtoname_downlevel.obj
 0001:00005808       ??_C@_15IDNNENKK@?$AAm?$AAs?$AA?$AA@ 0000000180006808     libucrt:lcidtoname_downlevel.obj
 0001:00005810       ??_C@_15MACJNBMH@?$AAk?$AAk?$AA?$AA@ 0000000180006810     libucrt:lcidtoname_downlevel.obj
 0001:00005818       ??_C@_15DKDJEOND@?$AAk?$AAy?$AA?$AA@ 0000000180006818     libucrt:lcidtoname_downlevel.obj
 0001:00005820       ??_C@_15DFGDLJBG@?$AAs?$AAw?$AA?$AA@ 0000000180006820     libucrt:lcidtoname_downlevel.obj
 0001:00005828       ??_C@_15BBFAICNG@?$AAu?$AAz?$AA?$AA@ 0000000180006828     libucrt:lcidtoname_downlevel.obj
 0001:00005830       ??_C@_15DKNDCGEA@?$AAt?$AAt?$AA?$AA@ 0000000180006830     libucrt:lcidtoname_downlevel.obj
 0001:00005838       ??_C@_15MGIFMDPL@?$AAp?$AAa?$AA?$AA@ 0000000180006838     libucrt:lcidtoname_downlevel.obj
 0001:00005840       ??_C@_15HCNDBBA@?$AAg?$AAu?$AA?$AA@ 0000000180006840     libucrt:lcidtoname_downlevel.obj
 0001:00005848       ??_C@_15FNBEIBON@?$AAt?$AAa?$AA?$AA@ 0000000180006848     libucrt:lcidtoname_downlevel.obj
 0001:00005850       ??_C@_15NCHGBGLK@?$AAt?$AAe?$AA?$AA@ 0000000180006850     libucrt:lcidtoname_downlevel.obj
 0001:00005858       ??_C@_15PHPHCBPF@?$AAk?$AAn?$AA?$AA@ 0000000180006858     libucrt:lcidtoname_downlevel.obj
 0001:00005860       ??_C@_15DLGBCKMP@?$AAm?$AAr?$AA?$AA@ 0000000180006860     libucrt:lcidtoname_downlevel.obj
 0001:00005868       ??_C@_15EABBLBFF@?$AAs?$AAa?$AA?$AA@ 0000000180006868     libucrt:lcidtoname_downlevel.obj
 0001:00005870       ??_C@_15CBKOMCOI@?$AAm?$AAn?$AA?$AA@ 0000000180006870     libucrt:lcidtoname_downlevel.obj
 0001:00005878       ??_C@_15CKDMCJAF@?$AAg?$AAl?$AA?$AA@ 0000000180006878     libucrt:lcidtoname_downlevel.obj
 0001:00005880       ??_C@_17CNJFBPG@?$AAk?$AAo?$AAk?$AA?$AA@ 0000000180006880     libucrt:lcidtoname_downlevel.obj
 0001:00005888       ??_C@_17FFBJICPL@?$AAs?$AAy?$AAr?$AA?$AA@ 0000000180006888     libucrt:lcidtoname_downlevel.obj
 0001:00005890       ??_C@_17KPNDCPAF@?$AAd?$AAi?$AAv?$AA?$AA@ 0000000180006890     libucrt:lcidtoname_downlevel.obj
 0001:00005898       ??_C@_1M@OKAHONE@?$AAa?$AAr?$AA?9?$AAS?$AAA?$AA?$AA@ 0000000180006898     libucrt:lcidtoname_downlevel.obj
 0001:000058a8       ??_C@_1M@FFFIGIGK@?$AAb?$AAg?$AA?9?$AAB?$AAG?$AA?$AA@ 00000001800068a8     libucrt:lcidtoname_downlevel.obj
 0001:00005b10       ??_C@_1BA@BALFACEM@?$AAC?$AAO?$AAN?$AAO?$AAU?$AAT?$AA$?$AA?$AA@ 0000000180006b10     libucrt:initcon.obj
 0001:00005b20       __log10_256_lead           0000000180006b20     libucrt:log10_256_lead_tail_table.obj
 0001:00006330       __log10_256_tail           0000000180007330     libucrt:log10_256_lead_tail_table.obj
 0001:00006b40       __log_F_inv_qword          0000000180007b40     libucrt:log_f_inv_qword_table.obj
 0001:00007350       ??_C@_05HGHHAHAP@log10?$AA@ 0000000180008350     libucrt:log_special.obj
 0001:000073a0       _load_config_used          00000001800083a0     LIBCMT:loadcfg.obj
 0001:000074a0       ??_R4exception@std@@6B@    00000001800084a0     LIBCMT:throw_bad_alloc.obj
 0001:000074c8       ??_R3exception@std@@8      00000001800084c8     LIBCMT:throw_bad_alloc.obj
 0001:000074e0       ??_R2exception@std@@8      00000001800084e0     LIBCMT:throw_bad_alloc.obj
 0001:000074f0       ??_R1A@?0A@EA@exception@std@@8 00000001800084f0     LIBCMT:throw_bad_alloc.obj
 0001:00007518       ??_R4bad_alloc@std@@6B@    0000000180008518     LIBCMT:throw_bad_alloc.obj
 0001:00007540       ??_R3bad_alloc@std@@8      0000000180008540     LIBCMT:throw_bad_alloc.obj
 0001:00007558       ??_R2bad_alloc@std@@8      0000000180008558     LIBCMT:throw_bad_alloc.obj
 0001:00007570       ??_R1A@?0A@EA@bad_alloc@std@@8 0000000180008570     LIBCMT:throw_bad_alloc.obj
 0001:00007598       ??_R4bad_array_new_length@std@@6B@ 0000000180008598     LIBCMT:throw_bad_alloc.obj
 0001:000075c0       ??_R3bad_array_new_length@std@@8 00000001800085c0     LIBCMT:throw_bad_alloc.obj
 0001:000075d8       ??_R2bad_array_new_length@std@@8 00000001800085d8     LIBCMT:throw_bad_alloc.obj
 0001:000075f8       ??_R1A@?0A@EA@bad_array_new_length@std@@8 00000001800085f8     LIBCMT:throw_bad_alloc.obj
 0001:00007620       ??_R4type_info@@6B@        0000000180008620     LIBCMT:std_type_info_static.obj
 0001:00007648       ??_R3type_info@@8          0000000180008648     LIBCMT:std_type_info_static.obj
 0001:00007660       ??_R2type_info@@8          0000000180008660     LIBCMT:std_type_info_static.obj
 0001:00007670       ??_R1A@?0A@EA@type_info@@8 0000000180008670     LIBCMT:std_type_info_static.obj
 0001:00007948       __rtc_iaa                  0000000180008948     LIBCMT:_initsect_.obj
 0001:00007950       __rtc_izz                  0000000180008950     LIBCMT:_initsect_.obj
 0001:00007958       __rtc_taa                  0000000180008958     LIBCMT:_initsect_.obj
 0001:00007960       __rtc_tzz                  0000000180008960     LIBCMT:_initsect_.obj
 0001:00007980       __chkstk                   0000000180008980 f   chkstk.obj
 0001:00007980       _alloca_probe              0000000180008980 f   chkstk.obj
 0001:000079e0       ??1?$DialogBuilderBase@UFarDialogItem@@@@MEAA@XZ 00000001800089e0 f i Brackets.obj
 0001:00007a60       ??_E?$DialogBuilderBase@UFarDialogItem@@@@MEAAPEAXI@Z 0000000180008a60 f i Brackets.obj
 0001:00007a60       ??_G?$DialogBuilderBase@UFarDialogItem@@@@MEAAPEAXI@Z 0000000180008a60 f i Brackets.obj
 0001:00007aa0       ??_G?$DialogItemBinding@UFarDialogItem@@@@UEAAPEAXI@Z 0000000180008aa0 f i Brackets.obj
 0001:00007aa0       ??_E?$DialogItemBinding@UFarDialogItem@@@@UEAAPEAXI@Z 0000000180008aa0 f i Brackets.obj
 0001:00007ad0       ??_EPluginCheckBoxBinding@@UEAAPEAXI@Z 0000000180008ad0 f i Brackets.obj
 0001:00007ad0       ??_GPluginEditFieldBinding@@UEAAPEAXI@Z 0000000180008ad0 f i Brackets.obj
 0001:00007ad0       ??_EPluginEditFieldBinding@@UEAAPEAXI@Z 0000000180008ad0 f i Brackets.obj
 0001:00007ad0       ??_GPluginCheckBoxBinding@@UEAAPEAXI@Z 0000000180008ad0 f i Brackets.obj
 0001:00007b00       ??_GPluginDialogBuilder@@UEAAPEAXI@Z 0000000180008b00 f i Brackets.obj
 0001:00007b00       ??_EPluginDialogBuilder@@UEAAPEAXI@Z 0000000180008b00 f i Brackets.obj
 0001:00007b50       ??_EPluginUIntEditFieldBinding@@UEAAPEAXI@Z 0000000180008b50 f i Brackets.obj
 0001:00007b50       ??_GPluginUIntEditFieldBinding@@UEAAPEAXI@Z 0000000180008b50 f i Brackets.obj
 0001:00007b50       ??_EPluginIntEditFieldBinding@@UEAAPEAXI@Z 0000000180008b50 f i Brackets.obj
 0001:00007b50       ??_GPluginIntEditFieldBinding@@UEAAPEAXI@Z 0000000180008b50 f i Brackets.obj
 0001:00007b80       ??_EPluginRadioButtonBinding@@UEAAPEAXI@Z 0000000180008b80 f i Brackets.obj
 0001:00007b80       ??_GPluginRadioButtonBinding@@UEAAPEAXI@Z 0000000180008b80 f i Brackets.obj
 0001:00007bb0       ?AddButtons@?$DialogBuilderBase@UFarDialogItem@@@@QEAAXHPEBHHH@Z 0000000180008bb0 f i Brackets.obj
 0001:00007ec0       ?AddDialogItem@?$DialogBuilderBase@UFarDialogItem@@@@IEAAPEAUFarDialogItem@@W4FARDIALOGITEMTYPES@@PEB_W@Z 0000000180008ec0 f i Brackets.obj
 0001:00008070       ?AddUIntEditField@?$DialogBuilderBase@UFarDialogItem@@@@UEAAPEAUFarDialogItem@@PEAIH@Z 0000000180009070 f i Brackets.obj
 0001:00008070       ?AddIntEditField@?$DialogBuilderBase@UFarDialogItem@@@@UEAAPEAUFarDialogItem@@PEAHH@Z 0000000180009070 f i Brackets.obj
 0001:00008070       ?CreateCheckBoxBinding@?$DialogBuilderBase@UFarDialogItem@@@@MEAAPEAU?$DialogItemBinding@UFarDialogItem@@@@PEAHH@Z 0000000180009070 f i Brackets.obj
 0001:00008070       ?CreateRadioButtonBinding@?$DialogBuilderBase@UFarDialogItem@@@@MEAAPEAU?$DialogItemBinding@UFarDialogItem@@@@PEAH@Z 0000000180009070 f i Brackets.obj
 0001:00008070       ?GetLangString@?$DialogBuilderBase@UFarDialogItem@@@@MEAAPEB_WH@Z 0000000180009070 f i Brackets.obj
 0001:00008080       ?AddIntEditField@PluginDialogBuilder@@UEAAPEAUFarDialogItem@@PEAHH@Z 0000000180009080 f i Brackets.obj
 0001:000081e0       ?AddUIntEditField@PluginDialogBuilder@@UEAAPEAUFarDialogItem@@PEAIH@Z 00000001800091e0 f i Brackets.obj
 0001:00008340       ?Config@@YAHXZ             0000000180009340 f   Brackets.obj
 0001:00009160       ?CreateCheckBoxBinding@PluginDialogBuilder@@MEAAPEAU?$DialogItemBinding@UFarDialogItem@@@@PEAHH@Z 000000018000a160 f i Brackets.obj
 0001:000091e0       ?CreateRadioButtonBinding@PluginDialogBuilder@@MEAAPEAU?$DialogItemBinding@UFarDialogItem@@@@PEAH@Z 000000018000a1e0 f i Brackets.obj
 0001:00009250       ?DoShowDialog@?$DialogBuilderBase@UFarDialogItem@@@@MEAA_JXZ 000000018000a250 f i Brackets.obj
 0001:00009260       ?DoShowDialog@PluginDialogBuilder@@MEAA_JXZ 000000018000a260 f i Brackets.obj
 0001:00009310       ?GetLangString@PluginDialogBuilder@@MEAAPEB_WH@Z 000000018000a310 f i Brackets.obj
 0001:00009320       _guard_check_icall_nop     000000018000a320 f i LIBCMT:guard_support.obj
 0001:00009320       ?InitDialogItem@?$DialogBuilderBase@UFarDialogItem@@@@MEAAXPEAUFarDialogItem@@PEB_W@Z 000000018000a320 f i Brackets.obj
 0001:00009320       ?SaveValue@?$DialogItemBinding@UFarDialogItem@@@@UEAAXPEAUFarDialogItem@@H@Z 000000018000a320 f i Brackets.obj
 0001:00009330       ?InitDialogItem@PluginDialogBuilder@@MEAAXPEAUFarDialogItem@@PEB_W@Z 000000018000a330 f i Brackets.obj
 0001:00009360       ?SaveValue@PluginCheckBoxBinding@@UEAAXPEAUFarDialogItem@@H@Z 000000018000a360 f i Brackets.obj
 0001:000093c0       ?SaveValue@PluginEditFieldBinding@@UEAAXPEAUFarDialogItem@@H@Z 000000018000a3c0 f i Brackets.obj
 0001:00009400       ?SaveValue@PluginIntEditFieldBinding@@UEAAXPEAUFarDialogItem@@H@Z 000000018000a400 f i Brackets.obj
 0001:00009450       ?SaveValue@PluginRadioButtonBinding@@UEAAXPEAUFarDialogItem@@H@Z 000000018000a450 f i Brackets.obj
 0001:000094a0       ?SaveValue@PluginUIntEditFieldBinding@@UEAAXPEAUFarDialogItem@@H@Z 000000018000a4a0 f i Brackets.obj
 0001:000094f0       ?ShowMenu@@YAHH@Z          000000018000a4f0 f   Brackets.obj
 0001:00009680       ?TextWidth@?$DialogBuilderBase@UFarDialogItem@@@@MEAAHAEBUFarDialogItem@@@Z 000000018000a680 f i Brackets.obj
 0001:00009690       ?TextWidth@PluginDialogBuilder@@MEAAHAEBUFarDialogItem@@@Z 000000018000a690 f i Brackets.obj
 0001:000096a0       ?UpdateBorderSize@?$DialogBuilderBase@UFarDialogItem@@@@IEAAXXZ 000000018000a6a0 f i Brackets.obj
 0001:00009880       ConfigureW                 000000018000a880 f   Brackets.obj
 0001:00009890       GetGlobalInfoW             000000018000a890 f   Brackets.obj
 0001:00009910       GetPluginInfoW             000000018000a910 f   Brackets.obj
 0001:00009980       OpenW                      000000018000a980 f   Brackets.obj
 0001:0000a690       SetStartupInfoW            000000018000b690 f   Brackets.obj
 0001:0000a9dc       ??2@YAPEAX_K@Z             000000018000b9dc f   LIBCMT:new_scalar.obj
 0001:0000aa18       ??3@YAXPEAX_K@Z            000000018000ba18 f   LIBCMT:delete_scalar_size.obj
 0001:0000aa18       ??_V@YAXPEAX@Z             000000018000ba18 f   LIBCMT:delete_array.obj
 0001:0000aa20       ??_U@YAPEAX_K@Z            000000018000ba20 f   LIBCMT:new_array.obj
 0001:0000ad48       _DllMainCRTStartup         000000018000bd48 f   LIBCMT:dll_dllmain.obj
 0001:0000ad88       ??0bad_alloc@std@@QEAA@AEBV01@@Z 000000018000bd88 f i LIBCMT:throw_bad_alloc.obj
 0001:0000adc8       ??0bad_alloc@std@@QEAA@XZ  000000018000bdc8 f i LIBCMT:throw_bad_alloc.obj
 0001:0000ade8       ??0bad_array_new_length@std@@QEAA@AEBV01@@Z 000000018000bde8 f i LIBCMT:throw_bad_alloc.obj
 0001:0000ae28       ??0bad_array_new_length@std@@QEAA@XZ 000000018000be28 f i LIBCMT:throw_bad_alloc.obj
 0001:0000ae48       ??0exception@std@@QEAA@AEBV01@@Z 000000018000be48 f i LIBCMT:throw_bad_alloc.obj
 0001:0000ae80       ??1bad_array_new_length@std@@UEAA@XZ 000000018000be80 f i LIBCMT:throw_bad_alloc.obj
 0001:0000ae80       ??1bad_alloc@std@@UEAA@XZ  000000018000be80 f i LIBCMT:throw_bad_alloc.obj
 0001:0000ae94       ??_Ebad_array_new_length@std@@UEAAPEAXI@Z 000000018000be94 f i LIBCMT:throw_bad_alloc.obj
 0001:0000ae94       ??_Gbad_array_new_length@std@@UEAAPEAXI@Z 000000018000be94 f i LIBCMT:throw_bad_alloc.obj
 0001:0000ae94       ??_Eexception@std@@UEAAPEAXI@Z 000000018000be94 f i LIBCMT:throw_bad_alloc.obj
 0001:0000ae94       ??_Gexception@std@@UEAAPEAXI@Z 000000018000be94 f i LIBCMT:throw_bad_alloc.obj
 0001:0000ae94       ??_Gbad_alloc@std@@UEAAPEAXI@Z 000000018000be94 f i LIBCMT:throw_bad_alloc.obj
 0001:0000ae94       ??_Ebad_alloc@std@@UEAAPEAXI@Z 000000018000be94 f i LIBCMT:throw_bad_alloc.obj
 0001:0000aed8       ?__scrt_throw_std_bad_alloc@@YAXXZ 000000018000bed8 f   LIBCMT:throw_bad_alloc.obj
 0001:0000aef8       ?__scrt_throw_std_bad_array_new_length@@YAXXZ 000000018000bef8 f   LIBCMT:throw_bad_alloc.obj
 0001:0000af18       ?what@exception@std@@UEBAPEBDXZ 000000018000bf18 f i LIBCMT:throw_bad_alloc.obj
 0001:0000af2c       ??3@YAXPEAX@Z              000000018000bf2c f   LIBCMT:delete_scalar.obj
 0001:0000af34       __security_init_cookie     000000018000bf34 f   LIBCMT:gs_support.obj
 0001:0000afe4       DllMain                    000000018000bfe4 f   LIBCMT:dll_dllmain_stub.obj
 0001:0000afe4       _get_startup_argv_mode     000000018000bfe4 f   LIBCMT:argv_mode.obj
 0001:0000afec       ?__scrt_initialize_type_info@@YAXXZ 000000018000bfec f   LIBCMT:tncleanup.obj
 0001:0000affc       ?__scrt_uninitialize_type_info@@YAXXZ 000000018000bffc f   LIBCMT:tncleanup.obj
 0001:0000b008       __local_stdio_printf_options 000000018000c008 f i LIBCMT:default_local_stdio_options.obj
 0001:0000b010       __local_stdio_scanf_options 000000018000c010 f i LIBCMT:default_local_stdio_options.obj
 0001:0000b018       __scrt_initialize_default_local_stdio_options 000000018000c018 f   LIBCMT:default_local_stdio_options.obj
 0001:0000b034       __scrt_acquire_startup_lock 000000018000c034 f   LIBCMT:utility.obj
 0001:0000b070       __scrt_dllmain_after_initialize_c 000000018000c070 f   LIBCMT:utility.obj
 0001:0000b0a4       __scrt_dllmain_before_initialize_c 000000018000c0a4 f   LIBCMT:utility.obj
 0001:0000b0bc       __scrt_dllmain_crt_thread_attach 000000018000c0bc f   LIBCMT:utility.obj
 0001:0000b0e4       __scrt_dllmain_crt_thread_detach 000000018000c0e4 f   LIBCMT:utility.obj
 0001:0000b0fc       __scrt_dllmain_exception_filter 000000018000c0fc f   LIBCMT:utility.obj
 0001:0000b15c       __scrt_dllmain_uninitialize_c 000000018000c15c f   LIBCMT:utility.obj
 0001:0000b18c       __scrt_dllmain_uninitialize_critical 000000018000c18c f   LIBCMT:utility.obj
 0001:0000b1a0       __scrt_initialize_crt      000000018000c1a0 f   LIBCMT:utility.obj
 0001:0000b1ec       __scrt_initialize_onexit_tables 000000018000c1ec f   LIBCMT:utility.obj
 0001:0000b2c8       __scrt_is_nonwritable_in_current_image 000000018000c2c8 f   LIBCMT:utility.obj
 0001:0000b364       __scrt_release_startup_lock 000000018000c364 f   LIBCMT:utility.obj
 0001:0000b388       __scrt_uninitialize_crt    000000018000c388 f   LIBCMT:utility.obj
 0001:0000b3b4       __scrt_get_dyn_tls_init_callback 000000018000c3b4 f   LIBCMT:dyn_tls_init.obj
 0001:0000b3bc       __crt_debugger_hook        000000018000c3bc f   LIBCMT:utility_desktop.obj
 0001:0000b3c4       __scrt_fastfail            000000018000c3c4 f   LIBCMT:utility_desktop.obj
 0001:0000b510       _RTC_Initialize            000000018000c510 f   LIBCMT:_initsect_.obj
 0001:0000b54c       _RTC_Terminate             000000018000c54c f   LIBCMT:_initsect_.obj
 0001:0000b588       ??_Etype_info@@UEAAPEAXI@Z 000000018000c588 f i LIBCMT:std_type_info_static.obj
 0001:0000b588       ??_Gtype_info@@UEAAPEAXI@Z 000000018000c588 f i LIBCMT:std_type_info_static.obj
 0001:0000b5b4       __isa_available_init       000000018000c5b4 f   LIBCMT:_cpu_disp_.obj
 0001:0000b770       __scrt_is_ucrt_dll_in_use  000000018000c770 f   LIBCMT:ucrt_detection.obj
 0001:0000b790       memset                     000000018000c790 f   libvcruntime:memset.obj
 0001:0000b940       __C_specific_handler       000000018000c940 f   libvcruntime:_riscchandler_.obj
 0001:0000bb4c       __std_exception_copy       000000018000cb4c f   libvcruntime:std_exception.obj
 0001:0000bbdc       __std_exception_destroy    000000018000cbdc f   libvcruntime:std_exception.obj
 0001:0000bc04       _CxxThrowException         000000018000cc04 f   libvcruntime:throw.obj
 0001:0000bcc4       __std_type_info_destroy_list 000000018000ccc4 f   libvcruntime:std_type_info.obj
 0001:0000bcf0       __vcrt_initialize          000000018000ccf0 f   libvcruntime:initialization.obj
 0001:0000bd24       __vcrt_thread_attach       000000018000cd24 f   libvcruntime:initialization.obj
 0001:0000bd38       __vcrt_thread_detach       000000018000cd38 f   libvcruntime:initialization.obj
 0001:0000bd4c       __vcrt_uninitialize        000000018000cd4c f   libvcruntime:initialization.obj
 0001:0000bd6c       __vcrt_uninitialize_critical 000000018000cd6c f   libvcruntime:initialization.obj
 0001:0000bd90       _local_unwind              000000018000cd90 f   libvcruntime:_jmpuwind_.obj
 0001:0000bdc0       _NLG_Notify                000000018000cdc0 f   libvcruntime:_jmpuwind_.obj
 0001:0000bde0       __NLG_Dispatch2            000000018000cde0 f   libvcruntime:_jmpuwind_.obj
 0001:0000bdf0       __NLG_Return2              000000018000cdf0 f   libvcruntime:_jmpuwind_.obj
 0001:0000bdf4       __except_validate_context_record 000000018000cdf4 f   libvcruntime:jbcxrval.obj
 0001:0000be2c       __vcrt_freefls             000000018000ce2c f   libvcruntime:per_thread_data.obj
 0001:0000be4c       __vcrt_freeptd             000000018000ce4c f   libvcruntime:per_thread_data.obj
 0001:0000be9c       __vcrt_getptd_noexit       000000018000ce9c f   libvcruntime:per_thread_data.obj
 0001:0000bf54       __vcrt_initialize_ptd      000000018000cf54 f   libvcruntime:per_thread_data.obj
 0001:0000bfa4       __vcrt_uninitialize_ptd    000000018000cfa4 f   libvcruntime:per_thread_data.obj
 0001:0000bfc8       __vcrt_initialize_locks    000000018000cfc8 f   libvcruntime:locks.obj
 0001:0000c010       __vcrt_uninitialize_locks  000000018000d010 f   libvcruntime:locks.obj
 0001:0000c220       __vcrt_FlsAlloc            000000018000d220 f   libvcruntime:winapi_downlevel.obj
 0001:0000c268       __vcrt_FlsFree             000000018000d268 f   libvcruntime:winapi_downlevel.obj
 0001:0000c2b0       __vcrt_FlsGetValue         000000018000d2b0 f   libvcruntime:winapi_downlevel.obj
 0001:0000c2f8       __vcrt_FlsSetValue         000000018000d2f8 f   libvcruntime:winapi_downlevel.obj
 0001:0000c34c       __vcrt_InitializeCriticalSectionEx 000000018000d34c f   libvcruntime:winapi_downlevel.obj
 0001:0000c3b0       __vcrt_initialize_winapi_thunks 000000018000d3b0 f   libvcruntime:winapi_downlevel.obj
 0001:0000c3e0       __vcrt_uninitialize_winapi_thunks 000000018000d3e0 f   libvcruntime:winapi_downlevel.obj
 0001:0000c420       __vcrt_initialize_pure_virtual_call_handler 000000018000d420 f   libvcruntime:purevirt_data.obj
 0001:0000c440       memmove                    000000018000d440 f   libvcruntime:memcpy.obj
 0001:0000c440       memcpy                     000000018000d440 f   libvcruntime:memcpy.obj
 0001:0000c8a0       _CallSettingFrame          000000018000d8a0 f   libvcruntime:handlers.obj
 0001:0000c8e0       __DestructExceptionObject  000000018000d8e0 f   libvcruntime:ehhelpers.obj
 0001:0000c954       ?_CallMemberFunction0@@YAXQEAX0@Z 000000018000d954 f i libvcruntime:ehhelpers.obj
 0001:0000c958       __acrt_initialize_new_handler 000000018000d958 f   libucrt:new_handler.obj
 0001:0000c960       _callnewh                  000000018000d960 f   libucrt:new_handler.obj
 0001:0000c990       _query_new_handler         000000018000d990 f   libucrt:new_handler.obj
 0001:0000c9c4       malloc                     000000018000d9c4 f   libucrt:malloc.obj
 0001:0000c9cc       _initterm                  000000018000d9cc f   libucrt:initterm.obj
 0001:0000ca30       _initterm_e                000000018000da30 f   libucrt:initterm.obj
 0001:0000ca70       free                       000000018000da70 f   libucrt:free.obj
 0001:0000ca84       _seh_filter_dll            000000018000da84 f   libucrt:exception_filter.obj
 0001:0000ca98       _seh_filter_exe            000000018000da98 f   libucrt:exception_filter.obj
 0001:0000cea4       __acrt_initialize_thread_local_exit_callback 000000018000dea4 f   libucrt:exit.obj
 0001:0000ceac       _cexit                     000000018000deac f   libucrt:exit.obj
 0001:0000cebc       _exit                      000000018000debc f   libucrt:exit.obj
 0001:0000cec8       _is_c_termination_complete 000000018000dec8 f   libucrt:exit.obj
 0001:0000d08c       __acrt_allocate_buffer_for_argv 000000018000e08c f   libucrt:argv_parsing.obj
 0001:0000d0ec       _configure_narrow_argv     000000018000e0ec f   libucrt:argv_parsing.obj
 0001:0000d468       __dcrt_uninitialize_environments_nolock 000000018000e468 f   libucrt:environment_initialization.obj
 0001:0000d4a0       _initialize_narrow_environment 000000018000e4a0 f   libucrt:environment_initialization.obj
 0001:0000d630       _execute_onexit_table      000000018000e630 f   libucrt:onexit.obj
 0001:0000d66c       _initialize_onexit_table   000000018000e66c f   libucrt:onexit.obj
 0001:0000d6e4       __acrt_uninitialize_command_line 000000018000e6e4 f   libucrt:argv_data.obj
 0001:0000d7f0       __acrt_initialize          000000018000e7f0 f   libucrt:initialization.obj
 0001:0000d804       __acrt_thread_attach       000000018000e804 f   libucrt:initialization.obj
 0001:0000d818       __acrt_thread_detach       000000018000e818 f   libucrt:initialization.obj
 0001:0000d828       __acrt_uninitialize        000000018000e828 f   libucrt:initialization.obj
 0001:0000d860       __acrt_uninitialize_critical 000000018000e860 f   libucrt:initialization.obj
 0001:0000d870       terminate                  000000018000e870 f   libucrt:terminate.obj
 0001:0000d890       strcpy_s                   000000018000e890 f   libucrt:strcpy_s.obj
 0001:0000d8f0       ??0_LocaleUpdate@@QEAA@QEAU__crt_locale_pointers@@@Z 000000018000e8f0 f i libucrt:output.obj
 0001:0000d990       strncmp                    000000018000e990 f   libucrt:strncmp.obj
 0001:0000da10       abort                      000000018000ea10 f   libucrt:abort.obj
 0001:0000da68       calloc                     000000018000ea68 f   libucrt:calloc.obj
 0001:0000da70       wcsncmp                    000000018000ea70 f   libucrt:wcsncmp.obj
 0001:0000da9c       __acrt_initialize_locks    000000018000ea9c f   libucrt:locks.obj
 0001:0000dae4       __acrt_lock                000000018000eae4 f   libucrt:locks.obj
 0001:0000db00       __acrt_uninitialize_locks  000000018000eb00 f   libucrt:locks.obj
 0001:0000db38       __acrt_unlock              000000018000eb38 f   libucrt:locks.obj
 0001:0000db54       _malloc_base               000000018000eb54 f   libucrt:malloc_base.obj
 0001:0000dbb4       _free_base                 000000018000ebb4 f   libucrt:free_base.obj
 0001:0000df6c       __acrt_freeptd             000000018000ef6c f   libucrt:per_thread_data.obj
 0001:0000dfb0       __acrt_getptd              000000018000efb0 f   libucrt:per_thread_data.obj
 0001:0000e07c       __acrt_getptd_head         000000018000f07c f   libucrt:per_thread_data.obj
 0001:0000e124       __acrt_getptd_noexit       000000018000f124 f   libucrt:per_thread_data.obj
 0001:0000e1f4       __acrt_initialize_ptd      000000018000f1f4 f   libucrt:per_thread_data.obj
 0001:0000e230       __acrt_uninitialize_ptd    000000018000f230 f   libucrt:per_thread_data.obj
 0001:0000e254       __acrt_get_process_end_policy 000000018000f254 f   libucrt:win_policies.obj
 0001:0000e290       __acrt_call_reportfault    000000018000f290 f   libucrt:invalid_parameter.obj
 0001:0000e3ec       __acrt_initialize_invalid_parameter_handler 000000018000f3ec f   libucrt:invalid_parameter.obj
 0001:0000e3f4       _invalid_parameter         000000018000f3f4 f   libucrt:invalid_parameter.obj
 0001:0000e4a4       _invalid_parameter_noinfo  000000018000f4a4 f   libucrt:invalid_parameter.obj
 0001:0000e4c4       _invoke_watson             000000018000f4c4 f   libucrt:invalid_parameter.obj
 0001:0000e50c       __acrt_errno_from_os_error 000000018000f50c f   libucrt:errno.obj
 0001:0000e554       __acrt_errno_map_os_error  000000018000f554 f   libucrt:errno.obj
 0001:0000e5a4       __doserrno                 000000018000f5a4 f   libucrt:errno.obj
 0001:0000e5c4       _errno                     000000018000f5c4 f   libucrt:errno.obj
 0001:0000e5e4       _calloc_base               000000018000f5e4 f   libucrt:calloc_base.obj
 0001:0000ebc0       __acrt_expand_narrow_argv_wildcards 000000018000fbc0 f   libucrt:argv_wildcards.obj
 0001:0000f308       __acrt_initialize_multibyte 0000000180010308 f   libucrt:mbctype.obj
 0001:0000f368       __acrt_update_thread_multibyte_data 0000000180010368 f   libucrt:mbctype.obj
 0001:0000f384       _setmbcp_nolock            0000000180010384 f   libucrt:mbctype.obj
 0001:0000f6bc       _ismbblead                 00000001800106bc f   libucrt:ismbbyte.obj
 0001:0000f6d0       __acrt_initialize_command_line 00000001800106d0 f   libucrt:argv_data.obj
 0001:0000f6f8       __dcrt_get_narrow_environment_from_os 00000001800106f8 f   libucrt:get_environment_from_os.obj
 0001:0000f7fc       _recalloc                  00000001800107fc f   libucrt:recalloc.obj
 0001:0000f804       _recalloc_base             0000000180010804 f   libucrt:recalloc.obj
 0001:0000fa74       __acrt_AppPolicyGetProcessTerminationMethodInternal 0000000180010a74 f   libucrt:winapi_thunks.obj
 0001:0000fac4       __acrt_FlsAlloc            0000000180010ac4 f   libucrt:winapi_thunks.obj
 0001:0000fb0c       __acrt_FlsFree             0000000180010b0c f   libucrt:winapi_thunks.obj
 0001:0000fb54       __acrt_FlsGetValue         0000000180010b54 f   libucrt:winapi_thunks.obj
 0001:0000fb9c       __acrt_FlsSetValue         0000000180010b9c f   libucrt:winapi_thunks.obj
 0001:0000fbf0       __acrt_InitializeCriticalSectionEx 0000000180010bf0 f   libucrt:winapi_thunks.obj
 0001:0000fc54       __acrt_LCMapStringEx       0000000180010c54 f   libucrt:winapi_thunks.obj
 0001:0000fd30       __acrt_LocaleNameToLCID    0000000180010d30 f   libucrt:winapi_thunks.obj
 0001:0000fd80       __acrt_initialize_winapi_thunks 0000000180010d80 f   libucrt:winapi_thunks.obj
 0001:0000fdc8       __acrt_uninitialize_winapi_thunks 0000000180010dc8 f   libucrt:winapi_thunks.obj
 0001:0000fe0c       __acrt_initialize_heap     0000000180010e0c f   libucrt:heap_handle.obj
 0001:0000fe28       __acrt_uninitialize_heap   0000000180010e28 f   libucrt:heap_handle.obj
 0001:0001001c       __acrt_initialize_lowio    000000018001101c f   libucrt:ioinit.obj
 0001:00010058       __acrt_uninitialize_lowio  0000000180011058 f   libucrt:ioinit.obj
 0001:00010098       __acrt_execute_initializers 0000000180011098 f   libucrt:shared_initialization.obj
 0001:00010118       __acrt_execute_uninitializers 0000000180011118 f   libucrt:shared_initialization.obj
 0001:0001019c       __acrt_get_sigabrt_handler 000000018001119c f   libucrt:signal.obj
 0001:000101cc       __acrt_initialize_signal_handlers 00000001800111cc f   libucrt:signal.obj
 0001:000101ec       raise                      00000001800111ec f   libucrt:signal.obj
 0001:00010460       __acrt_has_user_matherr    0000000180011460 f   libucrt:matherr.obj
 0001:00010480       __acrt_initialize_user_matherr 0000000180011480 f   libucrt:matherr.obj
 0001:00010488       __acrt_invoke_user_matherr 0000000180011488 f   libucrt:matherr.obj
 0001:0001069c       __acrt_stdio_flush_nolock  000000018001169c f   libucrt:fflush.obj
 0001:00010718       _fflush_nolock             0000000180011718 f   libucrt:fflush.obj
 0001:00010764       _flushall                  0000000180011764 f   libucrt:fflush.obj
 0001:0001076c       __acrt_initialize_stdio    000000018001176c f   libucrt:_file.obj
 0001:0001088c       __acrt_uninitialize_stdio  000000018001188c f   libucrt:_file.obj
 0001:000108e8       _lock_file                 00000001800118e8 f   libucrt:_file.obj
 0001:000108f4       _unlock_file               00000001800118f4 f   libucrt:_file.obj
 0001:00010900       _mbtowc_l                  0000000180011900 f   libucrt:mbtowc.obj
 0001:00010a48       mbtowc                     0000000180011a48 f   libucrt:mbtowc.obj
 0001:00010a50       __acrt_update_locale_info  0000000180011a50 f   libucrt:locale_update.obj
 0001:00010a84       __acrt_update_multibyte_info 0000000180011a84 f   libucrt:locale_update.obj
 0001:00010ab8       _fileno                    0000000180011ab8 f   libucrt:fileno.obj
 0001:00010b50       __acrt_set_locale_changed  0000000180011b50 f   libucrt:wsetlocale.obj
 0001:00010b5c       __acrt_uninitialize_locale 0000000180011b5c f   libucrt:wsetlocale.obj
 0001:00010b8c       __pctype_func              0000000180011b8c f   libucrt:ctype.obj
 0001:00010bbc       _query_new_mode            0000000180011bbc f   libucrt:new_mode.obj
 0001:00010bc4       __acrt_add_locale_ref      0000000180011bc4 f   libucrt:locale_refcounting.obj
 0001:00010c50       __acrt_free_locale         0000000180011c50 f   libucrt:locale_refcounting.obj
 0001:00010dc8       __acrt_locale_add_lc_time_reference 0000000180011dc8 f   libucrt:locale_refcounting.obj
 0001:00010df0       __acrt_locale_free_lc_time_if_unreferenced 0000000180011df0 f   libucrt:locale_refcounting.obj
 0001:00010e28       __acrt_locale_release_lc_time_reference 0000000180011e28 f   libucrt:locale_refcounting.obj
 0001:00010e50       __acrt_release_locale_ref  0000000180011e50 f   libucrt:locale_refcounting.obj
 0001:00010ef8       __acrt_update_thread_locale_data 0000000180011ef8 f   libucrt:locale_refcounting.obj
 0001:00010f68       _updatetlocinfoEx_nolock   0000000180011f68 f   libucrt:locale_refcounting.obj
 0001:00010fd0       qsort                      0000000180011fd0 f   libucrt:qsort.obj
 0001:00011380       strncpy_s                  0000000180012380 f   libucrt:strncpy_s.obj
 0001:00011500       strpbrk                    0000000180012500 f   libucrt:strpbrk.obj
 0001:000118e0       _mbsdec                    00000001800128e0 f   libucrt:mbsdec.obj
 0001:000118e8       _mbsdec_l                  00000001800128e8 f   libucrt:mbsdec.obj
 0001:00011990       __acrt_GetStringTypeA      0000000180012990 f   libucrt:getstringtypea.obj
 0001:00011e38       __acrt_LCMapStringA        0000000180012e38 f   libucrt:lcmapstringa.obj
 0001:00011ed0       _msize                     0000000180012ed0 f   libucrt:msize.obj
 0001:00011ed8       _msize_base                0000000180012ed8 f   libucrt:msize.obj
 0001:00011f14       _realloc_base              0000000180012f14 f   libucrt:realloc_base.obj
 0001:0001205c       __acrt_DownlevelLocaleNameToLCID 000000018001305c f   libucrt:lcidtoname_downlevel.obj
 0001:00012090       __acrt_lowio_create_handle_array 0000000180013090 f   libucrt:osfinfo.obj
 0001:00012128       __acrt_lowio_destroy_handle_array 0000000180013128 f   libucrt:osfinfo.obj
 0001:00012178       __acrt_lowio_ensure_fh_exists 0000000180013178 f   libucrt:osfinfo.obj
 0001:00012220       __acrt_lowio_lock_fh       0000000180013220 f   libucrt:osfinfo.obj
 0001:00012244       __acrt_lowio_unlock_fh     0000000180013244 f   libucrt:osfinfo.obj
 0001:00012268       _free_osfhnd               0000000180013268 f   libucrt:osfinfo.obj
 0001:00012324       _get_osfhandle             0000000180013324 f   libucrt:osfinfo.obj
 0001:00012428       _commit                    0000000180013428 f   libucrt:commit.obj
 0001:00012a74       _write                     0000000180013a74 f   libucrt:write.obj
 0001:00012b60       _write_nolock              0000000180013b60 f   libucrt:write.obj
 0001:00012ea4       _fcloseall                 0000000180013ea4 f   libucrt:closeall.obj
 0001:00012f58       __acrt_stdio_free_buffer_nolock 0000000180013f58 f   libucrt:_freebuf.obj
 0001:00012f98       _isatty                    0000000180013f98 f   libucrt:isatty.obj
 0001:00012ff8       _isleadbyte_l              0000000180013ff8 f i libucrt:_wctype.obj
 0001:00013038       __acrt_MultiByteToWideChar 0000000180014038 f   libucrt:multibytetowidechar.obj
 0001:00013040       __acrt_locale_free_monetary 0000000180014040 f   libucrt:initmon.obj
 0001:0001314c       __acrt_locale_free_numeric 000000018001414c f   libucrt:initnum.obj
 0001:0001320c       __acrt_locale_free_time    000000018001420c f   libucrt:inittime.obj
 0001:00013314       __strncnt                  0000000180014314 f   libucrt:strncnt.obj
 0001:0001332c       _query_app_type            000000018001432c f   libucrt:report_runtime_error.obj
 0001:000133d0       _lseeki64_nolock           00000001800143d0 f   libucrt:lseek.obj
 0001:000133d8       _putwch_nolock             00000001800143d8 f   libucrt:putwch.obj
 0001:00013414       _fclose_nolock             0000000180014414 f   libucrt:fclose.obj
 0001:00013498       fclose                     0000000180014498 f   libucrt:fclose.obj
 0001:00013500       log10                      0000000180014500 f   libucrt:log10.obj
 0001:00013aac       __dcrt_lowio_ensure_console_output_initialized 0000000180014aac f   libucrt:initcon.obj
 0001:00013b00       __dcrt_terminate_console_output 0000000180014b00 f   libucrt:initcon.obj
 0001:00013b1c       __dcrt_write_console_w     0000000180014b1c f   libucrt:initcon.obj
 0001:00013c50       _close                     0000000180014c50 f   libucrt:close.obj
 0001:00013cf4       _close_nolock              0000000180014cf4 f   libucrt:close.obj
 0001:00013db0       ?__acrt_stdio_free_stream@@YAXV__crt_stdio_stream@@@Z 0000000180014db0 f   libucrt:stream.obj
 0001:00013ef0       _handle_error              0000000180014ef0 f   libucrt:libm_error.obj
 0001:00014020       __acrt_initialize_fma3     0000000180015020 f   libucrt:fma3_available.obj
 0001:00014090       _log10_special             0000000180015090 f   libucrt:log_special.obj
 0001:00014160       _get_fpsr                  0000000180015160 f   libucrt:fpsr.obj
 0001:00014170       _set_fpsr                  0000000180015170 f   libucrt:fpsr.obj
 0001:0001417a       _fclrf                     000000018001517a f   libucrt:fpsr.obj
 0001:0001418e       _frnd                      000000018001518e f   libucrt:fpsr.obj
 0001:000141b0       _raise_exc                 00000001800151b0 f   libucrt:fpexcept.obj
 0001:000141d8       _raise_exc_ex              00000001800151d8 f   libucrt:fpexcept.obj
 0001:000144e0       _set_errno_from_matherr    00000001800154e0 f   libucrt:fpexcept.obj
 0001:00014510       _clrfp                     0000000180015510 f   libucrt:fpctrl.obj
 0001:00014530       _ctrlfp                    0000000180015530 f   libucrt:fpctrl.obj
 0001:000145ac       _set_statfp                00000001800155ac f   libucrt:fpctrl.obj
 0001:000145cc       _statfp                    00000001800155cc f   libucrt:fpctrl.obj
 0001:000145dd       IsProcessorFeaturePresent  00000001800155dd f   kernel32:KERNEL32.dll
 0001:000145e3       RtlUnwindEx                00000001800155e3 f   kernel32:KERNEL32.dll
 0001:000145f0       _FindPESection             00000001800155f0 f   LIBCMT:pesect.obj
 0001:00014640       _IsNonwritableInCurrentImage 0000000180015640 f   LIBCMT:pesect.obj
 0001:00014690       _ValidateImageBase         0000000180015690 f   LIBCMT:pesect.obj
 0001:000146c0       __GSHandlerCheck           00000001800156c0 f   LIBCMT:_gshandler_.obj
 0001:000146e0       __GSHandlerCheckCommon     00000001800156e0 f   LIBCMT:_gshandler_.obj
 0001:00014750       __security_check_cookie    0000000180015750 f   LIBCMT:_amdsecgs_.obj
 0001:00014774       __raise_securityfailure    0000000180015774 f   LIBCMT:gs_report.obj
 0001:000147a8       __report_gsfailure         00000001800157a8 f   LIBCMT:gs_report.obj
 0001:0001487c       __report_rangecheckfailure 000000018001587c f   LIBCMT:gs_report.obj
 0001:00014890       __report_securityfailure   0000000180015890 f   LIBCMT:gs_report.obj
 0001:00014a20       memcmp                     0000000180015a20 f   libvcruntime:memcmp.obj
 0001:00014b00       _guard_dispatch_icall_nop  0000000180015b00 f   LIBCMT:_guard_dispatch_.obj
 0001:000158f8       _TI2?AVbad_alloc@std@@     00000001800168f8     LIBCMT:throw_bad_alloc.obj
 0001:00015918       _CTA2?AVbad_alloc@std@@    0000000180016918     LIBCMT:throw_bad_alloc.obj
 0001:00015930       _CT??_R0?AVbad_alloc@std@@@8??0bad_alloc@std@@QEAA@AEBV01@@Z24 0000000180016930     LIBCMT:throw_bad_alloc.obj
 0001:00015958       _CT??_R0?AVexception@std@@@8??0exception@std@@QEAA@AEBV01@@Z24 0000000180016958     LIBCMT:throw_bad_alloc.obj
 0001:00015980       _TI3?AVbad_array_new_length@std@@ 0000000180016980     LIBCMT:throw_bad_alloc.obj
 0001:000159a0       _CTA3?AVbad_array_new_length@std@@ 00000001800169a0     LIBCMT:throw_bad_alloc.obj
 0001:000159c0       _CT??_R0?AVbad_array_new_length@std@@@8??0bad_array_new_length@std@@QEAA@AEBV01@@Z24 00000001800169c0     LIBCMT:throw_bad_alloc.obj
 0002:00000070       __scrt_native_dllmain_reason 0000000180017070     LIBCMT:utility.obj
 0002:00000078       __security_cookie          0000000180017078     LIBCMT:gs_cookie.obj
 0002:00000080       __security_cookie_complement 0000000180017080     LIBCMT:gs_cookie.obj
 0002:00000088       __isa_available            0000000180017088     LIBCMT:_cpu_disp_.obj
 0002:0000008c       __isa_enabled              000000018001708c     LIBCMT:_cpu_disp_.obj
 0002:00000090       __memcpy_nt_iters          0000000180017090     LIBCMT:_cpu_disp_.obj
 0002:000000b0       __abort_behavior           00000001800170b0     libucrt:abort.obj
 0002:000000c0       __acrt_initial_multibyte_data 00000001800170c0     libucrt:mbctype.obj
 0002:00000600       __acrt_initial_locale_data 0000000180017600     libucrt:nlsdata.obj
 0002:00000758       __acrt_initial_locale_pointers 0000000180017758     libucrt:nlsdata.obj
 0002:00000768       __acrt_wide_c_locale_string 0000000180017768     libucrt:nlsdata.obj
 0002:00000770       _iob                       0000000180017770     libucrt:_file.obj
 0002:00000878       __globallocalestatus       0000000180017878     libucrt:glstatus.obj
 0002:00000880       __acrt_lconv_c             0000000180017880     libucrt:localeconv.obj
 0002:00000918       __acrt_lconv_static_decimal 0000000180017918     libucrt:localeconv.obj
 0002:0000091c       __acrt_lconv_static_W_decimal 000000018001791c     libucrt:localeconv.obj
 0002:00000940       _fltused                   0000000180017940     LIBCMT:fltused.obj
 0002:00000950       ??_R0?AVbad_alloc@std@@@8  0000000180017950     LIBCMT:throw_bad_alloc.obj
 0002:00000978       ??_R0?AVexception@std@@@8  0000000180017978     LIBCMT:throw_bad_alloc.obj
 0002:000009a0       ??_R0?AVbad_array_new_length@std@@@8 00000001800179a0     LIBCMT:throw_bad_alloc.obj
 0002:000009d0       ??_R0?AVtype_info@@@8      00000001800179d0     LIBCMT:std_type_info_static.obj
 0002:00000bd0       ?__type_info_root_node@@3U__type_info_node@@A 0000000180017bd0     LIBCMT:tncleanup.obj
 0002:00000be0       ?_OptionsStorage@?1??__local_stdio_printf_options@@9@4_KA 0000000180017be0     LIBCMT:default_local_stdio_options.obj
 0002:00000be8       ?_OptionsStorage@?1??__local_stdio_scanf_options@@9@4_KA 0000000180017be8     LIBCMT:default_local_stdio_options.obj
 0002:00000bf0       __scrt_current_native_startup_state 0000000180017bf0     LIBCMT:utility.obj
 0002:00000bf8       __scrt_native_startup_lock 0000000180017bf8     LIBCMT:utility.obj
 0002:00000c34       __scrt_debugger_hook_flag  0000000180017c34     LIBCMT:utility_desktop.obj
 0002:00000c38       __favor                    0000000180017c38     LIBCMT:_cpu_disp_.obj
 0002:00000c40       ?m_pGetParameter@UnDecorator@@0P6APEADJ@ZEA 0000000180017c40     libvcruntime:undname.obj
 0002:00000c48       ?m_CHPENameOffset@UnDecorator@@0KA 0000000180017c48     libvcruntime:undname.obj
 0002:00000c4c       ?m_recursionLevel@UnDecorator@@0KA 0000000180017c4c     libvcruntime:undname.obj
 0002:00000c50       ?pArgList@UnDecorator@@0PEAVReplicator@@EA 0000000180017c50     libvcruntime:undname.obj
 0002:00000c58       ?pZNameList@UnDecorator@@0PEAVReplicator@@EA 0000000180017c58     libvcruntime:undname.obj
 0002:00000c60       ?pTemplateArgList@UnDecorator@@0PEAVReplicator@@EA 0000000180017c60     libvcruntime:undname.obj
 0002:00000c68       ?gName@UnDecorator@@0PEBDEB 0000000180017c68     libvcruntime:undname.obj
 0002:00000c70       ?name@UnDecorator@@0PEBDEB 0000000180017c70     libvcruntime:undname.obj
 0002:00000c78       ?disableFlags@UnDecorator@@0KA 0000000180017c78     libvcruntime:undname.obj
 0002:00000c7c       ?fExplicitTemplateParams@UnDecorator@@0_NA 0000000180017c7c     libvcruntime:undname.obj
 0002:00000c7d       ?fGetTemplateArgumentList@UnDecorator@@0_NA 0000000180017c7d     libvcruntime:undname.obj
 0002:00000d98       __pPurecall                0000000180017d98     libvcruntime:purevirt_data.obj
 0002:00000da0       ?__WinRTOutOfMemoryExceptionCallback@@3P6APEAXXZEA 0000000180017da0     libvcruntime:ehhelpers.obj
 0002:00000dc0       ?c_exit_complete@?1???R<lambda_6e4b09c48022b2350581041d5f6b0c4c>@@QEBA@XZ@4_NA 0000000180017dc0     libucrt:exit.obj
 0002:00000ed8       _environ_table             0000000180017ed8     libucrt:environment_initialization.obj
 0002:00000ee0       _wenviron_table            0000000180017ee0     libucrt:environment_initialization.obj
 0002:00000ee8       __dcrt_initial_wide_environment 0000000180017ee8     libucrt:environment_initialization.obj
 0002:00000ef0       __dcrt_initial_narrow_environment 0000000180017ef0     libucrt:environment_initialization.obj
 0002:00000ef8       __acrt_atexit_table        0000000180017ef8     libucrt:onexit.obj
 0002:00000f10       __acrt_at_quick_exit_table 0000000180017f10     libucrt:onexit.obj
 0002:00001170       __acrt_current_multibyte_data 0000000180018170     libucrt:mbctype.obj
 0002:00001178       _mbctype                   0000000180018178     libucrt:mbctype.obj
 0002:00001180       _mbcasemap                 0000000180018180     libucrt:mbctype.obj
 0002:00001190       __argc                     0000000180018190     libucrt:argv_data.obj
 0002:00001198       __argv                     0000000180018198     libucrt:argv_data.obj
 0002:000011a0       __wargv                    00000001800181a0     libucrt:argv_data.obj
 0002:000011a8       _acmdln                    00000001800181a8     libucrt:argv_data.obj
 0002:000011b0       _wcmdln                    00000001800181b0     libucrt:argv_data.obj
 0002:000011b8       _pgmptr                    00000001800181b8     libucrt:argv_data.obj
 0002:00001370       __acrt_heap                0000000180018370     libucrt:heap_handle.obj
 0002:00001380       __pioinfo                  0000000180018380     libucrt:ioinit.obj
 0002:00001780       _nhandle                   0000000180018780     libucrt:ioinit.obj
 0002:000017b0       __acrt_current_locale_data 00000001800187b0     libucrt:nlsdata.obj
 0002:000017b8       _nstream                   00000001800187b8     libucrt:_file.obj
 0002:000017c0       __piob                     00000001800187c0     libucrt:_file.obj
 0002:000017c8       __acrt_stdout_buffer       00000001800187c8     libucrt:_sftbuf.obj
 0002:000017d0       __acrt_stderr_buffer       00000001800187d0     libucrt:_sftbuf.obj
 0002:000017d8       __acrt_locale_changed_data 00000001800187d8     libucrt:wsetlocale.obj
 0002:000017e0       __acrt_lconv_static_null   00000001800187e0     libucrt:localeconv.obj
 0002:000017e4       __acrt_lconv_static_W_null 00000001800187e4     libucrt:localeconv.obj
 0002:000017ec       __fma3_is_available        00000001800187ec     libucrt:fma3_available.obj
 0002:000017f0       __use_fma3_lib             00000001800187f0     libucrt:fma3_available.obj
 0002:00001d70       __scrt_ucrt_dll_is_in_use  0000000180018d70     <common>
 0002:00001d78       __dyn_tls_init_callback    0000000180018d78     <common>
 0004:00000000       __imp_lstrcmpiW            000000018001a000     kernel32:KERNEL32.dll
 0004:00000008       __imp_lstrcpynW            000000018001a008     kernel32:KERNEL32.dll
 0004:00000010       __imp_lstrlenW             000000018001a010     kernel32:KERNEL32.dll
 0004:00000018       __imp_CloseHandle          000000018001a018     kernel32:KERNEL32.dll
 0004:00000020       __imp_CreateFileW          000000018001a020     kernel32:KERNEL32.dll
 0004:00000028       __imp_SetFilePointerEx     000000018001a028     kernel32:KERNEL32.dll
 0004:00000030       __imp_QueryPerformanceCounter 000000018001a030     kernel32:KERNEL32.dll
 0004:00000038       __imp_GetCurrentProcessId  000000018001a038     kernel32:KERNEL32.dll
 0004:00000040       __imp_GetCurrentThreadId   000000018001a040     kernel32:KERNEL32.dll
 0004:00000048       __imp_GetSystemTimeAsFileTime 000000018001a048     kernel32:KERNEL32.dll
 0004:00000050       __imp_InitializeSListHead  000000018001a050     kernel32:KERNEL32.dll
 0004:00000058       __imp_RtlCaptureContext    000000018001a058     kernel32:KERNEL32.dll
 0004:00000060       __imp_RtlLookupFunctionEntry 000000018001a060     kernel32:KERNEL32.dll
 0004:00000068       __imp_RtlVirtualUnwind     000000018001a068     kernel32:KERNEL32.dll
 0004:00000070       __imp_IsDebuggerPresent    000000018001a070     kernel32:KERNEL32.dll
 0004:00000078       __imp_UnhandledExceptionFilter 000000018001a078     kernel32:KERNEL32.dll
 0004:00000080       __imp_SetUnhandledExceptionFilter 000000018001a080     kernel32:KERNEL32.dll
 0004:00000088       __imp_GetStartupInfoW      000000018001a088     kernel32:KERNEL32.dll
 0004:00000090       __imp_IsProcessorFeaturePresent 000000018001a090     kernel32:KERNEL32.dll
 0004:00000098       __imp_GetModuleHandleW     000000018001a098     kernel32:KERNEL32.dll
 0004:000000a0       __imp_RtlUnwindEx          000000018001a0a0     kernel32:KERNEL32.dll
 0004:000000a8       __imp_RtlPcToFileHeader    000000018001a0a8     kernel32:KERNEL32.dll
 0004:000000b0       __imp_RaiseException       000000018001a0b0     kernel32:KERNEL32.dll
 0004:000000b8       __imp_InterlockedFlushSList 000000018001a0b8     kernel32:KERNEL32.dll
 0004:000000c0       __imp_GetLastError         000000018001a0c0     kernel32:KERNEL32.dll
 0004:000000c8       __imp_SetLastError         000000018001a0c8     kernel32:KERNEL32.dll
 0004:000000d0       __imp_EnterCriticalSection 000000018001a0d0     kernel32:KERNEL32.dll
 0004:000000d8       __imp_LeaveCriticalSection 000000018001a0d8     kernel32:KERNEL32.dll
 0004:000000e0       __imp_DeleteCriticalSection 000000018001a0e0     kernel32:KERNEL32.dll
 0004:000000e8       __imp_InitializeCriticalSectionAndSpinCount 000000018001a0e8     kernel32:KERNEL32.dll
 0004:000000f0       __imp_TlsAlloc             000000018001a0f0     kernel32:KERNEL32.dll
 0004:000000f8       __imp_TlsGetValue          000000018001a0f8     kernel32:KERNEL32.dll
 0004:00000100       __imp_TlsSetValue          000000018001a100     kernel32:KERNEL32.dll
 0004:00000108       __imp_TlsFree              000000018001a108     kernel32:KERNEL32.dll
 0004:00000110       __imp_FreeLibrary          000000018001a110     kernel32:KERNEL32.dll
 0004:00000118       __imp_GetProcAddress       000000018001a118     kernel32:KERNEL32.dll
 0004:00000120       __imp_LoadLibraryExW       000000018001a120     kernel32:KERNEL32.dll
 0004:00000128       __imp_GetCurrentProcess    000000018001a128     kernel32:KERNEL32.dll
 0004:00000130       __imp_ExitProcess          000000018001a130     kernel32:KERNEL32.dll
 0004:00000138       __imp_TerminateProcess     000000018001a138     kernel32:KERNEL32.dll
 0004:00000140       __imp_GetModuleHandleExW   000000018001a140     kernel32:KERNEL32.dll
 0004:00000148       __imp_GetModuleFileNameA   000000018001a148     kernel32:KERNEL32.dll
 0004:00000150       __imp_MultiByteToWideChar  000000018001a150     kernel32:KERNEL32.dll
 0004:00000158       __imp_WideCharToMultiByte  000000018001a158     kernel32:KERNEL32.dll
 0004:00000160       __imp_HeapAlloc            000000018001a160     kernel32:KERNEL32.dll
 0004:00000168       __imp_HeapFree             000000018001a168     kernel32:KERNEL32.dll
 0004:00000170       __imp_FindClose            000000018001a170     kernel32:KERNEL32.dll
 0004:00000178       __imp_FindFirstFileExA     000000018001a178     kernel32:KERNEL32.dll
 0004:00000180       __imp_FindNextFileA        000000018001a180     kernel32:KERNEL32.dll
 0004:00000188       __imp_IsValidCodePage      000000018001a188     kernel32:KERNEL32.dll
 0004:00000190       __imp_GetACP               000000018001a190     kernel32:KERNEL32.dll
 0004:00000198       __imp_GetOEMCP             000000018001a198     kernel32:KERNEL32.dll
 0004:000001a0       __imp_GetCPInfo            000000018001a1a0     kernel32:KERNEL32.dll
 0004:000001a8       __imp_GetCommandLineA      000000018001a1a8     kernel32:KERNEL32.dll
 0004:000001b0       __imp_GetCommandLineW      000000018001a1b0     kernel32:KERNEL32.dll
 0004:000001b8       __imp_GetEnvironmentStringsW 000000018001a1b8     kernel32:KERNEL32.dll
 0004:000001c0       __imp_FreeEnvironmentStringsW 000000018001a1c0     kernel32:KERNEL32.dll
 0004:000001c8       __imp_LCMapStringW         000000018001a1c8     kernel32:KERNEL32.dll
 0004:000001d0       __imp_GetProcessHeap       000000018001a1d0     kernel32:KERNEL32.dll
 0004:000001d8       __imp_GetStdHandle         000000018001a1d8     kernel32:KERNEL32.dll
 0004:000001e0       __imp_GetFileType          000000018001a1e0     kernel32:KERNEL32.dll
 0004:000001e8       __imp_GetStringTypeW       000000018001a1e8     kernel32:KERNEL32.dll
 0004:000001f0       __imp_HeapSize             000000018001a1f0     kernel32:KERNEL32.dll
 0004:000001f8       __imp_HeapReAlloc          000000018001a1f8     kernel32:KERNEL32.dll
 0004:00000200       __imp_SetStdHandle         000000018001a200     kernel32:KERNEL32.dll
 0004:00000208       __imp_FlushFileBuffers     000000018001a208     kernel32:KERNEL32.dll
 0004:00000210       __imp_WriteFile            000000018001a210     kernel32:KERNEL32.dll
 0004:00000218       __imp_GetConsoleCP         000000018001a218     kernel32:KERNEL32.dll
 0004:00000220       __imp_GetConsoleMode       000000018001a220     kernel32:KERNEL32.dll
 0004:00000228       __imp_WriteConsoleW        000000018001a228     kernel32:KERNEL32.dll
 0004:00000230       \177KERNEL32_NULL_THUNK_DATA 000000018001a230     kernel32:KERNEL32.dll
 0004:00000238       __imp_MessageBeep          000000018001a238     user32:USER32.dll
 0004:00000240       \177USER32_NULL_THUNK_DATA 000000018001a240     user32:USER32.dll
 0004:00000248       __guard_check_icall_fptr   000000018001a248     LIBCMT:guard_support.obj
 0004:00000250       __guard_dispatch_icall_fptr 000000018001a250     LIBCMT:guard_support.obj
 0004:00000258       __IMPORT_DESCRIPTOR_KERNEL32 000000018001a258     kernel32:KERNEL32.dll
 0004:0000026c       __IMPORT_DESCRIPTOR_USER32 000000018001a26c     user32:USER32.dll
 0004:00000280       __NULL_IMPORT_DESCRIPTOR   000000018001a280     kernel32:KERNEL32.dll

 entry point at        0001:0000ad48

 Static symbols

 0001:000004c0       ?ExceptionTemplate@?1??_CxxThrowException@@9@4UEHExceptionRecord@@B 00000001800014c0     libvcruntime:throw.obj
 0001:00000500       ?tokenTable@@3QBQEBDB      0000000180001500     libvcruntime:undname.obj
 0001:00000578       ?rttiTable@@3QBQEBDB       0000000180001578     libvcruntime:undname.obj
 0001:000005a0       ?nameTable@@3QBQEBDB       00000001800015a0     libvcruntime:undname.obj
 0001:00000ea8       ?module_names@?A0x89697e75@@3QBQEB_WB 0000000180001ea8     libvcruntime:winapi_downlevel.obj
 0001:00000f78       ?candidate_modules@?1??try_get_FlsAlloc@@YAP6AKP6AXPEAX@Z@ZXZ@4QBW4module_id@?A0x89697e75@@B 0000000180001f78     libvcruntime:winapi_downlevel.obj
 0001:00000f90       ?candidate_modules@?1??try_get_FlsFree@@YAP6AHK@ZXZ@4QBW4module_id@?A0x89697e75@@B 0000000180001f90     libvcruntime:winapi_downlevel.obj
 0001:00000fa0       ?candidate_modules@?1??try_get_FlsGetValue@@YAP6APEAXK@ZXZ@4QBW4module_id@?A0x89697e75@@B 0000000180001fa0     libvcruntime:winapi_downlevel.obj
 0001:00000fb8       ?candidate_modules@?1??try_get_FlsSetValue@@YAP6AHKPEAX@ZXZ@4QBW4module_id@?A0x89697e75@@B 0000000180001fb8     libvcruntime:winapi_downlevel.obj
 0001:00000fd0       ?candidate_modules@?1??try_get_InitializeCriticalSectionEx@@YAP6AHPEAU_RTL_CRITICAL_SECTION@@KK@ZXZ@4QBW4module_id@?A0x89697e75@@B 0000000180001fd0     libvcruntime:winapi_downlevel.obj
 0001:00001100       __acrt_initializers        0000000180002100     libucrt:initialization.obj
 0001:00001200       ?errtable@@3QBUerrentry@?A0x31fdb9ec@@B 0000000180002200     libucrt:errno.obj
 0001:00001360       ?_mb_locale_names@@3QBQEB_WB 0000000180002360     libucrt:mbctype.obj
 0001:000013c0       ?module_names@?A0x391cf84c@@3QBQEB_WB 00000001800023c0     libucrt:winapi_thunks.obj
 0001:000018b8       ?candidate_modules@?1??try_get_FlsAlloc@@YAP6AKP6AXPEAX@Z@ZXZ@4QBW4module_id@?A0x391cf84c@@B 00000001800028b8     libucrt:winapi_thunks.obj
 0001:000018c0       ?candidate_modules@?1??try_get_FlsFree@@YAP6AHK@ZXZ@4QBW4module_id@?A0x391cf84c@@B 00000001800028c0     libucrt:winapi_thunks.obj
 0001:000018c8       ?candidate_modules@?1??try_get_FlsGetValue@@YAP6APEAXK@ZXZ@4QBW4module_id@?A0x391cf84c@@B 00000001800028c8     libucrt:winapi_thunks.obj
 0001:000018d0       ?candidate_modules@?1??try_get_FlsSetValue@@YAP6AHKPEAX@ZXZ@4QBW4module_id@?A0x391cf84c@@B 00000001800028d0     libucrt:winapi_thunks.obj
 0001:000018d8       ?candidate_modules@?1??try_get_InitializeCriticalSectionEx@@YAP6AHPEAU_RTL_CRITICAL_SECTION@@KK@ZXZ@4QBW4module_id@?A0x391cf84c@@B 00000001800028d8     libucrt:winapi_thunks.obj
 0001:000018e0       ?candidate_modules@?1??try_get_LCMapStringEx@@YAP6AHPEB_WK0HPEA_WHPEAU_nlsversioninfo@@PEAX_J@ZXZ@4QBW4module_id@?A0x391cf84c@@B 00000001800028e0     libucrt:winapi_thunks.obj
 0001:000018f8       ?candidate_modules@?1??try_get_LocaleNameToLCID@@YAP6AKPEB_WK@ZXZ@4QBW4module_id@?A0x391cf84c@@B 00000001800028f8     libucrt:winapi_thunks.obj
 0001:00001914       ?candidate_modules@?1??try_get_AppPolicyGetProcessTerminationMethod@@YAP6AJPEAXPEAW4AppPolicyProcessTerminationMethod@@@ZXZ@4QBW4module_id@?A0x391cf84c@@B 0000000180002914     libucrt:winapi_thunks.obj
 0001:00002fa0       ?LocaleNameToIndexTable@?A0x881e4c05@@3QBULocaleNameIndex@1@B 0000000180003fa0     libucrt:lcidtoname_downlevel.obj
 0001:00004840       ?LcidToLocaleNameTable@?A0x881e4c05@@3QBULcidToLocaleName@1@B 0000000180005840     libucrt:lcidtoname_downlevel.obj
 0001:000058c0       __real_ninf                00000001800068c0     libucrt:log10.obj
 0001:000058d0       __real_inf                 00000001800068d0     libucrt:log10.obj
 0001:000058e0       __real_neg_qnan            00000001800068e0     libucrt:log10.obj
 0001:000058f0       __real_qnanbit             00000001800068f0     libucrt:log10.obj
 0001:00005900       __int_1023                 0000000180006900     libucrt:log10.obj
 0001:00005910       __mask_001                 0000000180006910     libucrt:log10.obj
 0001:00005920       __mask_mant                0000000180006920     libucrt:log10.obj
 0001:00005930       __mask_mant_top8           0000000180006930     libucrt:log10.obj
 0001:00005940       __mask_mant9               0000000180006940     libucrt:log10.obj
 0001:00005950       __real_log10_e             0000000180006950     libucrt:log10.obj
 0001:00005960       __real_log10_e_lead        0000000180006960     libucrt:log10.obj
 0001:00005970       __real_log10_e_tail        0000000180006970     libucrt:log10.obj
 0001:00005980       __real_log10_2_lead        0000000180006980     libucrt:log10.obj
 0001:00005990       __real_log10_2_tail        0000000180006990     libucrt:log10.obj
 0001:000059a0       __real_two                 00000001800069a0     libucrt:log10.obj
 0001:000059b0       __real_one                 00000001800069b0     libucrt:log10.obj
 0001:000059c0       __real_half                00000001800069c0     libucrt:log10.obj
 0001:000059d0       __mask_100                 00000001800069d0     libucrt:log10.obj
 0001:000059e0       __real_1_over_512          00000001800069e0     libucrt:log10.obj
 0001:000059f0       __real_1_over_2            00000001800069f0     libucrt:log10.obj
 0001:00005a00       __real_1_over_3            0000000180006a00     libucrt:log10.obj
 0001:00005a10       __real_1_over_4            0000000180006a10     libucrt:log10.obj
 0001:00005a20       __real_1_over_5            0000000180006a20     libucrt:log10.obj
 0001:00005a30       __real_1_over_6            0000000180006a30     libucrt:log10.obj
 0001:00005a40       __real_neg_1023            0000000180006a40     libucrt:log10.obj
 0001:00005a50       __mask_2045                0000000180006a50     libucrt:log10.obj
 0001:00005a60       __real_threshold           0000000180006a60     libucrt:log10.obj
 0001:00005a70       __real_near_one_lt         0000000180006a70     libucrt:log10.obj
 0001:00005a80       __real_near_one_gt         0000000180006a80     libucrt:log10.obj
 0001:00005a90       __real_min_norm            0000000180006a90     libucrt:log10.obj
 0001:00005aa0       __real_notsign             0000000180006aa0     libucrt:log10.obj
 0001:00005ab0       __real_ca1                 0000000180006ab0     libucrt:log10.obj
 0001:00005ac0       __real_ca2                 0000000180006ac0     libucrt:log10.obj
 0001:00005ad0       __real_ca3                 0000000180006ad0     libucrt:log10.obj
 0001:00005ae0       __real_ca4                 0000000180006ae0     libucrt:log10.obj
 0001:00005af0       __mask_lower               0000000180006af0     libucrt:log10.obj
 0001:00005b00       __flag_x_zero              0000000180006b00     libucrt:log10.obj
 0001:00005b04       __flag_x_neg               0000000180006b04     libucrt:log10.obj
 0001:00005b08       __flag_x_nan               0000000180006b08     libucrt:log10.obj
 0001:00007360       __real@433fffffffffffff    0000000180008360     libucrt:fpsr.obj
 0001:00007368       __real@c33fffffffffffff    0000000180008368     libucrt:fpsr.obj
 0001:00007370       GS_ExceptionPointers       0000000180008370     LIBCMT:gs_report.obj
 0001:00007970       $$000000                   0000000180008970     chkstk.obj
 0001:00007e8c       $LN39                      0000000180008e8c     Brackets.obj
 0001:00009070       $LN301                     000000018000a070     Brackets.obj
 0001:000090a0       $LN300                     000000018000a0a0     Brackets.obj
 0001:000090d0       $LN299                     000000018000a0d0     Brackets.obj
 0001:00009100       $LN298                     000000018000a100     Brackets.obj
 0001:00009130       $LN297                     000000018000a130     Brackets.obj
 0001:00009844       $LN36                      000000018000a844     Brackets.obj
 0001:0000aa28       ?dllmain_crt_dispatch@@YAHQEAUHINSTANCE__@@KQEAX@Z 000000018000ba28 f   LIBCMT:dll_dllmain.obj
 0001:0000aa78       ?dllmain_crt_process_attach@@YAHQEAUHINSTANCE__@@QEAX@Z 000000018000ba78 f   LIBCMT:dll_dllmain.obj
 0001:0000ab90       ?dllmain_crt_process_detach@@YAH_N@Z 000000018000bb90 f   LIBCMT:dll_dllmain.obj
 0001:0000ac14       ?dllmain_dispatch@@YAHQEAUHINSTANCE__@@KQEAX@Z 000000018000bc14 f   LIBCMT:dll_dllmain.obj
 0001:0000b780       $$000000                   000000018000c780     libvcruntime:memset.obj
 0001:0000b87c       MsetTab                    000000018000c87c     libvcruntime:memset.obj
 0001:0000bd80       $$000000                   000000018000cd80     libvcruntime:_jmpuwind_.obj
 0001:0000c048       ?try_get_function@@YAPEAXW4function_id@?A0x89697e75@@QEBDQEBW4module_id@2@2@Z 000000018000d048 f   libvcruntime:winapi_downlevel.obj
 0001:0000c430       $$000000                   000000018000d430     libvcruntime:memcpy.obj
 0001:0000c4d7       MoveSmall                  000000018000d4d7     libvcruntime:memcpy.obj
 0001:0000c890       $$000000                   000000018000d890     libvcruntime:handlers.obj
 0001:0000cc24       ??$?RV<lambda_d80eeec6fff315bfe5c115232f3240e3>@@AEAV<lambda_6e4b09c48022b2350581041d5f6b0c4c>@@V<lambda_2358e3775559c9db80273638284d5e45>@@@?$__crt_seh_guarded_call@X@@QEAAX$$QEAV<lambda_d80eeec6fff315bfe5c115232f3240e3>@@AEAV<lambda_6e4b09c48022b2350581041d5f6b0c4c>@@$$QEAV<lambda_2358e3775559c9db80273638284d5e45>@@@Z 000000018000dc24 f   libucrt:exit.obj
 0001:0000cc5c       ??R<lambda_6e4b09c48022b2350581041d5f6b0c4c>@@QEBA@XZ 000000018000dc5c f   libucrt:exit.obj
 0001:0000cd34       ?atexit_exception_filter@@YAHK@Z 000000018000dd34 f   libucrt:exit.obj
 0001:0000cd40       ?common_exit@@YAXHW4_crt_exit_cleanup_mode@@W4_crt_exit_return_mode@@@Z 000000018000dd40 f   libucrt:exit.obj
 0001:0000cdfc       ?exit_or_terminate_process@@YAXI@Z 000000018000ddfc f   libucrt:exit.obj
 0001:0000ce48       ?try_cor_exit_process@@YAXI@Z 000000018000de48 f   libucrt:exit.obj
 0001:0000ced0       ??$parse_command_line@D@@YAXPEADPEAPEAD0PEA_K2@Z 000000018000ded0 f   libucrt:argv_parsing.obj
 0001:0000d274       ??$common_initialize_environment_nolock@D@@YAHXZ 000000018000e274 f   libucrt:environment_initialization.obj
 0001:0000d2e0       ??$create_environment@D@@YAQEAPEADQEAD@Z 000000018000e2e0 f   libucrt:environment_initialization.obj
 0001:0000d3ec       ??$free_environment@D@@YAXQEAPEAD@Z 000000018000e3ec f   libucrt:environment_initialization.obj
 0001:0000d3ec       ??$free_environment@_W@@YAXQEAPEA_W@Z 000000018000e3ec f   libucrt:environment_initialization.obj
 0001:0000d430       ??$uninitialize_environment_internal@D@@YAXAEAPEAPEAD@Z 000000018000e430 f   libucrt:environment_initialization.obj
 0001:0000d44c       ??$uninitialize_environment_internal@_W@@YAXAEAPEAPEA_W@Z 000000018000e44c f   libucrt:environment_initialization.obj
 0001:0000d4a8       ??$?RV<lambda_7777bce6b2f8c936911f934f8298dc43>@@AEAV<lambda_f03950bc5685219e0bcd2087efbe011e>@@V<lambda_3883c3dff614d5e0c5f61bb1ac94921c>@@@?$__crt_seh_guarded_call@H@@QEAAH$$QEAV<lambda_7777bce6b2f8c936911f934f8298dc43>@@AEAV<lambda_f03950bc5685219e0bcd2087efbe011e>@@$$QEAV<lambda_3883c3dff614d5e0c5f61bb1ac94921c>@@@Z 000000018000e4a8 f   libucrt:onexit.obj
 0001:0000d4e4       ??R<lambda_f03950bc5685219e0bcd2087efbe011e>@@QEBAHXZ 000000018000e4e4 f   libucrt:onexit.obj
 0001:0000d6ac       initialize_global_variables 000000018000e6ac f   libucrt:initialization.obj
 0001:0000d6c0       initialize_c               000000018000e6c0 f   libucrt:initialization.obj
 0001:0000d6e4       initialize_global_state_isolation 000000018000e6e4 f   libucrt:initialization.obj
 0001:0000d6e4       uninitialize_global_state_isolation 000000018000e6e4 f   libucrt:initialization.obj
 0001:0000d6e4       initialize_environment     000000018000e6e4 f   libucrt:initialization.obj
 0001:0000d6e4       uninitialize_c             000000018000e6e4 f   libucrt:initialization.obj
 0001:0000d6e4       report_memory_leaks        000000018000e6e4 f   libucrt:initialization.obj
 0001:0000d6e8       uninitialize_environment   000000018000e6e8 f   libucrt:initialization.obj
 0001:0000d6f8       initialize_pointers        000000018000e6f8 f   libucrt:initialization.obj
 0001:0000d74c       uninitialize_vcruntime     000000018000e74c f   libucrt:initialization.obj
 0001:0000d754       uninitialize_allocated_memory 000000018000e754 f   libucrt:initialization.obj
 0001:0000d794       uninitialize_allocated_io_buffers 000000018000e794 f   libucrt:initialization.obj
 0001:0000d980       $$000000                   000000018000e980     libucrt:strncmp.obj
 0001:0000dbf4       ??$?RV<lambda_0ae27a3a962d80f24befdcbee591983d>@@AEAV<lambda_8d0ee55de4b1038c4002e0adecdf1839>@@V<lambda_dc504788e8f1664fe9b84e20bfb512f2>@@@?$__crt_seh_guarded_call@X@@QEAAX$$QEAV<lambda_0ae27a3a962d80f24befdcbee591983d>@@AEAV<lambda_8d0ee55de4b1038c4002e0adecdf1839>@@$$QEAV<lambda_dc504788e8f1664fe9b84e20bfb512f2>@@@Z 000000018000ebf4 f   libucrt:per_thread_data.obj
 0001:0000dc34       ??$?RV<lambda_2d41944a1d46af3157314b8a01080d33>@@AEAV<lambda_8f455de75cd7d7f24b4096f044d8b9e6>@@V<lambda_aa500f224e6afead328df44964fe2772>@@@?$__crt_seh_guarded_call@X@@QEAAX$$QEAV<lambda_2d41944a1d46af3157314b8a01080d33>@@AEAV<lambda_8f455de75cd7d7f24b4096f044d8b9e6>@@$$QEAV<lambda_aa500f224e6afead328df44964fe2772>@@@Z 000000018000ec34 f   libucrt:per_thread_data.obj
 0001:0000dc74       ??$?RV<lambda_aa87e3671a710a21b5dc78c0bdf72e11>@@AEAV<lambda_92619d2358a28f41a33ba319515a20b9>@@V<lambda_6992ecaafeb10aed2b74cb1fae11a551>@@@?$__crt_seh_guarded_call@X@@QEAAX$$QEAV<lambda_aa87e3671a710a21b5dc78c0bdf72e11>@@AEAV<lambda_92619d2358a28f41a33ba319515a20b9>@@$$QEAV<lambda_6992ecaafeb10aed2b74cb1fae11a551>@@@Z 000000018000ec74 f   libucrt:per_thread_data.obj
 0001:0000dcbc       ??$?RV<lambda_f2e299630e499de9f9a165e60fcd3db5>@@AEAV<lambda_2ae9d31cdba2644fcbeaf08da7c24588>@@V<lambda_40d01ff24d0e7b3814fdbdcee8eab3c7>@@@?$__crt_seh_guarded_call@X@@QEAAX$$QEAV<lambda_f2e299630e499de9f9a165e60fcd3db5>@@AEAV<lambda_2ae9d31cdba2644fcbeaf08da7c24588>@@$$QEAV<lambda_40d01ff24d0e7b3814fdbdcee8eab3c7>@@@Z 000000018000ecbc f   libucrt:per_thread_data.obj
 0001:0000dd1c       ?construct_ptd_array@@YAXQEAU__acrt_ptd@@@Z 000000018000ed1c f   libucrt:per_thread_data.obj
 0001:0000ddec       ?destroy_fls@@YAXPEAX@Z    000000018000edec f   libucrt:per_thread_data.obj
 0001:0000de0c       ?destroy_ptd_array@@YAXQEAU__acrt_ptd@@@Z 000000018000ee0c f   libucrt:per_thread_data.obj
 0001:0000df04       ?replace_current_thread_locale_nolock@@YAXQEAU__acrt_ptd@@QEAU__crt_locale_data@@@Z 000000018000ef04 f   libucrt:per_thread_data.obj
 0001:0000e65c       ?<lambda_invoker_cdecl>@<lambda_c2303d2482d7c3675ea2e24c4cfb6115>@@CAHPEBX0@Z 000000018000f65c f   libucrt:argv_wildcards.obj
 0001:0000e670       ??$common_expand_argv_wildcards@D@@YAHQEAPEADQEAPEAPEAD@Z 000000018000f670 f   libucrt:argv_wildcards.obj
 0001:0000e87c       ??$copy_and_add_argument_to_buffer@D@@YAHQEBD0_KAEAV?$argument_list@D@?A0x5f5c8891@@@Z 000000018000f87c f   libucrt:argv_wildcards.obj
 0001:0000ea14       ??$expand_argument_wildcards@D@@YAHQEAD0AEAV?$argument_list@D@?A0x5f5c8891@@@Z 000000018000fa14 f   libucrt:argv_wildcards.obj
 0001:0000ebc8       ??$?RV<lambda_efdfa57d1f175319df784efa44bb7b81>@@AEAV<lambda_5f0a4c1567f8adc6734073e5d1e1b35c>@@V<lambda_2e8a7d3640ea6ccb4c2413664c2db6fd>@@@?$__crt_seh_guarded_call@X@@QEAAX$$QEAV<lambda_efdfa57d1f175319df784efa44bb7b81>@@AEAV<lambda_5f0a4c1567f8adc6734073e5d1e1b35c>@@$$QEAV<lambda_2e8a7d3640ea6ccb4c2413664c2db6fd>@@@Z 000000018000fbc8 f   libucrt:mbctype.obj
 0001:0000ed9c       ?getSystemCP@@YAHH@Z       000000018000fd9c f   libucrt:mbctype.obj
 0001:0000ee1c       ?setSBCS@@YAXPEAU__crt_multibyte_data@@@Z 000000018000fe1c f   libucrt:mbctype.obj
 0001:0000eeac       ?setSBUpLow@@YAXPEAU__crt_multibyte_data@@@Z 000000018000feac f   libucrt:mbctype.obj
 0001:0000f08c       ?setmbcp_internal@@YAHH_NQEAU__acrt_ptd@@QEAPEAU__crt_multibyte_data@@@Z 000000018001008c f   libucrt:mbctype.obj
 0001:0000f250       ?update_thread_multibyte_data_internal@@YAPEAU__crt_multibyte_data@@QEAU__acrt_ptd@@QEAPEAU1@@Z 0000000180010250 f   libucrt:mbctype.obj
 0001:0000f644       ?x_ismbbtype_l@@YAHPEAU__crt_locale_pointers@@IHH@Z 0000000180010644 f   libucrt:ismbbyte.obj
 0001:0000f89c       ?try_get_function@@YAPEAXW4function_id@?A0x391cf84c@@QEBDQEBW4module_id@2@2@Z 000000018001089c f   libucrt:winapi_thunks.obj
 0001:0000fe34       ?initialize_inherited_file_handles_nolock@@YAXXZ 0000000180010e34 f   libucrt:ioinit.obj
 0001:0000ff20       ?initialize_stdio_handles_nolock@@YAXXZ 0000000180010f20 f   libucrt:ioinit.obj
 0001:00010154       ??$?RV<lambda_450d765d439847d4c735a33c368b5fc0>@@AEAV<lambda_44731a7d0e6d81c3e6aa82d741081786>@@V<lambda_601a2a7da3b7a96e9554ac7215c4b07c>@@@?$__crt_seh_guarded_call@P6AXH@Z@@QEAAP6AXH@Z$$QEAV<lambda_450d765d439847d4c735a33c368b5fc0>@@AEAV<lambda_44731a7d0e6d81c3e6aa82d741081786>@@$$QEAV<lambda_601a2a7da3b7a96e9554ac7215c4b07c>@@@Z 0000000180011154 f   libucrt:signal.obj
 0001:000104b8       ??$?RV<lambda_842d9ff0dc9ef11c61343bbaebe7f885>@@AEAV<lambda_c5860995281e5c4ce005b3de8f5874ee>@@V<lambda_d90129c13df834fdcbf8d2b88dafcf2d>@@@?$__crt_seh_guarded_call@X@@QEAAX$$QEAV<lambda_842d9ff0dc9ef11c61343bbaebe7f885>@@AEAV<lambda_c5860995281e5c4ce005b3de8f5874ee>@@$$QEAV<lambda_d90129c13df834fdcbf8d2b88dafcf2d>@@@Z 00000001800114b8 f   libucrt:fflush.obj
 0001:00010554       ??$?RV<lambda_886d6c58226a84441f68b9f2b8217b83>@@AEAV<lambda_ab61a845afdef5b7c387490eaf3616ee>@@V<lambda_f7f22ab5edc0698d5f6905b0d3f44752>@@@?$__crt_seh_guarded_call@X@@QEAAX$$QEAV<lambda_886d6c58226a84441f68b9f2b8217b83>@@AEAV<lambda_ab61a845afdef5b7c387490eaf3616ee>@@$$QEAV<lambda_f7f22ab5edc0698d5f6905b0d3f44752>@@@Z 0000000180011554 f   libucrt:fflush.obj
 0001:0001063c       ?common_flush_all@@YAH_N@Z 000000018001163c f   libucrt:fflush.obj
 0001:00010ae0       ??$?RV<lambda_410d79af7f07d98d83a3f525b3859a53>@@AEAV<lambda_3e16ef9562a7dcce91392c22ab16ea36>@@V<lambda_38119f0e861e05405d8a144b9b982f0a>@@@?$__crt_seh_guarded_call@X@@QEAAX$$QEAV<lambda_410d79af7f07d98d83a3f525b3859a53>@@AEAV<lambda_3e16ef9562a7dcce91392c22ab16ea36>@@$$QEAV<lambda_38119f0e861e05405d8a144b9b982f0a>@@@Z 0000000180011ae0 f   libucrt:wsetlocale.obj
 0001:00011454       fallbackMethod             0000000180012454 f   libucrt:strpbrk.obj
 0001:00011824       $LN78                      0000000180012824     libucrt:strpbrk.obj
 0001:00011860       $LN77                      0000000180012860     libucrt:strpbrk.obj
 0001:000118a0       $LN76                      00000001800128a0     libucrt:strpbrk.obj
 0001:00011978       ?initialize_multibyte@@YAHXZ 0000000180012978 f   libucrt:multibyte_initializer.obj
 0001:00011b20       ?__acrt_LCMapStringA_stat@@YAHPEAU__crt_locale_pointers@@PEB_WKPEBDHPEADHHH@Z 0000000180012b20 f   libucrt:lcmapstringa.obj
 0001:00011f90       ?GetTableIndexFromLocaleName@@YAHPEB_W@Z 0000000180012f90 f   libucrt:lcidtoname_downlevel.obj
 0001:0001239c       ??$?RV<lambda_a37b2b86f63e897a80ea819b0eb08c01>@@AEAV<lambda_38ce7e780aa69e748d6df282ebc68efe>@@V<lambda_99fb1378e971ab6e7edea83e3a7a83a2>@@@?$__crt_seh_guarded_call@H@@QEAAH$$QEAV<lambda_a37b2b86f63e897a80ea819b0eb08c01>@@AEAV<lambda_38ce7e780aa69e748d6df282ebc68efe>@@$$QEAV<lambda_99fb1378e971ab6e7edea83e3a7a83a2>@@@Z 000000018001339c f   libucrt:commit.obj
 0001:000124bc       ?write_double_translated_ansi_nolock@@YA?AUwrite_result@?A0x17268360@@HQEBDI@Z 00000001800134bc f   libucrt:write.obj
 0001:000126e0       ?write_text_ansi_nolock@@YA?AUwrite_result@?A0x17268360@@HQEBDI@Z 00000001800136e0 f   libucrt:write.obj
 0001:000127e4       ?write_text_utf16le_nolock@@YA?AUwrite_result@?A0x17268360@@HQEBDI@Z 00000001800137e4 f   libucrt:write.obj
 0001:00012900       ?write_text_utf8_nolock@@YA?AUwrite_result@?A0x17268360@@HQEBDI@Z 0000000180013900 f   libucrt:write.obj
 0001:000131b8       ?free_crt_array_internal@@YAXQEAPEBX_K@Z 00000001800141b8 f   libucrt:inittime.obj
 0001:00013334       ??$common_lseek_nolock@_J@@YA_JH_JH@Z 0000000180014334 f   libucrt:lseek.obj
 0001:00013500       $$000000                   0000000180014500     libucrt:log10.obj
 0001:00013bdc       ??$?RV<lambda_751a882b2c74d4b022dec766aa51a29a>@@AEAV<lambda_628dfdc04ba53c8bfc02c9951375f3f5>@@V<lambda_f6c7be5f7998530c34de24c7437d6b54>@@@?$__crt_seh_guarded_call@H@@QEAAH$$QEAV<lambda_751a882b2c74d4b022dec766aa51a29a>@@AEAV<lambda_628dfdc04ba53c8bfc02c9951375f3f5>@@$$QEAV<lambda_f6c7be5f7998530c34de24c7437d6b54>@@@Z 0000000180014bdc f   libucrt:close.obj
 0001:00013dcc       _call_matherr              0000000180014dcc f   libucrt:libm_error.obj
 0001:00013e34       _exception_enabled         0000000180014e34 f   libucrt:libm_error.obj
 0001:000140b0       _log_special_common        00000001800150b0 f   libucrt:log_special.obj
 0001:00014150       $$000000                   0000000180015150     libucrt:fpsr.obj
 0001:00014740       $$000000                   0000000180015740     LIBCMT:_amdsecgs_.obj
 0001:0001492c       capture_current_context    000000018001592c f   LIBCMT:gs_report.obj
 0001:0001499c       capture_previous_context   000000018001599c f   LIBCMT:gs_report.obj
 0001:00014a10       $$000000                   0000000180015a10     libvcruntime:memcmp.obj
 0001:00014af0       $$000000                   0000000180015af0     LIBCMT:_guard_dispatch_.obj
 0001:00014b10       ?fin$0@?0??dllmain_crt_process_attach@@YAHQEAUHINSTANCE__@@QEAX@Z@4HA 0000000180015b10 f   LIBCMT:dll_dllmain.obj
 0001:00014b27       ?fin$0@?0??dllmain_crt_process_detach@@YAH_N@Z@4HA 0000000180015b27 f   LIBCMT:dll_dllmain.obj
 0001:00014b43       ?filt$0@?0??dllmain_dispatch@@YAHQEAUHINSTANCE__@@KQEAX@Z@4HA 0000000180015b43 f   LIBCMT:dll_dllmain.obj
 0001:00014b79       __scrt_is_nonwritable_in_current_image$filt$0 0000000180015b79 f   LIBCMT:utility.obj
 0001:00014b91       __DestructExceptionObject$filt$0 0000000180015b91 f   libvcruntime:ehhelpers.obj
 0001:00014ba9       _query_new_handler$fin$0   0000000180015ba9 f   libucrt:new_handler.obj
 0001:00014bbf       ?fin$0@?0???$?RV<lambda_450d765d439847d4c735a33c368b5fc0>@@AEAV<lambda_44731a7d0e6d81c3e6aa82d741081786>@@V<lambda_601a2a7da3b7a96e9554ac7215c4b07c>@@@?$__crt_seh_guarded_call@P6AXH@Z@@QEAAP6AXH@Z$$QEAV<lambda_450d765d439847d4c735a33c368b5fc0>@@AEAV<lambda_44731a7d0e6d81c3e6aa82d741081786>@@$$QEAV<lambda_601a2a7da3b7a96e9554ac7215c4b07c>@@@Z@4HA 0000000180015bbf f   libucrt:signal.obj
 0001:00014bbf       ?fin$0@?0???$?RV<lambda_0ae27a3a962d80f24befdcbee591983d>@@AEAV<lambda_8d0ee55de4b1038c4002e0adecdf1839>@@V<lambda_dc504788e8f1664fe9b84e20bfb512f2>@@@?$__crt_seh_guarded_call@X@@QEAAX$$QEAV<lambda_0ae27a3a962d80f24befdcbee591983d>@@AEAV<lambda_8d0ee55de4b1038c4002e0adecdf1839>@@$$QEAV<lambda_dc504788e8f1664fe9b84e20bfb512f2>@@@Z@4HA 0000000180015bbf f   libucrt:per_thread_data.obj
 0001:00014bbf       ?fin$0@?0???$?RV<lambda_2d41944a1d46af3157314b8a01080d33>@@AEAV<lambda_8f455de75cd7d7f24b4096f044d8b9e6>@@V<lambda_aa500f224e6afead328df44964fe2772>@@@?$__crt_seh_guarded_call@X@@QEAAX$$QEAV<lambda_2d41944a1d46af3157314b8a01080d33>@@AEAV<lambda_8f455de75cd7d7f24b4096f044d8b9e6>@@$$QEAV<lambda_aa500f224e6afead328df44964fe2772>@@@Z@4HA 0000000180015bbf f   libucrt:per_thread_data.obj
 0001:00014bbf       ?fin$0@?0???$?RV<lambda_aa87e3671a710a21b5dc78c0bdf72e11>@@AEAV<lambda_92619d2358a28f41a33ba319515a20b9>@@V<lambda_6992ecaafeb10aed2b74cb1fae11a551>@@@?$__crt_seh_guarded_call@X@@QEAAX$$QEAV<lambda_aa87e3671a710a21b5dc78c0bdf72e11>@@AEAV<lambda_92619d2358a28f41a33ba319515a20b9>@@$$QEAV<lambda_6992ecaafeb10aed2b74cb1fae11a551>@@@Z@4HA 0000000180015bbf f   libucrt:per_thread_data.obj
 0001:00014bbf       ?fin$0@?0???$?RV<lambda_f2e299630e499de9f9a165e60fcd3db5>@@AEAV<lambda_2ae9d31cdba2644fcbeaf08da7c24588>@@V<lambda_40d01ff24d0e7b3814fdbdcee8eab3c7>@@@?$__crt_seh_guarded_call@X@@QEAAX$$QEAV<lambda_f2e299630e499de9f9a165e60fcd3db5>@@AEAV<lambda_2ae9d31cdba2644fcbeaf08da7c24588>@@$$QEAV<lambda_40d01ff24d0e7b3814fdbdcee8eab3c7>@@@Z@4HA 0000000180015bbf f   libucrt:per_thread_data.obj
 0001:00014bbf       ?fin$0@?0???$?RV<lambda_efdfa57d1f175319df784efa44bb7b81>@@AEAV<lambda_5f0a4c1567f8adc6734073e5d1e1b35c>@@V<lambda_2e8a7d3640ea6ccb4c2413664c2db6fd>@@@?$__crt_seh_guarded_call@X@@QEAAX$$QEAV<lambda_efdfa57d1f175319df784efa44bb7b81>@@AEAV<lambda_5f0a4c1567f8adc6734073e5d1e1b35c>@@$$QEAV<lambda_2e8a7d3640ea6ccb4c2413664c2db6fd>@@@Z@4HA 0000000180015bbf f   libucrt:mbctype.obj
 0001:00014bbf       ?fin$0@?0???$?RV<lambda_7777bce6b2f8c936911f934f8298dc43>@@AEAV<lambda_f03950bc5685219e0bcd2087efbe011e>@@V<lambda_3883c3dff614d5e0c5f61bb1ac94921c>@@@?$__crt_seh_guarded_call@H@@QEAAH$$QEAV<lambda_7777bce6b2f8c936911f934f8298dc43>@@AEAV<lambda_f03950bc5685219e0bcd2087efbe011e>@@$$QEAV<lambda_3883c3dff614d5e0c5f61bb1ac94921c>@@@Z@4HA 0000000180015bbf f   libucrt:onexit.obj
 0001:00014bbf       ?fin$0@?0???$?RV<lambda_d80eeec6fff315bfe5c115232f3240e3>@@AEAV<lambda_6e4b09c48022b2350581041d5f6b0c4c>@@V<lambda_2358e3775559c9db80273638284d5e45>@@@?$__crt_seh_guarded_call@X@@QEAAX$$QEAV<lambda_d80eeec6fff315bfe5c115232f3240e3>@@AEAV<lambda_6e4b09c48022b2350581041d5f6b0c4c>@@$$QEAV<lambda_2358e3775559c9db80273638284d5e45>@@@Z@4HA 0000000180015bbf f   libucrt:exit.obj
 0001:00014bd9       ?filt$0@?0???R<lambda_6e4b09c48022b2350581041d5f6b0c4c>@@QEBA@XZ@4HA 0000000180015bd9 f   libucrt:exit.obj
 0001:00014bf4       ?fin$0@?0??update_thread_multibyte_data_internal@@YAPEAU__crt_multibyte_data@@QEAU__acrt_ptd@@QEAPEAU1@@Z@4HA 0000000180015bf4 f   libucrt:mbctype.obj
 0001:00014c0d       __acrt_lowio_ensure_fh_exists$fin$0 0000000180015c0d f   libucrt:osfinfo.obj
 0001:00014c0d       __acrt_initialize_lowio$fin$0 0000000180015c0d f   libucrt:ioinit.obj
 0001:00014c26       raise$fin$0                0000000180015c26 f   libucrt:signal.obj
 0001:00014c47       ?fin$0@?0???$?RV<lambda_842d9ff0dc9ef11c61343bbaebe7f885>@@AEAV<lambda_c5860995281e5c4ce005b3de8f5874ee>@@V<lambda_d90129c13df834fdcbf8d2b88dafcf2d>@@@?$__crt_seh_guarded_call@X@@QEAAX$$QEAV<lambda_842d9ff0dc9ef11c61343bbaebe7f885>@@AEAV<lambda_c5860995281e5c4ce005b3de8f5874ee>@@$$QEAV<lambda_d90129c13df834fdcbf8d2b88dafcf2d>@@@Z@4HA 0000000180015c47 f   libucrt:fflush.obj
 0001:00014c62       ?fin$0@?0???$?RV<lambda_886d6c58226a84441f68b9f2b8217b83>@@AEAV<lambda_ab61a845afdef5b7c387490eaf3616ee>@@V<lambda_f7f22ab5edc0698d5f6905b0d3f44752>@@@?$__crt_seh_guarded_call@X@@QEAAX$$QEAV<lambda_886d6c58226a84441f68b9f2b8217b83>@@AEAV<lambda_ab61a845afdef5b7c387490eaf3616ee>@@$$QEAV<lambda_f7f22ab5edc0698d5f6905b0d3f44752>@@@Z@4HA 0000000180015c62 f   libucrt:fflush.obj
 0001:00014c7f       ?fin$0@?0???$?RV<lambda_410d79af7f07d98d83a3f525b3859a53>@@AEAV<lambda_3e16ef9562a7dcce91392c22ab16ea36>@@V<lambda_38119f0e861e05405d8a144b9b982f0a>@@@?$__crt_seh_guarded_call@X@@QEAAX$$QEAV<lambda_410d79af7f07d98d83a3f525b3859a53>@@AEAV<lambda_3e16ef9562a7dcce91392c22ab16ea36>@@$$QEAV<lambda_38119f0e861e05405d8a144b9b982f0a>@@@Z@4HA 0000000180015c7f f   libucrt:wsetlocale.obj
 0001:00014c99       __acrt_update_thread_locale_data$fin$0 0000000180015c99 f   libucrt:locale_refcounting.obj
 0001:00014cb2       ?fin$0@?0???$?RV<lambda_a37b2b86f63e897a80ea819b0eb08c01>@@AEAV<lambda_38ce7e780aa69e748d6df282ebc68efe>@@V<lambda_99fb1378e971ab6e7edea83e3a7a83a2>@@@?$__crt_seh_guarded_call@H@@QEAAH$$QEAV<lambda_a37b2b86f63e897a80ea819b0eb08c01>@@AEAV<lambda_38ce7e780aa69e748d6df282ebc68efe>@@$$QEAV<lambda_99fb1378e971ab6e7edea83e3a7a83a2>@@@Z@4HA 0000000180015cb2 f   libucrt:commit.obj
 0001:00014cb2       ?fin$0@?0???$?RV<lambda_751a882b2c74d4b022dec766aa51a29a>@@AEAV<lambda_628dfdc04ba53c8bfc02c9951375f3f5>@@V<lambda_f6c7be5f7998530c34de24c7437d6b54>@@@?$__crt_seh_guarded_call@H@@QEAAH$$QEAV<lambda_751a882b2c74d4b022dec766aa51a29a>@@AEAV<lambda_628dfdc04ba53c8bfc02c9951375f3f5>@@$$QEAV<lambda_f6c7be5f7998530c34de24c7437d6b54>@@@Z@4HA 0000000180015cb2 f   libucrt:close.obj
 0001:00014ccc       _write$fin$0               0000000180015ccc f   libucrt:write.obj
 0001:00014ce3       _fcloseall$fin$0           0000000180015ce3 f   libucrt:closeall.obj
 0001:00014cfc       fclose$fin$0               0000000180015cfc f   libucrt:fclose.obj
 0001:00014d14       _ctrlfp$filt$0             0000000180015d14 f   libucrt:fpctrl.obj
 0001:00014d40       _IsNonwritableInCurrentImage$filt$0 0000000180015d40 f   LIBCMT:pesect.obj
 0001:00014d60       $xdatasym                  0000000180015d60     chkstk.obj
 0001:00014d68       $unwind$abort              0000000180015d68     libucrt:abort.obj
 0001:00014d68       $unwind$_isatty            0000000180015d68     libucrt:isatty.obj
 0001:00014d68       $unwind$uninitialize_allocated_io_buffers 0000000180015d68     libucrt:initialization.obj
 0001:00014d68       $unwind$uninitialize_environment 0000000180015d68     libucrt:initialization.obj
 0001:00014d68       $unwind$initialize_c       0000000180015d68     libucrt:initialization.obj
 0001:00014d68       $unwind$__acrt_thread_detach 0000000180015d68     libucrt:initialization.obj
 0001:00014d68       $unwind$__acrt_update_thread_multibyte_data 0000000180015d68     libucrt:mbctype.obj
 0001:00014d68       $unwind$__acrt_initialize_multibyte 0000000180015d68     libucrt:mbctype.obj
 0001:00014d68       $unwind$__acrt_thread_attach 0000000180015d68     libucrt:initialization.obj
 0001:00014d68       $unwind$__acrt_initialize_command_line 0000000180015d68     libucrt:argv_data.obj
 0001:00014d68       $unwind$__acrt_uninitialize_critical 0000000180015d68     libucrt:initialization.obj
 0001:00014d68       $unwind$_get_osfhandle     0000000180015d68     libucrt:osfinfo.obj
 0001:00014d68       $unwind$__acrt_uninitialize 0000000180015d68     libucrt:initialization.obj
 0001:00014d68       $unwind$__acrt_initialize_ptd 0000000180015d68     libucrt:per_thread_data.obj
 0001:00014d68       $unwind$??$uninitialize_environment_internal@_W@@YAXAEAPEAPEA_W@Z 0000000180015d68     libucrt:environment_initialization.obj
 0001:00014d68       $unwind$??$uninitialize_environment_internal@D@@YAXAEAPEAPEAD@Z 0000000180015d68     libucrt:environment_initialization.obj
 0001:00014d68       $unwind$__acrt_DownlevelLocaleNameToLCID 0000000180015d68     libucrt:lcidtoname_downlevel.obj
 0001:00014d68       $unwind$__dcrt_uninitialize_environments_nolock 0000000180015d68     libucrt:environment_initialization.obj
 0001:00014d68       $unwind$__dcrt_terminate_console_output 0000000180015d68     libucrt:initcon.obj
 0001:00014d68       $unwind$__acrt_uninitialize_ptd 0000000180015d68     libucrt:per_thread_data.obj
 0001:00014d68       $unwind$_set_errno_from_matherr 0000000180015d68     libucrt:fpexcept.obj
 0001:00014d68       $unwind$_invoke_watson     0000000180015d68     libucrt:invalid_parameter.obj
 0001:00014d68       $unwind$__vcrt_uninitialize_ptd 0000000180015d68     libvcruntime:per_thread_data.obj
 0001:00014d68       $unwind$_msize_base        0000000180015d68     libucrt:msize.obj
 0001:00014d68       $unwind$_errno             0000000180015d68     libucrt:errno.obj
 0001:00014d68       $unwind$__vcrt_initialize_ptd 0000000180015d68     libvcruntime:per_thread_data.obj
 0001:00014d68       $unwind$__vcrt_thread_detach 0000000180015d68     libvcruntime:initialization.obj
 0001:00014d68       $unwind$__acrt_initialize_heap 0000000180015d68     libucrt:heap_handle.obj
 0001:00014d68       $unwind$_statfp            0000000180015d68     libucrt:fpctrl.obj
 0001:00014d68       $unwind$__vcrt_thread_attach 0000000180015d68     libvcruntime:initialization.obj
 0001:00014d68       $unwind$__vcrt_uninitialize_critical 0000000180015d68     libvcruntime:initialization.obj
 0001:00014d68       $unwind$__vcrt_uninitialize 0000000180015d68     libvcruntime:initialization.obj
 0001:00014d68       $unwind$?initialize_multibyte@@YAHXZ 0000000180015d68     libucrt:multibyte_initializer.obj
 0001:00014d68       $unwind$__doserrno         0000000180015d68     libucrt:errno.obj
 0001:00014d68       $unwind$__vcrt_initialize  0000000180015d68     libvcruntime:initialization.obj
 0001:00014d68       $unwind$__scrt_dllmain_crt_thread_detach 0000000180015d68     LIBCMT:utility.obj
 0001:00014d68       $unwind$__GSHandlerCheck   0000000180015d68     LIBCMT:_gshandler_.obj
 0001:00014d68       $unwind$__scrt_dllmain_crt_thread_attach 0000000180015d68     LIBCMT:utility.obj
 0001:00014d68       $unwind$__scrt_dllmain_uninitialize_critical 0000000180015d68     LIBCMT:utility.obj
 0001:00014d68       $unwind$__scrt_dllmain_uninitialize_c 0000000180015d68     LIBCMT:utility.obj
 0001:00014d68       $unwind$__scrt_dllmain_after_initialize_c 0000000180015d68     LIBCMT:utility.obj
 0001:00014d68       $unwind$__scrt_dllmain_before_initialize_c 0000000180015d68     LIBCMT:utility.obj
 0001:00014d68       $unwind$__scrt_acquire_startup_lock 0000000180015d68     LIBCMT:utility.obj
 0001:00014d68       $unwind$__report_rangecheckfailure 0000000180015d68     LIBCMT:gs_report.obj
 0001:00014d68       $unwind$__scrt_initialize_default_local_stdio_options 0000000180015d68     LIBCMT:default_local_stdio_options.obj
 0001:00014d68       $unwind$?dllmain_crt_dispatch@@YAHQEAUHINSTANCE__@@KQEAX@Z 0000000180015d68     LIBCMT:dll_dllmain.obj
 0001:00014d68       $unwind$_fileno            0000000180015d68     libucrt:fileno.obj
 0001:00014d68       $unwind$GetGlobalInfoW     0000000180015d68     Brackets.obj
 0001:00014d68       $unwind$ConfigureW         0000000180015d68     Brackets.obj
 0001:00014d68       $unwind$__pctype_func      0000000180015d68     libucrt:ctype.obj
 0001:00014d68       $unwind$__vcrt_freefls     0000000180015d68     libvcruntime:per_thread_data.obj
 0001:00014d68       $unwind$__acrt_release_locale_ref 0000000180015d68     libucrt:locale_refcounting.obj
 0001:00014d70       $unwind$__acrt_stdio_free_buffer_nolock 0000000180015d70     libucrt:_freebuf.obj
 0001:00014d70       $unwind$_clrfp             0000000180015d70     libucrt:fpctrl.obj
 0001:00014d70       $unwind$_set_statfp        0000000180015d70     libucrt:fpctrl.obj
 0001:00014d70       $unwind$__acrt_freeptd     0000000180015d70     libucrt:per_thread_data.obj
 0001:00014d70       $unwind$__vcrt_freeptd     0000000180015d70     libvcruntime:per_thread_data.obj
 0001:00014d70       $unwind$__acrt_getptd_head 0000000180015d70     libucrt:per_thread_data.obj
 0001:00014d70       $unwind$__vcrt_initialize_locks 0000000180015d70     libvcruntime:locks.obj
 0001:00014d70       $unwind$??_Gtype_info@@UEAAPEAXI@Z 0000000180015d70     LIBCMT:std_type_info_static.obj
 0001:00014d70       $unwind$?try_cor_exit_process@@YAXI@Z 0000000180015d70     libucrt:exit.obj
 0001:00014d70       $unwind$__acrt_get_process_end_policy 0000000180015d70     libucrt:win_policies.obj
 0001:00014d70       $unwind$?exit_or_terminate_process@@YAXI@Z 0000000180015d70     libucrt:exit.obj
 0001:00014d70       $unwind$??_G?$DialogItemBinding@UFarDialogItem@@@@UEAAPEAXI@Z 0000000180015d70     Brackets.obj
 0001:00014d70       $unwind$??0bad_array_new_length@std@@QEAA@AEBV01@@Z 0000000180015d70     LIBCMT:throw_bad_alloc.obj
 0001:00014d70       $unwind$?SaveValue@PluginCheckBoxBinding@@UEAAXPEAUFarDialogItem@@H@Z 0000000180015d70     Brackets.obj
 0001:00014d70       $unwind$__vcrt_uninitialize_locks 0000000180015d70     libvcruntime:locks.obj
 0001:00014d70       $unwind$__acrt_allocate_buffer_for_argv 0000000180015d70     libucrt:argv_parsing.obj
 0001:00014d70       $unwind$_callnewh          0000000180015d70     libucrt:new_handler.obj
 0001:00014d70       $unwind$__scrt_uninitialize_crt 0000000180015d70     LIBCMT:utility.obj
 0001:00014d70       $unwind$??_GPluginRadioButtonBinding@@UEAAPEAXI@Z 0000000180015d70     Brackets.obj
 0001:00014d70       $unwind$??0bad_alloc@std@@QEAA@AEBV01@@Z 0000000180015d70     LIBCMT:throw_bad_alloc.obj
 0001:00014d70       $unwind$__acrt_AppPolicyGetProcessTerminationMethodInternal 0000000180015d70     libucrt:winapi_thunks.obj
 0001:00014d70       $unwind$??0exception@std@@QEAA@AEBV01@@Z 0000000180015d70     LIBCMT:throw_bad_alloc.obj
 0001:00014d70       $unwind$?SaveValue@PluginEditFieldBinding@@UEAAXPEAUFarDialogItem@@H@Z 0000000180015d70     Brackets.obj
 0001:00014d70       $unwind$??_GPluginCheckBoxBinding@@UEAAPEAXI@Z 0000000180015d70     Brackets.obj
 0001:00014d70       $unwind$??_GPluginEditFieldBinding@@UEAAPEAXI@Z 0000000180015d70     Brackets.obj
 0001:00014d70       $unwind$_malloc_base       0000000180015d70     libucrt:malloc_base.obj
 0001:00014d70       $unwind$??2@YAPEAX_K@Z     0000000180015d70     LIBCMT:new_scalar.obj
 0001:00014d70       $unwind$__acrt_update_multibyte_info 0000000180015d70     libucrt:locale_update.obj
 0001:00014d70       $unwind$__acrt_uninitialize_locks 0000000180015d70     libucrt:locks.obj
 0001:00014d70       $unwind$__acrt_update_locale_info 0000000180015d70     libucrt:locale_update.obj
 0001:00014d70       $unwind$__std_type_info_destroy_list 0000000180015d70     libvcruntime:std_type_info.obj
 0001:00014d70       $unwind$__acrt_initialize_locks 0000000180015d70     libucrt:locks.obj
 0001:00014d70       $unwind$__vcrt_FlsAlloc    0000000180015d70     libvcruntime:winapi_downlevel.obj
 0001:00014d70       $unwind$__acrt_uninitialize_stdio 0000000180015d70     libucrt:_file.obj
 0001:00014d70       $unwind$__raise_securityfailure 0000000180015d70     LIBCMT:gs_report.obj
 0001:00014d70       $unwind$?SaveValue@PluginIntEditFieldBinding@@UEAAXPEAUFarDialogItem@@H@Z 0000000180015d70     Brackets.obj
 0001:00014d70       $unwind$__scrt_initialize_crt 0000000180015d70     LIBCMT:utility.obj
 0001:00014d70       $unwind$__acrt_uninitialize_winapi_thunks 0000000180015d70     libucrt:winapi_thunks.obj
 0001:00014d70       $unwind$__vcrt_FlsFree     0000000180015d70     libvcruntime:winapi_downlevel.obj
 0001:00014d70       $unwind$__scrt_release_startup_lock 0000000180015d70     LIBCMT:utility.obj
 0001:00014d70       $unwind$__vcrt_FlsGetValue 0000000180015d70     libvcruntime:winapi_downlevel.obj
 0001:00014d70       $unwind$__acrt_FlsAlloc    0000000180015d70     libucrt:winapi_thunks.obj
 0001:00014d70       $unwind$??_GPluginUIntEditFieldBinding@@UEAAPEAXI@Z 0000000180015d70     Brackets.obj
 0001:00014d70       $unwind$_calloc_base       0000000180015d70     libucrt:calloc_base.obj
 0001:00014d70       $unwind$__acrt_FlsFree     0000000180015d70     libucrt:winapi_thunks.obj
 0001:00014d70       $unwind$?SaveValue@PluginUIntEditFieldBinding@@UEAAXPEAUFarDialogItem@@H@Z 0000000180015d70     Brackets.obj
 0001:00014d70       $unwind$strcpy_s           0000000180015d70     libucrt:strcpy_s.obj
 0001:00014d70       $unwind$__acrt_FlsGetValue 0000000180015d70     libucrt:winapi_thunks.obj
 0001:00014d70       $unwind$??_GPluginIntEditFieldBinding@@UEAAPEAXI@Z 0000000180015d70     Brackets.obj
 0001:00014d70       $unwind$_fflush_nolock     0000000180015d70     libucrt:fflush.obj
 0001:00014d70       $unwind$__std_exception_destroy 0000000180015d70     libvcruntime:std_exception.obj
 0001:00014d70       $unwind$initialize_pointers 0000000180015d70     libucrt:initialization.obj
 0001:00014d70       $unwind$uninitialize_allocated_memory 0000000180015d70     libucrt:initialization.obj
 0001:00014d70       $unwind$GetPluginInfoW     0000000180015d70     Brackets.obj
 0001:00014d78       $unwind$OpenW              0000000180015d78     Brackets.obj
 0001:00014d90       $unwind$SetStartupInfoW    0000000180015d90     Brackets.obj
 0001:00014da4       $unwind$?CreateRadioButtonBinding@PluginDialogBuilder@@MEAAPEAU?$DialogItemBinding@UFarDialogItem@@@@PEAH@Z 0000000180015da4     Brackets.obj
 0001:00014da4       $unwind$??0_LocaleUpdate@@QEAA@QEAU__crt_locale_pointers@@@Z 0000000180015da4     libucrt:output.obj
 0001:00014da4       $unwind$_realloc_base      0000000180015da4     libucrt:realloc_base.obj
 0001:00014da4       $unwind$_updatetlocinfoEx_nolock 0000000180015da4     libucrt:locale_refcounting.obj
 0001:00014da4       $unwind$__acrt_errno_map_os_error 0000000180015da4     libucrt:errno.obj
 0001:00014da4       $unwind$?SaveValue@PluginRadioButtonBinding@@UEAAXPEAUFarDialogItem@@H@Z 0000000180015da4     Brackets.obj
 0001:00014da4       $unwind$?replace_current_thread_locale_nolock@@YAXQEAU__acrt_ptd@@QEAU__crt_locale_data@@@Z 0000000180015da4     libucrt:per_thread_data.obj
 0001:00014da4       $unwind$_fclose_nolock     0000000180015da4     libucrt:fclose.obj
 0001:00014da4       $unwind$??_GPluginDialogBuilder@@UEAAPEAXI@Z 0000000180015da4     Brackets.obj
 0001:00014da4       $unwind$_RTC_Initialize    0000000180015da4     LIBCMT:_initsect_.obj
 0001:00014da4       $unwind$__vcrt_FlsSetValue 0000000180015da4     libvcruntime:winapi_downlevel.obj
 0001:00014da4       $unwind$__acrt_FlsSetValue 0000000180015da4     libucrt:winapi_thunks.obj
 0001:00014da4       $unwind$__acrt_LocaleNameToLCID 0000000180015da4     libucrt:winapi_thunks.obj
 0001:00014da4       $unwind$__acrt_getptd_noexit 0000000180015da4     libucrt:per_thread_data.obj
 0001:00014da4       $unwind$??_G?$DialogBuilderBase@UFarDialogItem@@@@MEAAPEAXI@Z 0000000180015da4     Brackets.obj
 0001:00014da4       $unwind$__acrt_getptd      0000000180015da4     libucrt:per_thread_data.obj
 0001:00014da4       $unwind$??$common_initialize_environment_nolock@D@@YAHXZ 0000000180015da4     libucrt:environment_initialization.obj
 0001:00014da4       $unwind$_RTC_Terminate     0000000180015da4     LIBCMT:_initsect_.obj
 0001:00014da4       $unwind$__acrt_execute_uninitializers 0000000180015da4     libucrt:shared_initialization.obj
 0001:00014da4       $unwind$??_Gexception@std@@UEAAPEAXI@Z 0000000180015da4     LIBCMT:throw_bad_alloc.obj
 0001:00014da4       $unwind$??_Gbad_array_new_length@std@@UEAAPEAXI@Z 0000000180015da4     LIBCMT:throw_bad_alloc.obj
 0001:00014da4       $unwind$_close_nolock      0000000180015da4     libucrt:close.obj
 0001:00014da4       $unwind$__acrt_uninitialize_lowio 0000000180015da4     libucrt:ioinit.obj
 0001:00014da4       $unwind$??_Gbad_alloc@std@@UEAAPEAXI@Z 0000000180015da4     LIBCMT:throw_bad_alloc.obj
 0001:00014da4       $unwind$?InitDialogItem@PluginDialogBuilder@@MEAAXPEAUFarDialogItem@@PEB_W@Z 0000000180015da4     Brackets.obj
 0001:00014da4       $unwind$_initterm_e        0000000180015da4     libucrt:initterm.obj
 0001:00014da4       $unwind$strncpy_s          0000000180015da4     libucrt:strncpy_s.obj
 0001:00014db0       $unwind$?AddDialogItem@?$DialogBuilderBase@UFarDialogItem@@@@IEAAPEAUFarDialogItem@@W4FARDIALOGITEMTYPES@@PEB_W@Z 0000000180015db0     Brackets.obj
 0001:00014db0       $unwind$?AddIntEditField@PluginDialogBuilder@@UEAAPEAUFarDialogItem@@PEAHH@Z 0000000180015db0     Brackets.obj
 0001:00014db0       $unwind$?AddUIntEditField@PluginDialogBuilder@@UEAAPEAUFarDialogItem@@PEAIH@Z 0000000180015db0     Brackets.obj
 0001:00014dc8       $unwind$?UpdateBorderSize@?$DialogBuilderBase@UFarDialogItem@@@@IEAAXXZ 0000000180015dc8     Brackets.obj
 0001:00014dd8       $chain$1$?UpdateBorderSize@?$DialogBuilderBase@UFarDialogItem@@@@IEAAXXZ 0000000180015dd8     Brackets.obj
 0001:00014df0       $chain$2$?UpdateBorderSize@?$DialogBuilderBase@UFarDialogItem@@@@IEAAXXZ 0000000180015df0     Brackets.obj
 0001:00014e04       $chain$3$?UpdateBorderSize@?$DialogBuilderBase@UFarDialogItem@@@@IEAAXXZ 0000000180015e04     Brackets.obj
 0001:00014e14       $chain$4$?UpdateBorderSize@?$DialogBuilderBase@UFarDialogItem@@@@IEAAXXZ 0000000180015e14     Brackets.obj
 0001:00014e24       $unwind$??1?$DialogBuilderBase@UFarDialogItem@@@@MEAA@XZ 0000000180015e24     Brackets.obj
 0001:00014e30       $chain$0$??1?$DialogBuilderBase@UFarDialogItem@@@@MEAA@XZ 0000000180015e30     Brackets.obj
 0001:00014e44       $chain$1$??1?$DialogBuilderBase@UFarDialogItem@@@@MEAA@XZ 0000000180015e44     Brackets.obj
 0001:00014e54       $unwind$?AddButtons@?$DialogBuilderBase@UFarDialogItem@@@@QEAAXHPEBHHH@Z 0000000180015e54     Brackets.obj
 0001:00014e60       $chain$4$?AddButtons@?$DialogBuilderBase@UFarDialogItem@@@@QEAAXHPEBHHH@Z 0000000180015e60     Brackets.obj
 0001:00014e84       $chain$5$?AddButtons@?$DialogBuilderBase@UFarDialogItem@@@@QEAAXHPEBHHH@Z 0000000180015e84     Brackets.obj
 0001:00014e94       $unwind$?DoShowDialog@PluginDialogBuilder@@MEAA_JXZ 0000000180015e94     Brackets.obj
 0001:00014ea0       $unwind$?free_crt_array_internal@@YAXQEAPEBX_K@Z 0000000180015ea0     libucrt:inittime.obj
 0001:00014ea0       $unwind$??$common_lseek_nolock@_J@@YA_JH_JH@Z 0000000180015ea0     libucrt:lseek.obj
 0001:00014ea0       $unwind$_exception_enabled 0000000180015ea0     libucrt:libm_error.obj
 0001:00014ea0       $unwind$__acrt_stdio_flush_nolock 0000000180015ea0     libucrt:fflush.obj
 0001:00014ea0       $unwind$__vcrt_InitializeCriticalSectionEx 0000000180015ea0     libvcruntime:winapi_downlevel.obj
 0001:00014ea0       $unwind$__vcrt_getptd_noexit 0000000180015ea0     libvcruntime:per_thread_data.obj
 0001:00014ea0       $unwind$?CreateCheckBoxBinding@PluginDialogBuilder@@MEAAPEAU?$DialogItemBinding@UFarDialogItem@@@@PEAHH@Z 0000000180015ea0     Brackets.obj
 0001:00014ea0       $unwind$__acrt_execute_initializers 0000000180015ea0     libucrt:shared_initialization.obj
 0001:00014ea0       $unwind$__acrt_InitializeCriticalSectionEx 0000000180015ea0     libucrt:winapi_thunks.obj
 0001:00014ea0       $unwind$_DllMainCRTStartup 0000000180015ea0     LIBCMT:dll_dllmain.obj
 0001:00014eb0       $unwind$?Config@@YAHXZ     0000000180015eb0     Brackets.obj
 0001:00014ed0       $unwind$?ShowMenu@@YAHH@Z  0000000180015ed0     Brackets.obj
 0001:00014ee4       $unwind$?dllmain_crt_process_attach@@YAHQEAUHINSTANCE__@@QEAX@Z 0000000180015ee4     LIBCMT:dll_dllmain.obj
 0001:00014f20       $unwind$__acrt_initialize_lowio$fin$0 0000000180015f20     libucrt:ioinit.obj
 0001:00014f20       $unwind$?fin$0@?0??dllmain_crt_process_detach@@YAH_N@Z@4HA 0000000180015f20     LIBCMT:dll_dllmain.obj
 0001:00014f20       $unwind$?fin$0@?0???$?RV<lambda_2d41944a1d46af3157314b8a01080d33>@@AEAV<lambda_8f455de75cd7d7f24b4096f044d8b9e6>@@V<lambda_aa500f224e6afead328df44964fe2772>@@@?$__crt_seh_guarded_call@X@@QEAAX$$QEAV<lambda_2d41944a1d46af3157314b8a01080d33>@@AEAV<lambda_8f455de75cd7d7f24b4096f044d8b9e6>@@$$QEAV<lambda_aa500f224e6afead328df44964fe2772>@@@Z@4HA 0000000180015f20     libucrt:per_thread_data.obj
 0001:00014f20       $unwind$?fin$0@?0???$?RV<lambda_0ae27a3a962d80f24befdcbee591983d>@@AEAV<lambda_8d0ee55de4b1038c4002e0adecdf1839>@@V<lambda_dc504788e8f1664fe9b84e20bfb512f2>@@@?$__crt_seh_guarded_call@X@@QEAAX$$QEAV<lambda_0ae27a3a962d80f24befdcbee591983d>@@AEAV<lambda_8d0ee55de4b1038c4002e0adecdf1839>@@$$QEAV<lambda_dc504788e8f1664fe9b84e20bfb512f2>@@@Z@4HA 0000000180015f20     libucrt:per_thread_data.obj
 0001:00014f20       $unwind$?fin$0@?0??dllmain_crt_process_attach@@YAHQEAUHINSTANCE__@@QEAX@Z@4HA 0000000180015f20     LIBCMT:dll_dllmain.obj
 0001:00014f20       $unwind$_fcloseall$fin$0   0000000180015f20     libucrt:closeall.obj
 0001:00014f20       $unwind$_write$fin$0       0000000180015f20     libucrt:write.obj
 0001:00014f20       $unwind$?fin$0@?0???$?RV<lambda_f2e299630e499de9f9a165e60fcd3db5>@@AEAV<lambda_2ae9d31cdba2644fcbeaf08da7c24588>@@V<lambda_40d01ff24d0e7b3814fdbdcee8eab3c7>@@@?$__crt_seh_guarded_call@X@@QEAAX$$QEAV<lambda_f2e299630e499de9f9a165e60fcd3db5>@@AEAV<lambda_2ae9d31cdba2644fcbeaf08da7c24588>@@$$QEAV<lambda_40d01ff24d0e7b3814fdbdcee8eab3c7>@@@Z@4HA 0000000180015f20     libucrt:per_thread_data.obj
 0001:00014f20       $unwind$?fin$0@?0???$?RV<lambda_842d9ff0dc9ef11c61343bbaebe7f885>@@AEAV<lambda_c5860995281e5c4ce005b3de8f5874ee>@@V<lambda_d90129c13df834fdcbf8d2b88dafcf2d>@@@?$__crt_seh_guarded_call@X@@QEAAX$$QEAV<lambda_842d9ff0dc9ef11c61343bbaebe7f885>@@AEAV<lambda_c5860995281e5c4ce005b3de8f5874ee>@@$$QEAV<lambda_d90129c13df834fdcbf8d2b88dafcf2d>@@@Z@4HA 0000000180015f20     libucrt:fflush.obj
 0001:00014f20       $unwind$_ctrlfp$filt$0     0000000180015f20     libucrt:fpctrl.obj
 0001:00014f20       $unwind$?fin$0@?0???$?RV<lambda_450d765d439847d4c735a33c368b5fc0>@@AEAV<lambda_44731a7d0e6d81c3e6aa82d741081786>@@V<lambda_601a2a7da3b7a96e9554ac7215c4b07c>@@@?$__crt_seh_guarded_call@P6AXH@Z@@QEAAP6AXH@Z$$QEAV<lambda_450d765d439847d4c735a33c368b5fc0>@@AEAV<lambda_44731a7d0e6d81c3e6aa82d741081786>@@$$QEAV<lambda_601a2a7da3b7a96e9554ac7215c4b07c>@@@Z@4HA 0000000180015f20     libucrt:signal.obj
 0001:00014f20       $unwind$fclose$fin$0       0000000180015f20     libucrt:fclose.obj
 0001:00014f20       $unwind$_IsNonwritableInCurrentImage$filt$0 0000000180015f20     LIBCMT:pesect.obj
 0001:00014f20       $unwind$?fin$0@?0???$?RV<lambda_7777bce6b2f8c936911f934f8298dc43>@@AEAV<lambda_f03950bc5685219e0bcd2087efbe011e>@@V<lambda_3883c3dff614d5e0c5f61bb1ac94921c>@@@?$__crt_seh_guarded_call@H@@QEAAH$$QEAV<lambda_7777bce6b2f8c936911f934f8298dc43>@@AEAV<lambda_f03950bc5685219e0bcd2087efbe011e>@@$$QEAV<lambda_3883c3dff614d5e0c5f61bb1ac94921c>@@@Z@4HA 0000000180015f20     libucrt:onexit.obj
 0001:00014f20       $unwind$__DestructExceptionObject$filt$0 0000000180015f20     libvcruntime:ehhelpers.obj
 0001:00014f20       $unwind$?fin$0@?0???$?RV<lambda_410d79af7f07d98d83a3f525b3859a53>@@AEAV<lambda_3e16ef9562a7dcce91392c22ab16ea36>@@V<lambda_38119f0e861e05405d8a144b9b982f0a>@@@?$__crt_seh_guarded_call@X@@QEAAX$$QEAV<lambda_410d79af7f07d98d83a3f525b3859a53>@@AEAV<lambda_3e16ef9562a7dcce91392c22ab16ea36>@@$$QEAV<lambda_38119f0e861e05405d8a144b9b982f0a>@@@Z@4HA 0000000180015f20     libucrt:wsetlocale.obj
 0001:00014f20       $unwind$?fin$0@?0???$?RV<lambda_a37b2b86f63e897a80ea819b0eb08c01>@@AEAV<lambda_38ce7e780aa69e748d6df282ebc68efe>@@V<lambda_99fb1378e971ab6e7edea83e3a7a83a2>@@@?$__crt_seh_guarded_call@H@@QEAAH$$QEAV<lambda_a37b2b86f63e897a80ea819b0eb08c01>@@AEAV<lambda_38ce7e780aa69e748d6df282ebc68efe>@@$$QEAV<lambda_99fb1378e971ab6e7edea83e3a7a83a2>@@@Z@4HA 0000000180015f20     libucrt:commit.obj
 0001:00014f20       $unwind$_query_new_handler$fin$0 0000000180015f20     libucrt:new_handler.obj
 0001:00014f20       $unwind$?fin$0@?0???$?RV<lambda_d80eeec6fff315bfe5c115232f3240e3>@@AEAV<lambda_6e4b09c48022b2350581041d5f6b0c4c>@@V<lambda_2358e3775559c9db80273638284d5e45>@@@?$__crt_seh_guarded_call@X@@QEAAX$$QEAV<lambda_d80eeec6fff315bfe5c115232f3240e3>@@AEAV<lambda_6e4b09c48022b2350581041d5f6b0c4c>@@$$QEAV<lambda_2358e3775559c9db80273638284d5e45>@@@Z@4HA 0000000180015f20     libucrt:exit.obj
 0001:00014f20       $unwind$__acrt_lowio_ensure_fh_exists$fin$0 0000000180015f20     libucrt:osfinfo.obj
 0001:00014f20       $unwind$?filt$0@?0???R<lambda_6e4b09c48022b2350581041d5f6b0c4c>@@QEBA@XZ@4HA 0000000180015f20     libucrt:exit.obj
 0001:00014f20       $unwind$?fin$0@?0???$?RV<lambda_751a882b2c74d4b022dec766aa51a29a>@@AEAV<lambda_628dfdc04ba53c8bfc02c9951375f3f5>@@V<lambda_f6c7be5f7998530c34de24c7437d6b54>@@@?$__crt_seh_guarded_call@H@@QEAAH$$QEAV<lambda_751a882b2c74d4b022dec766aa51a29a>@@AEAV<lambda_628dfdc04ba53c8bfc02c9951375f3f5>@@$$QEAV<lambda_f6c7be5f7998530c34de24c7437d6b54>@@@Z@4HA 0000000180015f20     libucrt:close.obj
 0001:00014f20       $unwind$?fin$0@?0???$?RV<lambda_886d6c58226a84441f68b9f2b8217b83>@@AEAV<lambda_ab61a845afdef5b7c387490eaf3616ee>@@V<lambda_f7f22ab5edc0698d5f6905b0d3f44752>@@@?$__crt_seh_guarded_call@X@@QEAAX$$QEAV<lambda_886d6c58226a84441f68b9f2b8217b83>@@AEAV<lambda_ab61a845afdef5b7c387490eaf3616ee>@@$$QEAV<lambda_f7f22ab5edc0698d5f6905b0d3f44752>@@@Z@4HA 0000000180015f20     libucrt:fflush.obj
 0001:00014f20       $unwind$raise$fin$0        0000000180015f20     libucrt:signal.obj
 0001:00014f20       $unwind$__acrt_update_thread_locale_data$fin$0 0000000180015f20     libucrt:locale_refcounting.obj
 0001:00014f20       $unwind$?fin$0@?0??update_thread_multibyte_data_internal@@YAPEAU__crt_multibyte_data@@QEAU__acrt_ptd@@QEAPEAU1@@Z@4HA 0000000180015f20     libucrt:mbctype.obj
 0001:00014f20       $unwind$?fin$0@?0???$?RV<lambda_aa87e3671a710a21b5dc78c0bdf72e11>@@AEAV<lambda_92619d2358a28f41a33ba319515a20b9>@@V<lambda_6992ecaafeb10aed2b74cb1fae11a551>@@@?$__crt_seh_guarded_call@X@@QEAAX$$QEAV<lambda_aa87e3671a710a21b5dc78c0bdf72e11>@@AEAV<lambda_92619d2358a28f41a33ba319515a20b9>@@$$QEAV<lambda_6992ecaafeb10aed2b74cb1fae11a551>@@@Z@4HA 0000000180015f20     libucrt:per_thread_data.obj
 0001:00014f20       $unwind$?fin$0@?0???$?RV<lambda_efdfa57d1f175319df784efa44bb7b81>@@AEAV<lambda_5f0a4c1567f8adc6734073e5d1e1b35c>@@V<lambda_2e8a7d3640ea6ccb4c2413664c2db6fd>@@@?$__crt_seh_guarded_call@X@@QEAAX$$QEAV<lambda_efdfa57d1f175319df784efa44bb7b81>@@AEAV<lambda_5f0a4c1567f8adc6734073e5d1e1b35c>@@$$QEAV<lambda_2e8a7d3640ea6ccb4c2413664c2db6fd>@@@Z@4HA 0000000180015f20     libucrt:mbctype.obj
 0001:00014f28       $unwind$?dllmain_crt_process_detach@@YAH_N@Z 0000000180015f28     LIBCMT:dll_dllmain.obj
 0001:00014f5c       $unwind$?dllmain_dispatch@@YAHQEAUHINSTANCE__@@KQEAX@Z 0000000180015f5c     LIBCMT:dll_dllmain.obj
 0001:00014f84       $unwind$?filt$0@?0??dllmain_dispatch@@YAHQEAUHINSTANCE__@@KQEAX@Z@4HA 0000000180015f84     LIBCMT:dll_dllmain.obj
 0001:00014f8c       $unwind$?__scrt_throw_std_bad_alloc@@YAXXZ 0000000180015f8c     LIBCMT:throw_bad_alloc.obj
 0001:00014f8c       $unwind$_raise_exc         0000000180015f8c     libucrt:fpexcept.obj
 0001:00014f8c       $unwind$?__scrt_throw_std_bad_array_new_length@@YAXXZ 0000000180015f8c     LIBCMT:throw_bad_alloc.obj
 0001:00014f94       $unwind$__security_init_cookie 0000000180015f94     LIBCMT:gs_support.obj
 0001:00014fa0       $unwind$__scrt_is_nonwritable_in_current_image 0000000180015fa0     LIBCMT:utility.obj
 0001:00014fc0       $unwind$__scrt_is_nonwritable_in_current_image$filt$0 0000000180015fc0     LIBCMT:utility.obj
 0001:00014fc8       $unwind$__scrt_initialize_onexit_tables 0000000180015fc8     LIBCMT:utility.obj
 0001:00014fd4       $unwind$?setSBCS@@YAXPEAU__crt_multibyte_data@@@Z 0000000180015fd4     libucrt:mbctype.obj
 0001:00014fd4       $unwind$_recalloc_base     0000000180015fd4     libucrt:recalloc.obj
 0001:00014fd4       $unwind$__scrt_dllmain_exception_filter 0000000180015fd4     LIBCMT:utility.obj
 0001:00014fd4       $unwind$__acrt_lowio_create_handle_array 0000000180015fd4     libucrt:osfinfo.obj
 0001:00014fd4       $unwind$_initterm          0000000180015fd4     libucrt:initterm.obj
 0001:00014fd4       $unwind$_seh_filter_exe    0000000180015fd4     libucrt:exception_filter.obj
 0001:00014fd4       $unwind$__acrt_free_locale 0000000180015fd4     libucrt:locale_refcounting.obj
 0001:00014fe8       $unwind$__scrt_fastfail    0000000180015fe8     LIBCMT:utility_desktop.obj
 0001:00014ff8       $unwind$__isa_available_init 0000000180015ff8     LIBCMT:_cpu_disp_.obj
 0001:00015010       $xdatasym                  0000000180016010     LIBCMT:_guard_dispatch_.obj
 0001:00015018       $xdatasym                  0000000180016018     libvcruntime:memset.obj
 0001:0001501c       $unwind$__C_specific_handler 000000018001601c     libvcruntime:_riscchandler_.obj
 0001:00015038       $unwind$?initialize_stdio_handles_nolock@@YAXXZ 0000000180016038     libucrt:ioinit.obj
 0001:00015038       $unwind$__std_exception_copy 0000000180016038     libvcruntime:std_exception.obj
 0001:00015038       $unwind$_free_osfhnd       0000000180016038     libucrt:osfinfo.obj
 0001:0001504c       $unwind$_CxxThrowException 000000018001604c     libvcruntime:throw.obj
 0001:00015060       $xdatasym                  0000000180016060     libvcruntime:_jmpuwind_.obj
 0001:00015074       $unwind$__acrt_initialize_winapi_thunks 0000000180016074     libucrt:winapi_thunks.obj
 0001:00015074       $unwind$__vcrt_initialize_winapi_thunks 0000000180016074     libvcruntime:winapi_downlevel.obj
 0001:0001507c       $unwind$__vcrt_uninitialize_winapi_thunks 000000018001607c     libvcruntime:winapi_downlevel.obj
 0001:00015084       $unwind$?try_get_function@@YAPEAXW4function_id@?A0x89697e75@@QEBDQEBW4module_id@2@2@Z 0000000180016084     libvcruntime:winapi_downlevel.obj
 0001:00015084       $unwind$??R<lambda_f03950bc5685219e0bcd2087efbe011e>@@QEBAHXZ 0000000180016084     libucrt:onexit.obj
 0001:00015084       $unwind$?try_get_function@@YAPEAXW4function_id@?A0x391cf84c@@QEBDQEBW4module_id@2@2@Z 0000000180016084     libucrt:winapi_thunks.obj
 0001:000150a0       $xdatasym                  00000001800160a0     libvcruntime:memcpy.obj
 0001:000150a8       $xdatasym                  00000001800160a8     libvcruntime:handlers.obj
 0001:000150b0       $unwind$__DestructExceptionObject 00000001800160b0     libvcruntime:ehhelpers.obj
 0001:000150d0       $unwind$_query_new_handler 00000001800160d0     libucrt:new_handler.obj
 0001:000150f0       $unwind$?common_exit@@YAXHW4_crt_exit_cleanup_mode@@W4_crt_exit_return_mode@@@Z 00000001800160f0     libucrt:exit.obj
 0001:000150fc       $unwind$??R<lambda_6e4b09c48022b2350581041d5f6b0c4c>@@QEBA@XZ 00000001800160fc     libucrt:exit.obj
 0001:0001511c       $unwind$??$?RV<lambda_d80eeec6fff315bfe5c115232f3240e3>@@AEAV<lambda_6e4b09c48022b2350581041d5f6b0c4c>@@V<lambda_2358e3775559c9db80273638284d5e45>@@@?$__crt_seh_guarded_call@X@@QEAAX$$QEAV<lambda_d80eeec6fff315bfe5c115232f3240e3>@@AEAV<lambda_6e4b09c48022b2350581041d5f6b0c4c>@@$$QEAV<lambda_2358e3775559c9db80273638284d5e45>@@@Z 000000018001611c     libucrt:exit.obj
 0001:00015140       $unwind$_configure_narrow_argv 0000000180016140     libucrt:argv_parsing.obj
 0001:00015154       $unwind$??$parse_command_line@D@@YAXPEADPEAPEAD0PEA_K2@Z 0000000180016154     libucrt:argv_parsing.obj
 0001:00015170       $unwind$??$free_environment@_W@@YAXQEAPEA_W@Z 0000000180016170     libucrt:environment_initialization.obj
 0001:00015170       $unwind$??$free_environment@D@@YAXQEAPEAD@Z 0000000180016170     libucrt:environment_initialization.obj
 0001:0001517c       $unwind$??$create_environment@D@@YAQEAPEADQEAD@Z 000000018001617c     libucrt:environment_initialization.obj
 0001:00015194       $unwind$_execute_onexit_table 0000000180016194     libucrt:onexit.obj
 0001:0001519c       $unwind$??$?RV<lambda_7777bce6b2f8c936911f934f8298dc43>@@AEAV<lambda_f03950bc5685219e0bcd2087efbe011e>@@V<lambda_3883c3dff614d5e0c5f61bb1ac94921c>@@@?$__crt_seh_guarded_call@H@@QEAAH$$QEAV<lambda_7777bce6b2f8c936911f934f8298dc43>@@AEAV<lambda_f03950bc5685219e0bcd2087efbe011e>@@$$QEAV<lambda_3883c3dff614d5e0c5f61bb1ac94921c>@@@Z 000000018001619c     libucrt:onexit.obj
 0001:000151c0       $unwind$terminate          00000001800161c0     libucrt:terminate.obj
 0001:000151e0       $xdatasym                  00000001800161e0     libucrt:strncmp.obj
 0001:000151e4       $unwind$__acrt_locale_free_lc_time_if_unreferenced 00000001800161e4     libucrt:locale_refcounting.obj
 0001:000151e4       $unwind$__acrt_locale_free_numeric 00000001800161e4     libucrt:initnum.obj
 0001:000151e4       $unwind$?destroy_fls@@YAXPEAX@Z 00000001800161e4     libucrt:per_thread_data.obj
 0001:000151e4       $unwind$_free_base         00000001800161e4     libucrt:free_base.obj
 0001:000151ec       $unwind$?construct_ptd_array@@YAXQEAU__acrt_ptd@@@Z 00000001800161ec     libucrt:per_thread_data.obj
 0001:000151f4       $unwind$?destroy_ptd_array@@YAXQEAU__acrt_ptd@@@Z 00000001800161f4     libucrt:per_thread_data.obj
 0001:000151fc       $unwind$??$?RV<lambda_0ae27a3a962d80f24befdcbee591983d>@@AEAV<lambda_8d0ee55de4b1038c4002e0adecdf1839>@@V<lambda_dc504788e8f1664fe9b84e20bfb512f2>@@@?$__crt_seh_guarded_call@X@@QEAAX$$QEAV<lambda_0ae27a3a962d80f24befdcbee591983d>@@AEAV<lambda_8d0ee55de4b1038c4002e0adecdf1839>@@$$QEAV<lambda_dc504788e8f1664fe9b84e20bfb512f2>@@@Z 00000001800161fc     libucrt:per_thread_data.obj
 0001:00015220       $unwind$??$?RV<lambda_aa87e3671a710a21b5dc78c0bdf72e11>@@AEAV<lambda_92619d2358a28f41a33ba319515a20b9>@@V<lambda_6992ecaafeb10aed2b74cb1fae11a551>@@@?$__crt_seh_guarded_call@X@@QEAAX$$QEAV<lambda_aa87e3671a710a21b5dc78c0bdf72e11>@@AEAV<lambda_92619d2358a28f41a33ba319515a20b9>@@$$QEAV<lambda_6992ecaafeb10aed2b74cb1fae11a551>@@@Z 0000000180016220     libucrt:per_thread_data.obj
 0001:00015244       $unwind$??$?RV<lambda_f2e299630e499de9f9a165e60fcd3db5>@@AEAV<lambda_2ae9d31cdba2644fcbeaf08da7c24588>@@V<lambda_40d01ff24d0e7b3814fdbdcee8eab3c7>@@@?$__crt_seh_guarded_call@X@@QEAAX$$QEAV<lambda_f2e299630e499de9f9a165e60fcd3db5>@@AEAV<lambda_2ae9d31cdba2644fcbeaf08da7c24588>@@$$QEAV<lambda_40d01ff24d0e7b3814fdbdcee8eab3c7>@@@Z 0000000180016244     libucrt:per_thread_data.obj
 0001:00015268       $unwind$??$?RV<lambda_2d41944a1d46af3157314b8a01080d33>@@AEAV<lambda_8f455de75cd7d7f24b4096f044d8b9e6>@@V<lambda_aa500f224e6afead328df44964fe2772>@@@?$__crt_seh_guarded_call@X@@QEAAX$$QEAV<lambda_2d41944a1d46af3157314b8a01080d33>@@AEAV<lambda_8f455de75cd7d7f24b4096f044d8b9e6>@@$$QEAV<lambda_aa500f224e6afead328df44964fe2772>@@@Z 0000000180016268     libucrt:per_thread_data.obj
 0001:0001528c       $unwind$_invalid_parameter_noinfo 000000018001628c     libucrt:invalid_parameter.obj
 0001:0001528c       $unwind$_log10_special     000000018001628c     libucrt:log_special.obj
 0001:00015294       $unwind$__acrt_call_reportfault 0000000180016294     libucrt:invalid_parameter.obj
 0001:000152b4       $unwind$_invalid_parameter 00000001800162b4     libucrt:invalid_parameter.obj
 0001:000152c8       $unwind$??$common_expand_argv_wildcards@D@@YAHQEAPEADQEAPEAPEAD@Z 00000001800162c8     libucrt:argv_wildcards.obj
 0001:000152e0       $unwind$??$copy_and_add_argument_to_buffer@D@@YAHQEBD0_KAEAV?$argument_list@D@?A0x5f5c8891@@@Z 00000001800162e0     libucrt:argv_wildcards.obj
 0001:000152fc       $unwind$??$expand_argument_wildcards@D@@YAHQEAD0AEAV?$argument_list@D@?A0x5f5c8891@@@Z 00000001800162fc     libucrt:argv_wildcards.obj
 0001:0001531c       $unwind$_setmbcp_nolock    000000018001631c     libucrt:mbctype.obj
 0001:0001533c       $unwind$?getSystemCP@@YAHH@Z 000000018001633c     libucrt:mbctype.obj
 0001:0001533c       $unwind$__dcrt_lowio_ensure_console_output_initialized 000000018001633c     libucrt:initcon.obj
 0001:0001533c       $unwind$_isleadbyte_l      000000018001633c     libucrt:_wctype.obj
 0001:00015344       $unwind$?update_thread_multibyte_data_internal@@YAPEAU__crt_multibyte_data@@QEAU__acrt_ptd@@QEAPEAU1@@Z 0000000180016344     libucrt:mbctype.obj
 0001:0001536c       $unwind$?setmbcp_internal@@YAHH_NQEAU__acrt_ptd@@QEAPEAU__crt_multibyte_data@@@Z 000000018001636c     libucrt:mbctype.obj
 0001:0001537c       $unwind$?setSBUpLow@@YAXPEAU__crt_multibyte_data@@@Z 000000018001637c     libucrt:mbctype.obj
 0001:00015398       $unwind$??$?RV<lambda_efdfa57d1f175319df784efa44bb7b81>@@AEAV<lambda_5f0a4c1567f8adc6734073e5d1e1b35c>@@V<lambda_2e8a7d3640ea6ccb4c2413664c2db6fd>@@@?$__crt_seh_guarded_call@X@@QEAAX$$QEAV<lambda_efdfa57d1f175319df784efa44bb7b81>@@AEAV<lambda_5f0a4c1567f8adc6734073e5d1e1b35c>@@$$QEAV<lambda_2e8a7d3640ea6ccb4c2413664c2db6fd>@@@Z 0000000180016398     libucrt:mbctype.obj
 0001:000153c0       $unwind$?x_ismbbtype_l@@YAHPEAU__crt_locale_pointers@@IHH@Z 00000001800163c0     libucrt:ismbbyte.obj
 0001:000153d0       $unwind$__dcrt_get_narrow_environment_from_os 00000001800163d0     libucrt:get_environment_from_os.obj
 0001:000153e8       $unwind$__acrt_LCMapStringEx 00000001800163e8     libucrt:winapi_thunks.obj
 0001:000153fc       $unwind$__acrt_initialize_lowio 00000001800163fc     libucrt:ioinit.obj
 0001:0001541c       $unwind$?initialize_inherited_file_handles_nolock@@YAXXZ 000000018001641c     libucrt:ioinit.obj
 0001:00015438       $unwind$__acrt_get_sigabrt_handler 0000000180016438     libucrt:signal.obj
 0001:00015438       $unwind$__acrt_uninitialize_locale 0000000180016438     libucrt:wsetlocale.obj
 0001:00015440       $unwind$raise              0000000180016440     libucrt:signal.obj
 0001:0001546c       $unwind$??$?RV<lambda_450d765d439847d4c735a33c368b5fc0>@@AEAV<lambda_44731a7d0e6d81c3e6aa82d741081786>@@V<lambda_601a2a7da3b7a96e9554ac7215c4b07c>@@@?$__crt_seh_guarded_call@P6AXH@Z@@QEAAP6AXH@Z$$QEAV<lambda_450d765d439847d4c735a33c368b5fc0>@@AEAV<lambda_44731a7d0e6d81c3e6aa82d741081786>@@$$QEAV<lambda_601a2a7da3b7a96e9554ac7215c4b07c>@@@Z 000000018001646c     libucrt:signal.obj
 0001:00015490       $unwind$?common_flush_all@@YAH_N@Z 0000000180016490     libucrt:fflush.obj
 0001:00015498       $unwind$??$?RV<lambda_842d9ff0dc9ef11c61343bbaebe7f885>@@AEAV<lambda_c5860995281e5c4ce005b3de8f5874ee>@@V<lambda_d90129c13df834fdcbf8d2b88dafcf2d>@@@?$__crt_seh_guarded_call@X@@QEAAX$$QEAV<lambda_842d9ff0dc9ef11c61343bbaebe7f885>@@AEAV<lambda_c5860995281e5c4ce005b3de8f5874ee>@@$$QEAV<lambda_d90129c13df834fdcbf8d2b88dafcf2d>@@@Z 0000000180016498     libucrt:fflush.obj
 0001:000154bc       $unwind$??$?RV<lambda_886d6c58226a84441f68b9f2b8217b83>@@AEAV<lambda_ab61a845afdef5b7c387490eaf3616ee>@@V<lambda_f7f22ab5edc0698d5f6905b0d3f44752>@@@?$__crt_seh_guarded_call@X@@QEAAX$$QEAV<lambda_886d6c58226a84441f68b9f2b8217b83>@@AEAV<lambda_ab61a845afdef5b7c387490eaf3616ee>@@$$QEAV<lambda_f7f22ab5edc0698d5f6905b0d3f44752>@@@Z 00000001800164bc     libucrt:fflush.obj
 0001:000154e4       $unwind$__acrt_initialize_stdio 00000001800164e4     libucrt:_file.obj
 0001:000154fc       $unwind$_mbtowc_l          00000001800164fc     libucrt:mbtowc.obj
 0001:00015514       $unwind$??$?RV<lambda_410d79af7f07d98d83a3f525b3859a53>@@AEAV<lambda_3e16ef9562a7dcce91392c22ab16ea36>@@V<lambda_38119f0e861e05405d8a144b9b982f0a>@@@?$__crt_seh_guarded_call@X@@QEAAX$$QEAV<lambda_410d79af7f07d98d83a3f525b3859a53>@@AEAV<lambda_3e16ef9562a7dcce91392c22ab16ea36>@@$$QEAV<lambda_38119f0e861e05405d8a144b9b982f0a>@@@Z 0000000180016514     libucrt:wsetlocale.obj
 0001:0001553c       $unwind$__acrt_update_thread_locale_data 000000018001653c     libucrt:locale_refcounting.obj
 0001:00015560       $unwind$qsort              0000000180016560     libucrt:qsort.obj
 0001:00015578       $chain$4$qsort             0000000180016578     libucrt:qsort.obj
 0001:0001559c       $chain$5$qsort             000000018001659c     libucrt:qsort.obj
 0001:000155ac       $unwind$strpbrk            00000001800165ac     libucrt:strpbrk.obj
 0001:000155bc       $unwind$fallbackMethod     00000001800165bc     libucrt:strpbrk.obj
 0001:000155cc       $unwind$_mbsdec_l          00000001800165cc     libucrt:mbsdec.obj
 0001:000155d8       $unwind$__acrt_GetStringTypeA 00000001800165d8     libucrt:getstringtypea.obj
 0001:00015600       $unwind$__acrt_LCMapStringA 0000000180016600     libucrt:lcmapstringa.obj
 0001:00015610       $unwind$?__acrt_LCMapStringA_stat@@YAHPEAU__crt_locale_pointers@@PEB_WKPEBDHPEADHHH@Z 0000000180016610     libucrt:lcmapstringa.obj
 0001:00015638       $unwind$?GetTableIndexFromLocaleName@@YAHPEB_W@Z 0000000180016638     libucrt:lcidtoname_downlevel.obj
 0001:00015650       $unwind$__acrt_lowio_destroy_handle_array 0000000180016650     libucrt:osfinfo.obj
 0001:00015660       $unwind$__acrt_lowio_ensure_fh_exists 0000000180016660     libucrt:osfinfo.obj
 0001:0001568c       $unwind$_close             000000018001668c     libucrt:close.obj
 0001:0001568c       $unwind$_commit            000000018001668c     libucrt:commit.obj
 0001:00015694       $unwind$??$?RV<lambda_a37b2b86f63e897a80ea819b0eb08c01>@@AEAV<lambda_38ce7e780aa69e748d6df282ebc68efe>@@V<lambda_99fb1378e971ab6e7edea83e3a7a83a2>@@@?$__crt_seh_guarded_call@H@@QEAAH$$QEAV<lambda_a37b2b86f63e897a80ea819b0eb08c01>@@AEAV<lambda_38ce7e780aa69e748d6df282ebc68efe>@@$$QEAV<lambda_99fb1378e971ab6e7edea83e3a7a83a2>@@@Z 0000000180016694     libucrt:commit.obj
 0001:000156b8       $unwind$_write             00000001800166b8     libucrt:write.obj
 0001:000156e8       $unwind$_write_nolock      00000001800166e8     libucrt:write.obj
 0001:00015700       $unwind$?write_double_translated_ansi_nolock@@YA?AUwrite_result@?A0x17268360@@HQEBDI@Z 0000000180016700     libucrt:write.obj
 0001:00015720       $unwind$?write_text_ansi_nolock@@YA?AUwrite_result@?A0x17268360@@HQEBDI@Z 0000000180016720     libucrt:write.obj
 0001:00015720       $unwind$?write_text_utf16le_nolock@@YA?AUwrite_result@?A0x17268360@@HQEBDI@Z 0000000180016720     libucrt:write.obj
 0001:00015740       $unwind$?write_text_utf8_nolock@@YA?AUwrite_result@?A0x17268360@@HQEBDI@Z 0000000180016740     libucrt:write.obj
 0001:00015764       $unwind$_fcloseall         0000000180016764     libucrt:closeall.obj
 0001:00015788       $unwind$__acrt_locale_free_monetary 0000000180016788     libucrt:initmon.obj
 0001:00015790       $unwind$__acrt_locale_free_time 0000000180016790     libucrt:inittime.obj
 0001:000157a0       $unwind$_putwch_nolock     00000001800167a0     libucrt:putwch.obj
 0001:000157a8       $unwind$fclose             00000001800167a8     libucrt:fclose.obj
 0001:000157d0       $xdatasym                  00000001800167d0     libucrt:log10.obj
 0001:000157dc       $unwind$__dcrt_write_console_w 00000001800167dc     libucrt:initcon.obj
 0001:000157f0       $unwind$??$?RV<lambda_751a882b2c74d4b022dec766aa51a29a>@@AEAV<lambda_628dfdc04ba53c8bfc02c9951375f3f5>@@V<lambda_f6c7be5f7998530c34de24c7437d6b54>@@@?$__crt_seh_guarded_call@H@@QEAAH$$QEAV<lambda_751a882b2c74d4b022dec766aa51a29a>@@AEAV<lambda_628dfdc04ba53c8bfc02c9951375f3f5>@@$$QEAV<lambda_f6c7be5f7998530c34de24c7437d6b54>@@@Z 00000001800167f0     libucrt:close.obj
 0001:00015814       $unwind$_call_matherr      0000000180016814     libucrt:libm_error.obj
 0001:0001581c       $unwind$_handle_error      000000018001681c     libucrt:libm_error.obj
 0001:0001583c       $unwind$__acrt_initialize_fma3 000000018001683c     libucrt:fma3_available.obj
 0001:00015844       $unwind$_log_special_common 0000000180016844     libucrt:log_special.obj
 0001:00015850       $xdatasym                  0000000180016850     libucrt:fpsr.obj
 0001:00015858       $unwind$_raise_exc_ex      0000000180016858     libucrt:fpexcept.obj
 0001:0001586c       $unwind$_ctrlfp            000000018001686c     libucrt:fpctrl.obj
 0001:00015894       $unwind$_IsNonwritableInCurrentImage 0000000180016894     LIBCMT:pesect.obj
 0001:000158b8       $unwind$__GSHandlerCheckCommon 00000001800168b8     LIBCMT:_gshandler_.obj
 0001:000158c0       $xdatasym                  00000001800168c0     LIBCMT:_amdsecgs_.obj
 0001:000158c4       $unwind$__report_securityfailure 00000001800168c4     LIBCMT:gs_report.obj
 0001:000158cc       $unwind$__report_gsfailure 00000001800168cc     LIBCMT:gs_report.obj
 0001:000158d4       $unwind$capture_current_context 00000001800168d4     LIBCMT:gs_report.obj
 0001:000158e0       $unwind$capture_previous_context 00000001800168e0     LIBCMT:gs_report.obj
 0001:000158f0       $xdatasym                  00000001800168f0     libvcruntime:memcmp.obj
 0001:000159f0       .edata                     00000001800169f0     Brackets.exp
 0001:00015a18       rgpv                       0000000180016a18     Brackets.exp
 0001:00015a2c       rgszName                   0000000180016a2c     Brackets.exp
 0001:00015a40       rgwOrd                     0000000180016a40     Brackets.exp
 0001:00015a4a       szName                     0000000180016a4a     Brackets.exp
 0001:00015a57       $N00001                    0000000180016a57     Brackets.exp
 0001:00015a62       $N00002                    0000000180016a62     Brackets.exp
 0001:00015a71       $N00003                    0000000180016a71     Brackets.exp
 0001:00015a80       $N00004                    0000000180016a80     Brackets.exp
 0001:00015a86       $N00005                    0000000180016a86     Brackets.exp
 0002:00000000       ?HelpTopic@?1??ShowMenu@@YAHH@Z@4PAPEB_WA 0000000180017000     Brackets.obj
 0002:00000010       ?CmdName@?BB@??OpenW@@9@4PAU<unnamed-type-CmdName>@?BB@??1@YAPEAXPEBUOpenInfo@@@Z@A 0000000180017010     Brackets.obj
 0002:000000a0       ?__vcrt_flsindex@@3KA      00000001800170a0     libvcruntime:per_thread_data.obj
 0002:000000b4       ?__acrt_flsindex@@3KA      00000001800170b4     libucrt:per_thread_data.obj
 0002:000000b8       ?errno_no_memory@@3HA      00000001800170b8     libucrt:errno.obj
 0002:000000bc       ?doserrno_no_memory@@3KA   00000001800170bc     libucrt:errno.obj
 0002:000002f0       _mbctypes                  00000001800172f0     libucrt:mbctype.obj
 0002:00000400       _mbcasemaps                0000000180017400     libucrt:mbctype.obj
 0002:00000500       ?__rgctypeflag@@3PADA      0000000180017500     libucrt:mbctype.obj
 0002:00000510       ?__rgcode_page_info@@3PAUcode_page_info@@A 0000000180017510     libucrt:mbctype.obj
 0002:00000920       ?__dcrt_lowio_console_output_handle@@3PEAXEA 0000000180017920     libucrt:initcon.obj
 0002:00000930       ?dazSupported@?1??_ctrlfp@@9@9 0000000180017930     libucrt:fpctrl.obj
 0002:000009f0       ?Opt@@3UOptions@@A         00000001800179f0     Brackets.obj
 0002:00000ab0       ?Info@@3UPluginStartupInfo@@A 0000000180017ab0     Brackets.obj
 0002:00000bc0       ?PluginMenuStrings@?1??GetPluginInfoW@@9@4PAPEB_WA 0000000180017bc0     Brackets.obj
 0002:00000bc8       ?__proc_attached@@3HA      0000000180017bc8     LIBCMT:dll_dllmain.obj
 0002:00000bf4       ?module_local_atexit_table_initialized@@3_NA 0000000180017bf4     LIBCMT:utility.obj
 0002:00000c00       ?module_local_atexit_table@@3U_onexit_table_t@@A 0000000180017c00     LIBCMT:utility.obj
 0002:00000c18       ?module_local_at_quick_exit_table@@3U_onexit_table_t@@A 0000000180017c18     LIBCMT:utility.obj
 0002:00000c30       ?is_initialized_as_dll@@3_NA 0000000180017c30     LIBCMT:utility.obj
 0002:00000c80       ?heap@@3V_HeapManager@@A   0000000180017c80     libvcruntime:undname.obj
 0002:00000cb0       ?__vcrt_startup_thread_ptd@@3U__vcrt_ptd@@A 0000000180017cb0     libvcruntime:per_thread_data.obj
 0002:00000d28       __vcrt_lock_table          0000000180017d28     libvcruntime:locks.obj
 0002:00000d50       __vcrt_locks_initialized   0000000180017d50     libvcruntime:locks.obj
 0002:00000d58       ?module_handles@@3PAPEAUHINSTANCE__@@A 0000000180017d58     libvcruntime:winapi_downlevel.obj
 0002:00000d70       ?encoded_function_pointers@@3PAPEAXA 0000000180017d70     libvcruntime:winapi_downlevel.obj
 0002:00000da8       ?__acrt_new_handler@@3V?$dual_state_global@P6AH_K@Z@__crt_state_management@@A 0000000180017da8     libucrt:new_handler.obj
 0002:00000db0       ?c_termination_complete@@3JA 0000000180017db0     libucrt:exit.obj
 0002:00000db8       ?thread_local_exit_callback_func@@3P6AXPEAXK0@ZEA 0000000180017db8     libucrt:exit.obj
 0002:00000dd0       ?program_name@?1???$common_configure_argv@D@@YAHW4_crt_argv_mode@@@Z@4PADA 0000000180017dd0     libucrt:argv_parsing.obj
 0002:00000f30       ?__acrt_lock_table@@3PAU_RTL_CRITICAL_SECTION@@A 0000000180017f30     libucrt:locks.obj
 0002:00001160       ?__acrt_locks_initialized@@3IA 0000000180018160     libucrt:locks.obj
 0002:00001168       ?__acrt_invalid_parameter_handler@@3V?$dual_state_global@P6AXPEB_W00I_K@Z@__crt_state_management@@A 0000000180018168     libucrt:invalid_parameter.obj
 0002:00001188       ?fSystemSet@@3HA           0000000180018188     libucrt:mbctype.obj
 0002:0000118c       ?initialized@?1??__acrt_initialize_multibyte@@9@4_NA 000000018001818c     libucrt:mbctype.obj
 0002:000011c0       ?module_handles@@3PAPEAUHINSTANCE__@@A 00000001800181c0     libucrt:winapi_thunks.obj
 0002:00001260       ?encoded_function_pointers@@3PAPEAXA 0000000180018260     libucrt:winapi_thunks.obj
 0002:00001788       ?ctrlc_action@@3V?$dual_state_global@P6AXH@Z@__crt_state_management@@A 0000000180018788     libucrt:signal.obj
 0002:00001790       ?ctrlbreak_action@@3V?$dual_state_global@P6AXH@Z@__crt_state_management@@A 0000000180018790     libucrt:signal.obj
 0002:00001798       ?abort_action@@3V?$dual_state_global@P6AXH@Z@__crt_state_management@@A 0000000180018798     libucrt:signal.obj
 0002:000017a0       ?term_action@@3V?$dual_state_global@P6AXH@Z@__crt_state_management@@A 00000001800187a0     libucrt:signal.obj
 0002:000017a8       ?user_matherr@@3V?$dual_state_global@P6AHPEAU_exception@@@Z@__crt_state_management@@A 00000001800187a8     libucrt:matherr.obj
 0002:000017dc       ?__acrt_global_new_mode@@3V?$dual_state_global@J@__crt_state_management@@A 00000001800187dc     libucrt:new_mode.obj
 0002:000017e8       ?__acrt_app_type@@3W4_crt_app_type@@A 00000001800187e8     libucrt:report_runtime_error.obj
 0002:00001800       GS_ExceptionRecord         0000000180018800     LIBCMT:gs_report.obj
 0002:000018a0       GS_ContextRecord           00000001800188a0     LIBCMT:gs_report.obj
 0003:00000180       $pdata$ConfigureW          0000000180019180     Brackets.obj
 0003:0000018c       $pdata$GetGlobalInfoW      000000018001918c     Brackets.obj
 0003:00000198       $pdata$GetPluginInfoW      0000000180019198     Brackets.obj
 0003:000001a4       $pdata$OpenW               00000001800191a4     Brackets.obj
 0003:000001b0       $pdata$SetStartupInfoW     00000001800191b0     Brackets.obj
 0003:0000003c       $pdata$??_G?$DialogItemBinding@UFarDialogItem@@@@UEAAPEAXI@Z 000000018001903c     Brackets.obj
 0003:000000fc       $pdata$?SaveValue@PluginCheckBoxBinding@@UEAAXPEAUFarDialogItem@@H@Z 00000001800190fc     Brackets.obj
 0003:00000048       $pdata$??_GPluginCheckBoxBinding@@UEAAPEAXI@Z 0000000180019048     Brackets.obj
 0003:00000048       $pdata$??_GPluginEditFieldBinding@@UEAAPEAXI@Z 0000000180019048     Brackets.obj
 0003:00000120       $pdata$?SaveValue@PluginRadioButtonBinding@@UEAAXPEAUFarDialogItem@@H@Z 0000000180019120     Brackets.obj
 0003:0000006c       $pdata$??_GPluginRadioButtonBinding@@UEAAPEAXI@Z 000000018001906c     Brackets.obj
 0003:00000108       $pdata$?SaveValue@PluginEditFieldBinding@@UEAAXPEAUFarDialogItem@@H@Z 0000000180019108     Brackets.obj
 0003:00000114       $pdata$?SaveValue@PluginIntEditFieldBinding@@UEAAXPEAUFarDialogItem@@H@Z 0000000180019114     Brackets.obj
 0003:00000060       $pdata$??_GPluginUIntEditFieldBinding@@UEAAPEAXI@Z 0000000180019060     Brackets.obj
 0003:00000060       $pdata$??_GPluginIntEditFieldBinding@@UEAAPEAXI@Z 0000000180019060     Brackets.obj
 0003:0000012c       $pdata$?SaveValue@PluginUIntEditFieldBinding@@UEAAXPEAUFarDialogItem@@H@Z 000000018001912c     Brackets.obj
 0003:0000009c       $pdata$?AddDialogItem@?$DialogBuilderBase@UFarDialogItem@@@@IEAAPEAUFarDialogItem@@W4FARDIALOGITEMTYPES@@PEB_W@Z 000000018001909c     Brackets.obj
 0003:00000144       $pdata$?UpdateBorderSize@?$DialogBuilderBase@UFarDialogItem@@@@IEAAXXZ 0000000180019144     Brackets.obj
 0003:00000150       $pdata$1$?UpdateBorderSize@?$DialogBuilderBase@UFarDialogItem@@@@IEAAXXZ 0000000180019150     Brackets.obj
 0003:0000015c       $pdata$2$?UpdateBorderSize@?$DialogBuilderBase@UFarDialogItem@@@@IEAAXXZ 000000018001915c     Brackets.obj
 0003:00000168       $pdata$3$?UpdateBorderSize@?$DialogBuilderBase@UFarDialogItem@@@@IEAAXXZ 0000000180019168     Brackets.obj
 0003:00000174       $pdata$4$?UpdateBorderSize@?$DialogBuilderBase@UFarDialogItem@@@@IEAAXXZ 0000000180019174     Brackets.obj
 0003:0000000c       $pdata$??1?$DialogBuilderBase@UFarDialogItem@@@@MEAA@XZ 000000018001900c     Brackets.obj
 0003:00000018       $pdata$0$??1?$DialogBuilderBase@UFarDialogItem@@@@MEAA@XZ 0000000180019018     Brackets.obj
 0003:00000024       $pdata$1$??1?$DialogBuilderBase@UFarDialogItem@@@@MEAA@XZ 0000000180019024     Brackets.obj
 0003:00000078       $pdata$?AddButtons@?$DialogBuilderBase@UFarDialogItem@@@@QEAAXHPEBHHH@Z 0000000180019078     Brackets.obj
 0003:00000084       $pdata$4$?AddButtons@?$DialogBuilderBase@UFarDialogItem@@@@QEAAXHPEBHHH@Z 0000000180019084     Brackets.obj
 0003:00000090       $pdata$5$?AddButtons@?$DialogBuilderBase@UFarDialogItem@@@@QEAAXHPEBHHH@Z 0000000180019090     Brackets.obj
 0003:00000030       $pdata$??_G?$DialogBuilderBase@UFarDialogItem@@@@MEAAPEAXI@Z 0000000180019030     Brackets.obj
 0003:000000f0       $pdata$?InitDialogItem@PluginDialogBuilder@@MEAAXPEAUFarDialogItem@@PEB_W@Z 00000001800190f0     Brackets.obj
 0003:000000e4       $pdata$?DoShowDialog@PluginDialogBuilder@@MEAA_JXZ 00000001800190e4     Brackets.obj
 0003:000000cc       $pdata$?CreateCheckBoxBinding@PluginDialogBuilder@@MEAAPEAU?$DialogItemBinding@UFarDialogItem@@@@PEAHH@Z 00000001800190cc     Brackets.obj
 0003:000000d8       $pdata$?CreateRadioButtonBinding@PluginDialogBuilder@@MEAAPEAU?$DialogItemBinding@UFarDialogItem@@@@PEAH@Z 00000001800190d8     Brackets.obj
 0003:000000a8       $pdata$?AddIntEditField@PluginDialogBuilder@@UEAAPEAUFarDialogItem@@PEAHH@Z 00000001800190a8     Brackets.obj
 0003:000000b4       $pdata$?AddUIntEditField@PluginDialogBuilder@@UEAAPEAUFarDialogItem@@PEAIH@Z 00000001800190b4     Brackets.obj
 0003:00000054       $pdata$??_GPluginDialogBuilder@@UEAAPEAXI@Z 0000000180019054     Brackets.obj
 0003:000000c0       $pdata$?Config@@YAHXZ      00000001800190c0     Brackets.obj
 0003:00000138       $pdata$?ShowMenu@@YAHH@Z   0000000180019138     Brackets.obj
 0003:000001bc       $pdata$??2@YAPEAX_K@Z      00000001800191bc     LIBCMT:new_scalar.obj
 0003:000001d4       $pdata$?dllmain_crt_process_attach@@YAHQEAUHINSTANCE__@@QEAX@Z 00000001800191d4     LIBCMT:dll_dllmain.obj
 0003:00000dc8       $pdata$?fin$0@?0??dllmain_crt_process_attach@@YAHQEAUHINSTANCE__@@QEAX@Z@4HA 0000000180019dc8     LIBCMT:dll_dllmain.obj
 0003:000001e0       $pdata$?dllmain_crt_process_detach@@YAH_N@Z 00000001800191e0     LIBCMT:dll_dllmain.obj
 0003:00000dd4       $pdata$?fin$0@?0??dllmain_crt_process_detach@@YAH_N@Z@4HA 0000000180019dd4     LIBCMT:dll_dllmain.obj
 0003:000001c8       $pdata$?dllmain_crt_dispatch@@YAHQEAUHINSTANCE__@@KQEAX@Z 00000001800191c8     LIBCMT:dll_dllmain.obj
 0003:000001ec       $pdata$?dllmain_dispatch@@YAHQEAUHINSTANCE__@@KQEAX@Z 00000001800191ec     LIBCMT:dll_dllmain.obj
 0003:00000de0       $pdata$?filt$0@?0??dllmain_dispatch@@YAHQEAUHINSTANCE__@@KQEAX@Z@4HA 0000000180019de0     LIBCMT:dll_dllmain.obj
 0003:000001f8       $pdata$_DllMainCRTStartup  00000001800191f8     LIBCMT:dll_dllmain.obj
 0003:0000021c       $pdata$??0exception@std@@QEAA@AEBV01@@Z 000000018001921c     LIBCMT:throw_bad_alloc.obj
 0003:00000228       $pdata$??_Gbad_alloc@std@@UEAAPEAXI@Z 0000000180019228     LIBCMT:throw_bad_alloc.obj
 0003:00000228       $pdata$??_Gexception@std@@UEAAPEAXI@Z 0000000180019228     LIBCMT:throw_bad_alloc.obj
 0003:00000228       $pdata$??_Gbad_array_new_length@std@@UEAAPEAXI@Z 0000000180019228     LIBCMT:throw_bad_alloc.obj
 0003:00000204       $pdata$??0bad_alloc@std@@QEAA@AEBV01@@Z 0000000180019204     LIBCMT:throw_bad_alloc.obj
 0003:00000210       $pdata$??0bad_array_new_length@std@@QEAA@AEBV01@@Z 0000000180019210     LIBCMT:throw_bad_alloc.obj
 0003:00000234       $pdata$?__scrt_throw_std_bad_alloc@@YAXXZ 0000000180019234     LIBCMT:throw_bad_alloc.obj
 0003:00000240       $pdata$?__scrt_throw_std_bad_array_new_length@@YAXXZ 0000000180019240     LIBCMT:throw_bad_alloc.obj
 0003:0000024c       $pdata$__security_init_cookie 000000018001924c     LIBCMT:gs_support.obj
 0003:00000258       $pdata$__scrt_initialize_default_local_stdio_options 0000000180019258     LIBCMT:default_local_stdio_options.obj
 0003:000002dc       $pdata$__scrt_is_nonwritable_in_current_image 00000001800192dc     LIBCMT:utility.obj
 0003:00000dec       $pdata$__scrt_is_nonwritable_in_current_image$filt$0 0000000180019dec     LIBCMT:utility.obj
 0003:00000264       $pdata$__scrt_acquire_startup_lock 0000000180019264     LIBCMT:utility.obj
 0003:000002e8       $pdata$__scrt_release_startup_lock 00000001800192e8     LIBCMT:utility.obj
 0003:000002c4       $pdata$__scrt_initialize_crt 00000001800192c4     LIBCMT:utility.obj
 0003:000002f4       $pdata$__scrt_uninitialize_crt 00000001800192f4     LIBCMT:utility.obj
 0003:000002d0       $pdata$__scrt_initialize_onexit_tables 00000001800192d0     LIBCMT:utility.obj
 0003:000002a0       $pdata$__scrt_dllmain_exception_filter 00000001800192a0     LIBCMT:utility.obj
 0003:0000027c       $pdata$__scrt_dllmain_before_initialize_c 000000018001927c     LIBCMT:utility.obj
 0003:00000270       $pdata$__scrt_dllmain_after_initialize_c 0000000180019270     LIBCMT:utility.obj
 0003:000002ac       $pdata$__scrt_dllmain_uninitialize_c 00000001800192ac     LIBCMT:utility.obj
 0003:000002b8       $pdata$__scrt_dllmain_uninitialize_critical 00000001800192b8     LIBCMT:utility.obj
 0003:00000288       $pdata$__scrt_dllmain_crt_thread_attach 0000000180019288     LIBCMT:utility.obj
 0003:00000294       $pdata$__scrt_dllmain_crt_thread_detach 0000000180019294     LIBCMT:utility.obj
 0003:00000300       $pdata$__scrt_fastfail     0000000180019300     LIBCMT:utility_desktop.obj
 0003:0000030c       $pdata$_RTC_Initialize     000000018001930c     LIBCMT:_initsect_.obj
 0003:00000318       $pdata$_RTC_Terminate      0000000180019318     LIBCMT:_initsect_.obj
 0003:00000324       $pdata$??_Gtype_info@@UEAAPEAXI@Z 0000000180019324     LIBCMT:std_type_info_static.obj
 0003:00000330       $pdata$__isa_available_init 0000000180019330     LIBCMT:_cpu_disp_.obj
 0003:00000348       $pdata$__C_specific_handler 0000000180019348     libvcruntime:_riscchandler_.obj
 0003:00000354       $pdata$__std_exception_copy 0000000180019354     libvcruntime:std_exception.obj
 0003:00000360       $pdata$__std_exception_destroy 0000000180019360     libvcruntime:std_exception.obj
 0003:0000036c       $pdata$_CxxThrowException  000000018001936c     libvcruntime:throw.obj
 0003:00000378       $pdata$__std_type_info_destroy_list 0000000180019378     libvcruntime:std_type_info.obj
 0003:00000384       $pdata$__vcrt_initialize   0000000180019384     libvcruntime:initialization.obj
 0003:000003a8       $pdata$__vcrt_uninitialize 00000001800193a8     libvcruntime:initialization.obj
 0003:000003b4       $pdata$__vcrt_uninitialize_critical 00000001800193b4     libvcruntime:initialization.obj
 0003:00000390       $pdata$__vcrt_thread_attach 0000000180019390     libvcruntime:initialization.obj
 0003:0000039c       $pdata$__vcrt_thread_detach 000000018001939c     libvcruntime:initialization.obj
 0003:00000414       $pdata$__vcrt_initialize_ptd 0000000180019414     libvcruntime:per_thread_data.obj
 0003:00000420       $pdata$__vcrt_uninitialize_ptd 0000000180019420     libvcruntime:per_thread_data.obj
 0003:00000408       $pdata$__vcrt_getptd_noexit 0000000180019408     libvcruntime:per_thread_data.obj
 0003:000003fc       $pdata$__vcrt_freeptd      00000001800193fc     libvcruntime:per_thread_data.obj
 0003:000003f0       $pdata$__vcrt_freefls      00000001800193f0     libvcruntime:per_thread_data.obj
 0003:0000042c       $pdata$__vcrt_initialize_locks 000000018001942c     libvcruntime:locks.obj
 0003:00000438       $pdata$__vcrt_uninitialize_locks 0000000180019438     libvcruntime:locks.obj
 0003:00000450       $pdata$__vcrt_FlsAlloc     0000000180019450     libvcruntime:winapi_downlevel.obj
 0003:0000045c       $pdata$__vcrt_FlsFree      000000018001945c     libvcruntime:winapi_downlevel.obj
 0003:00000468       $pdata$__vcrt_FlsGetValue  0000000180019468     libvcruntime:winapi_downlevel.obj
 0003:00000474       $pdata$__vcrt_FlsSetValue  0000000180019474     libvcruntime:winapi_downlevel.obj
 0003:00000480       $pdata$__vcrt_InitializeCriticalSectionEx 0000000180019480     libvcruntime:winapi_downlevel.obj
 0003:0000048c       $pdata$__vcrt_initialize_winapi_thunks 000000018001948c     libvcruntime:winapi_downlevel.obj
 0003:00000498       $pdata$__vcrt_uninitialize_winapi_thunks 0000000180019498     libvcruntime:winapi_downlevel.obj
 0003:00000444       $pdata$?try_get_function@@YAPEAXW4function_id@?A0x89697e75@@QEBDQEBW4module_id@2@2@Z 0000000180019444     libvcruntime:winapi_downlevel.obj
 0003:000004bc       $pdata$__DestructExceptionObject 00000001800194bc     libvcruntime:ehhelpers.obj
 0003:00000df8       $pdata$__DestructExceptionObject$filt$0 0000000180019df8     libvcruntime:ehhelpers.obj
 0003:000004c8       $pdata$_callnewh           00000001800194c8     libucrt:new_handler.obj
 0003:000004d4       $pdata$_query_new_handler  00000001800194d4     libucrt:new_handler.obj
 0003:00000e04       $pdata$_query_new_handler$fin$0 0000000180019e04     libucrt:new_handler.obj
 0003:000004e0       $pdata$_initterm           00000001800194e0     libucrt:initterm.obj
 0003:000004ec       $pdata$_initterm_e         00000001800194ec     libucrt:initterm.obj
 0003:000004f8       $pdata$_seh_filter_exe     00000001800194f8     libucrt:exception_filter.obj
 0003:00000534       $pdata$?try_cor_exit_process@@YAXI@Z 0000000180019534     libucrt:exit.obj
 0003:00000528       $pdata$?exit_or_terminate_process@@YAXI@Z 0000000180019528     libucrt:exit.obj
 0003:0000051c       $pdata$?common_exit@@YAXHW4_crt_exit_cleanup_mode@@W4_crt_exit_return_mode@@@Z 000000018001951c     libucrt:exit.obj
 0003:00000510       $pdata$??R<lambda_6e4b09c48022b2350581041d5f6b0c4c>@@QEBA@XZ 0000000180019510     libucrt:exit.obj
 0003:00000e1c       $pdata$?filt$0@?0???R<lambda_6e4b09c48022b2350581041d5f6b0c4c>@@QEBA@XZ@4HA 0000000180019e1c     libucrt:exit.obj
 0003:00000504       $pdata$??$?RV<lambda_d80eeec6fff315bfe5c115232f3240e3>@@AEAV<lambda_6e4b09c48022b2350581041d5f6b0c4c>@@V<lambda_2358e3775559c9db80273638284d5e45>@@@?$__crt_seh_guarded_call@X@@QEAAX$$QEAV<lambda_d80eeec6fff315bfe5c115232f3240e3>@@AEAV<lambda_6e4b09c48022b2350581041d5f6b0c4c>@@$$QEAV<lambda_2358e3775559c9db80273638284d5e45>@@@Z 0000000180019504     libucrt:exit.obj
 0003:00000e10       $pdata$?fin$0@?0???$?RV<lambda_f2e299630e499de9f9a165e60fcd3db5>@@AEAV<lambda_2ae9d31cdba2644fcbeaf08da7c24588>@@V<lambda_40d01ff24d0e7b3814fdbdcee8eab3c7>@@@?$__crt_seh_guarded_call@X@@QEAAX$$QEAV<lambda_f2e299630e499de9f9a165e60fcd3db5>@@AEAV<lambda_2ae9d31cdba2644fcbeaf08da7c24588>@@$$QEAV<lambda_40d01ff24d0e7b3814fdbdcee8eab3c7>@@@Z@4HA 0000000180019e10     libucrt:per_thread_data.obj
 0003:00000e10       $pdata$?fin$0@?0???$?RV<lambda_7777bce6b2f8c936911f934f8298dc43>@@AEAV<lambda_f03950bc5685219e0bcd2087efbe011e>@@V<lambda_3883c3dff614d5e0c5f61bb1ac94921c>@@@?$__crt_seh_guarded_call@H@@QEAAH$$QEAV<lambda_7777bce6b2f8c936911f934f8298dc43>@@AEAV<lambda_f03950bc5685219e0bcd2087efbe011e>@@$$QEAV<lambda_3883c3dff614d5e0c5f61bb1ac94921c>@@@Z@4HA 0000000180019e10     libucrt:onexit.obj
 0003:00000e10       $pdata$?fin$0@?0???$?RV<lambda_d80eeec6fff315bfe5c115232f3240e3>@@AEAV<lambda_6e4b09c48022b2350581041d5f6b0c4c>@@V<lambda_2358e3775559c9db80273638284d5e45>@@@?$__crt_seh_guarded_call@X@@QEAAX$$QEAV<lambda_d80eeec6fff315bfe5c115232f3240e3>@@AEAV<lambda_6e4b09c48022b2350581041d5f6b0c4c>@@$$QEAV<lambda_2358e3775559c9db80273638284d5e45>@@@Z@4HA 0000000180019e10     libucrt:exit.obj
 0003:00000e10       $pdata$?fin$0@?0???$?RV<lambda_450d765d439847d4c735a33c368b5fc0>@@AEAV<lambda_44731a7d0e6d81c3e6aa82d741081786>@@V<lambda_601a2a7da3b7a96e9554ac7215c4b07c>@@@?$__crt_seh_guarded_call@P6AXH@Z@@QEAAP6AXH@Z$$QEAV<lambda_450d765d439847d4c735a33c368b5fc0>@@AEAV<lambda_44731a7d0e6d81c3e6aa82d741081786>@@$$QEAV<lambda_601a2a7da3b7a96e9554ac7215c4b07c>@@@Z@4HA 0000000180019e10     libucrt:signal.obj
 0003:00000e10       $pdata$?fin$0@?0???$?RV<lambda_aa87e3671a710a21b5dc78c0bdf72e11>@@AEAV<lambda_92619d2358a28f41a33ba319515a20b9>@@V<lambda_6992ecaafeb10aed2b74cb1fae11a551>@@@?$__crt_seh_guarded_call@X@@QEAAX$$QEAV<lambda_aa87e3671a710a21b5dc78c0bdf72e11>@@AEAV<lambda_92619d2358a28f41a33ba319515a20b9>@@$$QEAV<lambda_6992ecaafeb10aed2b74cb1fae11a551>@@@Z@4HA 0000000180019e10     libucrt:per_thread_data.obj
 0003:00000e10       $pdata$?fin$0@?0???$?RV<lambda_0ae27a3a962d80f24befdcbee591983d>@@AEAV<lambda_8d0ee55de4b1038c4002e0adecdf1839>@@V<lambda_dc504788e8f1664fe9b84e20bfb512f2>@@@?$__crt_seh_guarded_call@X@@QEAAX$$QEAV<lambda_0ae27a3a962d80f24befdcbee591983d>@@AEAV<lambda_8d0ee55de4b1038c4002e0adecdf1839>@@$$QEAV<lambda_dc504788e8f1664fe9b84e20bfb512f2>@@@Z@4HA 0000000180019e10     libucrt:per_thread_data.obj
 0003:00000e10       $pdata$?fin$0@?0???$?RV<lambda_efdfa57d1f175319df784efa44bb7b81>@@AEAV<lambda_5f0a4c1567f8adc6734073e5d1e1b35c>@@V<lambda_2e8a7d3640ea6ccb4c2413664c2db6fd>@@@?$__crt_seh_guarded_call@X@@QEAAX$$QEAV<lambda_efdfa57d1f175319df784efa44bb7b81>@@AEAV<lambda_5f0a4c1567f8adc6734073e5d1e1b35c>@@$$QEAV<lambda_2e8a7d3640ea6ccb4c2413664c2db6fd>@@@Z@4HA 0000000180019e10     libucrt:mbctype.obj
 0003:00000e10       $pdata$?fin$0@?0???$?RV<lambda_2d41944a1d46af3157314b8a01080d33>@@AEAV<lambda_8f455de75cd7d7f24b4096f044d8b9e6>@@V<lambda_aa500f224e6afead328df44964fe2772>@@@?$__crt_seh_guarded_call@X@@QEAAX$$QEAV<lambda_2d41944a1d46af3157314b8a01080d33>@@AEAV<lambda_8f455de75cd7d7f24b4096f044d8b9e6>@@$$QEAV<lambda_aa500f224e6afead328df44964fe2772>@@@Z@4HA 0000000180019e10     libucrt:per_thread_data.obj
 0003:00000558       $pdata$_configure_narrow_argv 0000000180019558     libucrt:argv_parsing.obj
 0003:0000054c       $pdata$__acrt_allocate_buffer_for_argv 000000018001954c     libucrt:argv_parsing.obj
 0003:00000540       $pdata$??$parse_command_line@D@@YAXPEADPEAPEAD0PEA_K2@Z 0000000180019540     libucrt:argv_parsing.obj
 0003:000005a0       $pdata$__dcrt_uninitialize_environments_nolock 00000001800195a0     libucrt:environment_initialization.obj
 0003:00000564       $pdata$??$common_initialize_environment_nolock@D@@YAHXZ 0000000180019564     libucrt:environment_initialization.obj
 0003:00000588       $pdata$??$uninitialize_environment_internal@D@@YAXAEAPEAPEAD@Z 0000000180019588     libucrt:environment_initialization.obj
 0003:00000594       $pdata$??$uninitialize_environment_internal@_W@@YAXAEAPEAPEA_W@Z 0000000180019594     libucrt:environment_initialization.obj
 0003:0000057c       $pdata$??$free_environment@D@@YAXQEAPEAD@Z 000000018001957c     libucrt:environment_initialization.obj
 0003:0000057c       $pdata$??$free_environment@_W@@YAXQEAPEA_W@Z 000000018001957c     libucrt:environment_initialization.obj
 0003:00000570       $pdata$??$create_environment@D@@YAQEAPEADQEAD@Z 0000000180019570     libucrt:environment_initialization.obj
 0003:000005c4       $pdata$_execute_onexit_table 00000001800195c4     libucrt:onexit.obj
 0003:000005b8       $pdata$??R<lambda_f03950bc5685219e0bcd2087efbe011e>@@QEBAHXZ 00000001800195b8     libucrt:onexit.obj
 0003:000005ac       $pdata$??$?RV<lambda_7777bce6b2f8c936911f934f8298dc43>@@AEAV<lambda_f03950bc5685219e0bcd2087efbe011e>@@V<lambda_3883c3dff614d5e0c5f61bb1ac94921c>@@@?$__crt_seh_guarded_call@H@@QEAAH$$QEAV<lambda_7777bce6b2f8c936911f934f8298dc43>@@AEAV<lambda_f03950bc5685219e0bcd2087efbe011e>@@$$QEAV<lambda_3883c3dff614d5e0c5f61bb1ac94921c>@@@Z 00000001800195ac     libucrt:onexit.obj
 0003:00000624       $pdata$__acrt_uninitialize 0000000180019624     libucrt:initialization.obj
 0003:00000630       $pdata$__acrt_uninitialize_critical 0000000180019630     libucrt:initialization.obj
 0003:0000060c       $pdata$__acrt_thread_attach 000000018001960c     libucrt:initialization.obj
 0003:00000618       $pdata$__acrt_thread_detach 0000000180019618     libucrt:initialization.obj
 0003:000005d0       $pdata$initialize_c        00000001800195d0     libucrt:initialization.obj
 0003:000005dc       $pdata$uninitialize_environment 00000001800195dc     libucrt:initialization.obj
 0003:000005e8       $pdata$initialize_pointers 00000001800195e8     libucrt:initialization.obj
 0003:000005f4       $pdata$uninitialize_allocated_memory 00000001800195f4     libucrt:initialization.obj
 0003:00000600       $pdata$uninitialize_allocated_io_buffers 0000000180019600     libucrt:initialization.obj
 0003:0000063c       $pdata$terminate           000000018001963c     libucrt:terminate.obj
 0003:00000648       $pdata$strcpy_s            0000000180019648     libucrt:strcpy_s.obj
 0003:00000654       $pdata$??0_LocaleUpdate@@QEAA@QEAU__crt_locale_pointers@@@Z 0000000180019654     libucrt:output.obj
 0003:0000066c       $pdata$abort               000000018001966c     libucrt:abort.obj
 0003:00000678       $pdata$__acrt_initialize_locks 0000000180019678     libucrt:locks.obj
 0003:00000684       $pdata$__acrt_uninitialize_locks 0000000180019684     libucrt:locks.obj
 0003:00000690       $pdata$_malloc_base        0000000180019690     libucrt:malloc_base.obj
 0003:0000069c       $pdata$_free_base          000000018001969c     libucrt:free_base.obj
 0003:00000738       $pdata$__acrt_initialize_ptd 0000000180019738     libucrt:per_thread_data.obj
 0003:00000744       $pdata$__acrt_uninitialize_ptd 0000000180019744     libucrt:per_thread_data.obj
 0003:00000714       $pdata$__acrt_getptd       0000000180019714     libucrt:per_thread_data.obj
 0003:00000720       $pdata$__acrt_getptd_head  0000000180019720     libucrt:per_thread_data.obj
 0003:0000072c       $pdata$__acrt_getptd_noexit 000000018001972c     libucrt:per_thread_data.obj
 0003:00000708       $pdata$__acrt_freeptd      0000000180019708     libucrt:per_thread_data.obj
 0003:000006e4       $pdata$?destroy_fls@@YAXPEAX@Z 00000001800196e4     libucrt:per_thread_data.obj
 0003:000006fc       $pdata$?replace_current_thread_locale_nolock@@YAXQEAU__acrt_ptd@@QEAU__crt_locale_data@@@Z 00000001800196fc     libucrt:per_thread_data.obj
 0003:000006d8       $pdata$?construct_ptd_array@@YAXQEAU__acrt_ptd@@@Z 00000001800196d8     libucrt:per_thread_data.obj
 0003:000006f0       $pdata$?destroy_ptd_array@@YAXQEAU__acrt_ptd@@@Z 00000001800196f0     libucrt:per_thread_data.obj
 0003:000006a8       $pdata$??$?RV<lambda_0ae27a3a962d80f24befdcbee591983d>@@AEAV<lambda_8d0ee55de4b1038c4002e0adecdf1839>@@V<lambda_dc504788e8f1664fe9b84e20bfb512f2>@@@?$__crt_seh_guarded_call@X@@QEAAX$$QEAV<lambda_0ae27a3a962d80f24befdcbee591983d>@@AEAV<lambda_8d0ee55de4b1038c4002e0adecdf1839>@@$$QEAV<lambda_dc504788e8f1664fe9b84e20bfb512f2>@@@Z 00000001800196a8     libucrt:per_thread_data.obj
 0003:000006c0       $pdata$??$?RV<lambda_aa87e3671a710a21b5dc78c0bdf72e11>@@AEAV<lambda_92619d2358a28f41a33ba319515a20b9>@@V<lambda_6992ecaafeb10aed2b74cb1fae11a551>@@@?$__crt_seh_guarded_call@X@@QEAAX$$QEAV<lambda_aa87e3671a710a21b5dc78c0bdf72e11>@@AEAV<lambda_92619d2358a28f41a33ba319515a20b9>@@$$QEAV<lambda_6992ecaafeb10aed2b74cb1fae11a551>@@@Z 00000001800196c0     libucrt:per_thread_data.obj
 0003:000006cc       $pdata$??$?RV<lambda_f2e299630e499de9f9a165e60fcd3db5>@@AEAV<lambda_2ae9d31cdba2644fcbeaf08da7c24588>@@V<lambda_40d01ff24d0e7b3814fdbdcee8eab3c7>@@@?$__crt_seh_guarded_call@X@@QEAAX$$QEAV<lambda_f2e299630e499de9f9a165e60fcd3db5>@@AEAV<lambda_2ae9d31cdba2644fcbeaf08da7c24588>@@$$QEAV<lambda_40d01ff24d0e7b3814fdbdcee8eab3c7>@@@Z 00000001800196cc     libucrt:per_thread_data.obj
 0003:000006b4       $pdata$??$?RV<lambda_2d41944a1d46af3157314b8a01080d33>@@AEAV<lambda_8f455de75cd7d7f24b4096f044d8b9e6>@@V<lambda_aa500f224e6afead328df44964fe2772>@@@?$__crt_seh_guarded_call@X@@QEAAX$$QEAV<lambda_2d41944a1d46af3157314b8a01080d33>@@AEAV<lambda_8f455de75cd7d7f24b4096f044d8b9e6>@@$$QEAV<lambda_aa500f224e6afead328df44964fe2772>@@@Z 00000001800196b4     libucrt:per_thread_data.obj
 0003:00000750       $pdata$__acrt_get_process_end_policy 0000000180019750     libucrt:win_policies.obj
 0003:00000774       $pdata$_invalid_parameter_noinfo 0000000180019774     libucrt:invalid_parameter.obj
 0003:00000780       $pdata$_invoke_watson      0000000180019780     libucrt:invalid_parameter.obj
 0003:0000075c       $pdata$__acrt_call_reportfault 000000018001975c     libucrt:invalid_parameter.obj
 0003:00000768       $pdata$_invalid_parameter  0000000180019768     libucrt:invalid_parameter.obj
 0003:000007a4       $pdata$_errno              00000001800197a4     libucrt:errno.obj
 0003:00000798       $pdata$__doserrno          0000000180019798     libucrt:errno.obj
 0003:0000078c       $pdata$__acrt_errno_map_os_error 000000018001978c     libucrt:errno.obj
 0003:000007b0       $pdata$_calloc_base        00000001800197b0     libucrt:calloc_base.obj
 0003:000007bc       $pdata$??$common_expand_argv_wildcards@D@@YAHQEAPEADQEAPEAPEAD@Z 00000001800197bc     libucrt:argv_wildcards.obj
 0003:000007c8       $pdata$??$copy_and_add_argument_to_buffer@D@@YAHQEBD0_KAEAV?$argument_list@D@?A0x5f5c8891@@@Z 00000001800197c8     libucrt:argv_wildcards.obj
 0003:000007d4       $pdata$??$expand_argument_wildcards@D@@YAHQEAD0AEAV?$argument_list@D@?A0x5f5c8891@@@Z 00000001800197d4     libucrt:argv_wildcards.obj
 0003:00000834       $pdata$__acrt_update_thread_multibyte_data 0000000180019834     libucrt:mbctype.obj
 0003:00000828       $pdata$__acrt_initialize_multibyte 0000000180019828     libucrt:mbctype.obj
 0003:00000840       $pdata$_setmbcp_nolock     0000000180019840     libucrt:mbctype.obj
 0003:000007ec       $pdata$?getSystemCP@@YAHH@Z 00000001800197ec     libucrt:mbctype.obj
 0003:000007f8       $pdata$?setSBCS@@YAXPEAU__crt_multibyte_data@@@Z 00000001800197f8     libucrt:mbctype.obj
 0003:0000081c       $pdata$?update_thread_multibyte_data_internal@@YAPEAU__crt_multibyte_data@@QEAU__acrt_ptd@@QEAPEAU1@@Z 000000018001981c     libucrt:mbctype.obj
 0003:00000e28       $pdata$?fin$0@?0??update_thread_multibyte_data_internal@@YAPEAU__crt_multibyte_data@@QEAU__acrt_ptd@@QEAPEAU1@@Z@4HA 0000000180019e28     libucrt:mbctype.obj
 0003:00000810       $pdata$?setmbcp_internal@@YAHH_NQEAU__acrt_ptd@@QEAPEAU__crt_multibyte_data@@@Z 0000000180019810     libucrt:mbctype.obj
 0003:00000804       $pdata$?setSBUpLow@@YAXPEAU__crt_multibyte_data@@@Z 0000000180019804     libucrt:mbctype.obj
 0003:000007e0       $pdata$??$?RV<lambda_efdfa57d1f175319df784efa44bb7b81>@@AEAV<lambda_5f0a4c1567f8adc6734073e5d1e1b35c>@@V<lambda_2e8a7d3640ea6ccb4c2413664c2db6fd>@@@?$__crt_seh_guarded_call@X@@QEAAX$$QEAV<lambda_efdfa57d1f175319df784efa44bb7b81>@@AEAV<lambda_5f0a4c1567f8adc6734073e5d1e1b35c>@@$$QEAV<lambda_2e8a7d3640ea6ccb4c2413664c2db6fd>@@@Z 00000001800197e0     libucrt:mbctype.obj
 0003:0000084c       $pdata$?x_ismbbtype_l@@YAHPEAU__crt_locale_pointers@@IHH@Z 000000018001984c     libucrt:ismbbyte.obj
 0003:00000858       $pdata$__acrt_initialize_command_line 0000000180019858     libucrt:argv_data.obj
 0003:00000864       $pdata$__dcrt_get_narrow_environment_from_os 0000000180019864     libucrt:get_environment_from_os.obj
 0003:00000870       $pdata$_recalloc_base      0000000180019870     libucrt:recalloc.obj
 0003:000008e8       $pdata$__acrt_initialize_winapi_thunks 00000001800198e8     libucrt:winapi_thunks.obj
 0003:000008f4       $pdata$__acrt_uninitialize_winapi_thunks 00000001800198f4     libucrt:winapi_thunks.obj
 0003:00000894       $pdata$__acrt_FlsAlloc     0000000180019894     libucrt:winapi_thunks.obj
 0003:000008a0       $pdata$__acrt_FlsFree      00000001800198a0     libucrt:winapi_thunks.obj
 0003:000008ac       $pdata$__acrt_FlsGetValue  00000001800198ac     libucrt:winapi_thunks.obj
 0003:000008b8       $pdata$__acrt_FlsSetValue  00000001800198b8     libucrt:winapi_thunks.obj
 0003:000008c4       $pdata$__acrt_InitializeCriticalSectionEx 00000001800198c4     libucrt:winapi_thunks.obj
 0003:000008d0       $pdata$__acrt_LCMapStringEx 00000001800198d0     libucrt:winapi_thunks.obj
 0003:000008dc       $pdata$__acrt_LocaleNameToLCID 00000001800198dc     libucrt:winapi_thunks.obj
 0003:00000888       $pdata$__acrt_AppPolicyGetProcessTerminationMethodInternal 0000000180019888     libucrt:winapi_thunks.obj
 0003:0000087c       $pdata$?try_get_function@@YAPEAXW4function_id@?A0x391cf84c@@QEBDQEBW4module_id@2@2@Z 000000018001987c     libucrt:winapi_thunks.obj
 0003:00000900       $pdata$__acrt_initialize_heap 0000000180019900     libucrt:heap_handle.obj
 0003:00000924       $pdata$__acrt_initialize_lowio 0000000180019924     libucrt:ioinit.obj
 0003:00000e34       $pdata$__acrt_lowio_ensure_fh_exists$fin$0 0000000180019e34     libucrt:osfinfo.obj
 0003:00000e34       $pdata$__acrt_initialize_lowio$fin$0 0000000180019e34     libucrt:ioinit.obj
 0003:00000930       $pdata$__acrt_uninitialize_lowio 0000000180019930     libucrt:ioinit.obj
 0003:0000090c       $pdata$?initialize_inherited_file_handles_nolock@@YAXXZ 000000018001990c     libucrt:ioinit.obj
 0003:00000918       $pdata$?initialize_stdio_handles_nolock@@YAXXZ 0000000180019918     libucrt:ioinit.obj
 0003:0000093c       $pdata$__acrt_execute_initializers 000000018001993c     libucrt:shared_initialization.obj
 0003:00000948       $pdata$__acrt_execute_uninitializers 0000000180019948     libucrt:shared_initialization.obj
 0003:00000960       $pdata$__acrt_get_sigabrt_handler 0000000180019960     libucrt:signal.obj
 0003:0000096c       $pdata$raise               000000018001996c     libucrt:signal.obj
 0003:00000e40       $pdata$raise$fin$0         0000000180019e40     libucrt:signal.obj
 0003:00000954       $pdata$??$?RV<lambda_450d765d439847d4c735a33c368b5fc0>@@AEAV<lambda_44731a7d0e6d81c3e6aa82d741081786>@@V<lambda_601a2a7da3b7a96e9554ac7215c4b07c>@@@?$__crt_seh_guarded_call@P6AXH@Z@@QEAAP6AXH@Z$$QEAV<lambda_450d765d439847d4c735a33c368b5fc0>@@AEAV<lambda_44731a7d0e6d81c3e6aa82d741081786>@@$$QEAV<lambda_601a2a7da3b7a96e9554ac7215c4b07c>@@@Z 0000000180019954     libucrt:signal.obj
 0003:000009a8       $pdata$_fflush_nolock      00000001800199a8     libucrt:fflush.obj
 0003:0000099c       $pdata$__acrt_stdio_flush_nolock 000000018001999c     libucrt:fflush.obj
 0003:00000990       $pdata$?common_flush_all@@YAH_N@Z 0000000180019990     libucrt:fflush.obj
 0003:00000978       $pdata$??$?RV<lambda_842d9ff0dc9ef11c61343bbaebe7f885>@@AEAV<lambda_c5860995281e5c4ce005b3de8f5874ee>@@V<lambda_d90129c13df834fdcbf8d2b88dafcf2d>@@@?$__crt_seh_guarded_call@X@@QEAAX$$QEAV<lambda_842d9ff0dc9ef11c61343bbaebe7f885>@@AEAV<lambda_c5860995281e5c4ce005b3de8f5874ee>@@$$QEAV<lambda_d90129c13df834fdcbf8d2b88dafcf2d>@@@Z 0000000180019978     libucrt:fflush.obj
 0003:00000e4c       $pdata$?fin$0@?0???$?RV<lambda_842d9ff0dc9ef11c61343bbaebe7f885>@@AEAV<lambda_c5860995281e5c4ce005b3de8f5874ee>@@V<lambda_d90129c13df834fdcbf8d2b88dafcf2d>@@@?$__crt_seh_guarded_call@X@@QEAAX$$QEAV<lambda_842d9ff0dc9ef11c61343bbaebe7f885>@@AEAV<lambda_c5860995281e5c4ce005b3de8f5874ee>@@$$QEAV<lambda_d90129c13df834fdcbf8d2b88dafcf2d>@@@Z@4HA 0000000180019e4c     libucrt:fflush.obj
 0003:00000984       $pdata$??$?RV<lambda_886d6c58226a84441f68b9f2b8217b83>@@AEAV<lambda_ab61a845afdef5b7c387490eaf3616ee>@@V<lambda_f7f22ab5edc0698d5f6905b0d3f44752>@@@?$__crt_seh_guarded_call@X@@QEAAX$$QEAV<lambda_886d6c58226a84441f68b9f2b8217b83>@@AEAV<lambda_ab61a845afdef5b7c387490eaf3616ee>@@$$QEAV<lambda_f7f22ab5edc0698d5f6905b0d3f44752>@@@Z 0000000180019984     libucrt:fflush.obj
 0003:00000e58       $pdata$?fin$0@?0???$?RV<lambda_886d6c58226a84441f68b9f2b8217b83>@@AEAV<lambda_ab61a845afdef5b7c387490eaf3616ee>@@V<lambda_f7f22ab5edc0698d5f6905b0d3f44752>@@@?$__crt_seh_guarded_call@X@@QEAAX$$QEAV<lambda_886d6c58226a84441f68b9f2b8217b83>@@AEAV<lambda_ab61a845afdef5b7c387490eaf3616ee>@@$$QEAV<lambda_f7f22ab5edc0698d5f6905b0d3f44752>@@@Z@4HA 0000000180019e58     libucrt:fflush.obj
 0003:000009b4       $pdata$__acrt_initialize_stdio 00000001800199b4     libucrt:_file.obj
 0003:000009c0       $pdata$__acrt_uninitialize_stdio 00000001800199c0     libucrt:_file.obj
 0003:000009cc       $pdata$_mbtowc_l           00000001800199cc     libucrt:mbtowc.obj
 0003:000009d8       $pdata$__acrt_update_locale_info 00000001800199d8     libucrt:locale_update.obj
 0003:000009e4       $pdata$__acrt_update_multibyte_info 00000001800199e4     libucrt:locale_update.obj
 0003:000009f0       $pdata$_fileno             00000001800199f0     libucrt:fileno.obj
 0003:00000a08       $pdata$__acrt_uninitialize_locale 0000000180019a08     libucrt:wsetlocale.obj
 0003:000009fc       $pdata$??$?RV<lambda_410d79af7f07d98d83a3f525b3859a53>@@AEAV<lambda_3e16ef9562a7dcce91392c22ab16ea36>@@V<lambda_38119f0e861e05405d8a144b9b982f0a>@@@?$__crt_seh_guarded_call@X@@QEAAX$$QEAV<lambda_410d79af7f07d98d83a3f525b3859a53>@@AEAV<lambda_3e16ef9562a7dcce91392c22ab16ea36>@@$$QEAV<lambda_38119f0e861e05405d8a144b9b982f0a>@@@Z 00000001800199fc     libucrt:wsetlocale.obj
 0003:00000e64       $pdata$?fin$0@?0???$?RV<lambda_410d79af7f07d98d83a3f525b3859a53>@@AEAV<lambda_3e16ef9562a7dcce91392c22ab16ea36>@@V<lambda_38119f0e861e05405d8a144b9b982f0a>@@@?$__crt_seh_guarded_call@X@@QEAAX$$QEAV<lambda_410d79af7f07d98d83a3f525b3859a53>@@AEAV<lambda_3e16ef9562a7dcce91392c22ab16ea36>@@$$QEAV<lambda_38119f0e861e05405d8a144b9b982f0a>@@@Z@4HA 0000000180019e64     libucrt:wsetlocale.obj
 0003:00000a14       $pdata$__pctype_func       0000000180019a14     libucrt:ctype.obj
 0003:00000a38       $pdata$__acrt_release_locale_ref 0000000180019a38     libucrt:locale_refcounting.obj
 0003:00000a20       $pdata$__acrt_free_locale  0000000180019a20     libucrt:locale_refcounting.obj
 0003:00000a2c       $pdata$__acrt_locale_free_lc_time_if_unreferenced 0000000180019a2c     libucrt:locale_refcounting.obj
 0003:00000a44       $pdata$__acrt_update_thread_locale_data 0000000180019a44     libucrt:locale_refcounting.obj
 0003:00000e70       $pdata$__acrt_update_thread_locale_data$fin$0 0000000180019e70     libucrt:locale_refcounting.obj
 0003:00000a50       $pdata$_updatetlocinfoEx_nolock 0000000180019a50     libucrt:locale_refcounting.obj
 0003:00000a5c       $pdata$qsort               0000000180019a5c     libucrt:qsort.obj
 0003:00000a68       $pdata$4$qsort             0000000180019a68     libucrt:qsort.obj
 0003:00000a74       $pdata$5$qsort             0000000180019a74     libucrt:qsort.obj
 0003:00000a80       $pdata$strncpy_s           0000000180019a80     libucrt:strncpy_s.obj
 0003:00000a98       $pdata$strpbrk             0000000180019a98     libucrt:strpbrk.obj
 0003:00000a8c       $pdata$fallbackMethod      0000000180019a8c     libucrt:strpbrk.obj
 0003:00000aa4       $pdata$_mbsdec_l           0000000180019aa4     libucrt:mbsdec.obj
 0003:00000ab0       $pdata$?initialize_multibyte@@YAHXZ 0000000180019ab0     libucrt:multibyte_initializer.obj
 0003:00000abc       $pdata$__acrt_GetStringTypeA 0000000180019abc     libucrt:getstringtypea.obj
 0003:00000ad4       $pdata$__acrt_LCMapStringA 0000000180019ad4     libucrt:lcmapstringa.obj
 0003:00000ac8       $pdata$?__acrt_LCMapStringA_stat@@YAHPEAU__crt_locale_pointers@@PEB_WKPEBDHPEADHHH@Z 0000000180019ac8     libucrt:lcmapstringa.obj
 0003:00000ae0       $pdata$_msize_base         0000000180019ae0     libucrt:msize.obj
 0003:00000aec       $pdata$_realloc_base       0000000180019aec     libucrt:realloc_base.obj
 0003:00000b04       $pdata$__acrt_DownlevelLocaleNameToLCID 0000000180019b04     libucrt:lcidtoname_downlevel.obj
 0003:00000af8       $pdata$?GetTableIndexFromLocaleName@@YAHPEB_W@Z 0000000180019af8     libucrt:lcidtoname_downlevel.obj
 0003:00000b40       $pdata$_get_osfhandle      0000000180019b40     libucrt:osfinfo.obj
 0003:00000b34       $pdata$_free_osfhnd        0000000180019b34     libucrt:osfinfo.obj
 0003:00000b10       $pdata$__acrt_lowio_create_handle_array 0000000180019b10     libucrt:osfinfo.obj
 0003:00000b1c       $pdata$__acrt_lowio_destroy_handle_array 0000000180019b1c     libucrt:osfinfo.obj
 0003:00000b28       $pdata$__acrt_lowio_ensure_fh_exists 0000000180019b28     libucrt:osfinfo.obj
 0003:00000b58       $pdata$_commit             0000000180019b58     libucrt:commit.obj
 0003:00000b4c       $pdata$??$?RV<lambda_a37b2b86f63e897a80ea819b0eb08c01>@@AEAV<lambda_38ce7e780aa69e748d6df282ebc68efe>@@V<lambda_99fb1378e971ab6e7edea83e3a7a83a2>@@@?$__crt_seh_guarded_call@H@@QEAAH$$QEAV<lambda_a37b2b86f63e897a80ea819b0eb08c01>@@AEAV<lambda_38ce7e780aa69e748d6df282ebc68efe>@@$$QEAV<lambda_99fb1378e971ab6e7edea83e3a7a83a2>@@@Z 0000000180019b4c     libucrt:commit.obj
 0003:00000e7c       $pdata$?fin$0@?0???$?RV<lambda_751a882b2c74d4b022dec766aa51a29a>@@AEAV<lambda_628dfdc04ba53c8bfc02c9951375f3f5>@@V<lambda_f6c7be5f7998530c34de24c7437d6b54>@@@?$__crt_seh_guarded_call@H@@QEAAH$$QEAV<lambda_751a882b2c74d4b022dec766aa51a29a>@@AEAV<lambda_628dfdc04ba53c8bfc02c9951375f3f5>@@$$QEAV<lambda_f6c7be5f7998530c34de24c7437d6b54>@@@Z@4HA 0000000180019e7c     libucrt:close.obj
 0003:00000e7c       $pdata$?fin$0@?0???$?RV<lambda_a37b2b86f63e897a80ea819b0eb08c01>@@AEAV<lambda_38ce7e780aa69e748d6df282ebc68efe>@@V<lambda_99fb1378e971ab6e7edea83e3a7a83a2>@@@?$__crt_seh_guarded_call@H@@QEAAH$$QEAV<lambda_a37b2b86f63e897a80ea819b0eb08c01>@@AEAV<lambda_38ce7e780aa69e748d6df282ebc68efe>@@$$QEAV<lambda_99fb1378e971ab6e7edea83e3a7a83a2>@@@Z@4HA 0000000180019e7c     libucrt:commit.obj
 0003:00000b94       $pdata$_write              0000000180019b94     libucrt:write.obj
 0003:00000e88       $pdata$_write$fin$0        0000000180019e88     libucrt:write.obj
 0003:00000ba0       $pdata$_write_nolock       0000000180019ba0     libucrt:write.obj
 0003:00000b64       $pdata$?write_double_translated_ansi_nolock@@YA?AUwrite_result@?A0x17268360@@HQEBDI@Z 0000000180019b64     libucrt:write.obj
 0003:00000b70       $pdata$?write_text_ansi_nolock@@YA?AUwrite_result@?A0x17268360@@HQEBDI@Z 0000000180019b70     libucrt:write.obj
 0003:00000b7c       $pdata$?write_text_utf16le_nolock@@YA?AUwrite_result@?A0x17268360@@HQEBDI@Z 0000000180019b7c     libucrt:write.obj
 0003:00000b88       $pdata$?write_text_utf8_nolock@@YA?AUwrite_result@?A0x17268360@@HQEBDI@Z 0000000180019b88     libucrt:write.obj
 0003:00000bac       $pdata$_fcloseall          0000000180019bac     libucrt:closeall.obj
 0003:00000e94       $pdata$_fcloseall$fin$0    0000000180019e94     libucrt:closeall.obj
 0003:00000bb8       $pdata$__acrt_stdio_free_buffer_nolock 0000000180019bb8     libucrt:_freebuf.obj
 0003:00000bc4       $pdata$_isatty             0000000180019bc4     libucrt:isatty.obj
 0003:00000bd0       $pdata$_isleadbyte_l       0000000180019bd0     libucrt:_wctype.obj
 0003:00000bdc       $pdata$__acrt_locale_free_monetary 0000000180019bdc     libucrt:initmon.obj
 0003:00000be8       $pdata$__acrt_locale_free_numeric 0000000180019be8     libucrt:initnum.obj
 0003:00000c00       $pdata$__acrt_locale_free_time 0000000180019c00     libucrt:inittime.obj
 0003:00000bf4       $pdata$?free_crt_array_internal@@YAXQEAPEBX_K@Z 0000000180019bf4     libucrt:inittime.obj
 0003:00000c0c       $pdata$??$common_lseek_nolock@_J@@YA_JH_JH@Z 0000000180019c0c     libucrt:lseek.obj
 0003:00000c18       $pdata$_putwch_nolock      0000000180019c18     libucrt:putwch.obj
 0003:00000c30       $pdata$fclose              0000000180019c30     libucrt:fclose.obj
 0003:00000ea0       $pdata$fclose$fin$0        0000000180019ea0     libucrt:fclose.obj
 0003:00000c24       $pdata$_fclose_nolock      0000000180019c24     libucrt:fclose.obj
 0003:00000c48       $pdata$__dcrt_lowio_ensure_console_output_initialized 0000000180019c48     libucrt:initcon.obj
 0003:00000c60       $pdata$__dcrt_write_console_w 0000000180019c60     libucrt:initcon.obj
 0003:00000c54       $pdata$__dcrt_terminate_console_output 0000000180019c54     libucrt:initcon.obj
 0003:00000c78       $pdata$_close              0000000180019c78     libucrt:close.obj
 0003:00000c84       $pdata$_close_nolock       0000000180019c84     libucrt:close.obj
 0003:00000c6c       $pdata$??$?RV<lambda_751a882b2c74d4b022dec766aa51a29a>@@AEAV<lambda_628dfdc04ba53c8bfc02c9951375f3f5>@@V<lambda_f6c7be5f7998530c34de24c7437d6b54>@@@?$__crt_seh_guarded_call@H@@QEAAH$$QEAV<lambda_751a882b2c74d4b022dec766aa51a29a>@@AEAV<lambda_628dfdc04ba53c8bfc02c9951375f3f5>@@$$QEAV<lambda_f6c7be5f7998530c34de24c7437d6b54>@@@Z 0000000180019c6c     libucrt:close.obj
 0003:00000c90       $pdata$_call_matherr       0000000180019c90     libucrt:libm_error.obj
 0003:00000c9c       $pdata$_exception_enabled  0000000180019c9c     libucrt:libm_error.obj
 0003:00000ca8       $pdata$_handle_error       0000000180019ca8     libucrt:libm_error.obj
 0003:00000cb4       $pdata$__acrt_initialize_fma3 0000000180019cb4     libucrt:fma3_available.obj
 0003:00000ccc       $pdata$_log_special_common 0000000180019ccc     libucrt:log_special.obj
 0003:00000cc0       $pdata$_log10_special      0000000180019cc0     libucrt:log_special.obj
 0003:00000cfc       $pdata$_set_errno_from_matherr 0000000180019cfc     libucrt:fpexcept.obj
 0003:00000ce4       $pdata$_raise_exc          0000000180019ce4     libucrt:fpexcept.obj
 0003:00000cf0       $pdata$_raise_exc_ex       0000000180019cf0     libucrt:fpexcept.obj
 0003:00000d08       $pdata$_clrfp              0000000180019d08     libucrt:fpctrl.obj
 0003:00000d14       $pdata$_ctrlfp             0000000180019d14     libucrt:fpctrl.obj
 0003:00000eac       $pdata$_ctrlfp$filt$0      0000000180019eac     libucrt:fpctrl.obj
 0003:00000d2c       $pdata$_statfp             0000000180019d2c     libucrt:fpctrl.obj
 0003:00000d20       $pdata$_set_statfp         0000000180019d20     libucrt:fpctrl.obj
 0003:00000d38       $pdata$_IsNonwritableInCurrentImage 0000000180019d38     LIBCMT:pesect.obj
 0003:00000eb8       $pdata$_IsNonwritableInCurrentImage$filt$0 0000000180019eb8     LIBCMT:pesect.obj
 0003:00000d50       $pdata$__GSHandlerCheckCommon 0000000180019d50     LIBCMT:_gshandler_.obj
 0003:00000d44       $pdata$__GSHandlerCheck    0000000180019d44     LIBCMT:_gshandler_.obj
 0003:00000d8c       $pdata$__report_securityfailure 0000000180019d8c     LIBCMT:gs_report.obj
 0003:00000d80       $pdata$__report_rangecheckfailure 0000000180019d80     LIBCMT:gs_report.obj
 0003:00000d74       $pdata$__report_gsfailure  0000000180019d74     LIBCMT:gs_report.obj
 0003:00000d98       $pdata$capture_current_context 0000000180019d98     LIBCMT:gs_report.obj
 0003:00000da4       $pdata$capture_previous_context 0000000180019da4     LIBCMT:gs_report.obj
 0003:00000d68       $pdata$__raise_securityfailure 0000000180019d68     LIBCMT:gs_report.obj
 0004:00000504       .idata$6                   000000018001a504     kernel32:KERNEL32.dll
 0004:00000520       .idata$6                   000000018001a520     user32:USER32.dll
 0005:00000060       $R000000                   000000018001b060     Brackets.res
